:020000040000FA
:107800005469616E59696E673130300000000000C4
:1078100054593230302E303830303030625F747925
:10782000424154333247313339474B3634464200B4
:1078300043414E5F5354440000000000000000002C
:1078400043414E5F43485F300000000000000000ED
:1078500043414E5F3530304B6270730000000000D2
:107860009407000014070000DF070000000000007C
:020000040000FA
:1080000098330020E9800000F1800000F380000038
:108010000000000000000000000000000000000060
:10802000000000000000000000000000FB800000D5
:108030000000000000000000FF800000DDCE010015
:10804000E91601002D1701005D1701008D170100D1
:10805000BD170100ED1701001D1801004D180100AA
:108060007D180100AD180100E1180100F5180100AC
:1080700005190100391901004919010059190100B8
:108080008D190100D1190100191A0100611A0100AE
:10809000A91A0100F11A0100011B0100351B0100A2
:1080A000691B0100991B0100CD1B0100011C01008F
:1080B000111C0100211C0100551C0100891C01003C
:1080C000EF72E8FF03B40148019001BD897F0020F1
:1080D0000448854600F02CFA00480047A913020026
:1080E000C046C046983300201648804716480047CF
:1080F000FEE7FEE7FEE7FEE7FEE7FEE7FEE7FEE758
:10810000FEE7FEE7FEE7FEE7FEE7FEE7FEE7FEE747
:10811000FEE7FEE7FEE7FEE7FEE7FEE7FEE7FEE737
:10812000FEE7FEE7FEE7FEE7FEE7FEE7FEE7FEE727
:10813000FEE7FEE7FEE7FEE7FEE7FEE7FEE7FEE717
:10814000FEE70000FDD40100D180000030B50B46F1
:10815000014600202022012409E00D46D5409D4221
:1081600005D31D469540491B2546954040191546A7
:10817000521E002DF1DC30BD70B5002425460028CC
:1081800001DA01244042002901DA01254942FFF7C2
:10819000DDFFAC4200D04042002C00D0494270BD0F
:1081A000F0B51FB40646002082B005464024019178
:1081B00000901BE0019922460F46304600F066F918
:1081C000049A059B801A994110D3104619462246FD
:1081D00000F04CF9361A8F41019722460120002108
:1081E000009F00F043F938184D4100902046641E6E
:1081F0000028DFDC019B00982946324607B0F0BD1D
:10820000F0B51FB486B0002000900190029006984F
:10821000069980B204900798090C020400141143D7
:1082200007900027089D099806913E463C4603901A
:108230000398A9B20204000C039004982D0C154376
:1082400048430021224600F011F9C719714110344A
:108250000E46402CECDB3846029A00F007F9009AF3
:10826000019B8018009059410298019110300290B2
:108270004028CCDB00980BB0F0BD03460B439B07B6
:1082800003D009E008C9121F08C0042AFAD203E08B
:108290000B780370401C491C521EF9D27047D2B2B1
:1082A00001E00270401C491EFBD270470022F6E735
:1082B00010B513460A4604461946FFF7F0FF20465C
:1082C00010BD30B504460020034600E05B1C93421D
:1082D00003D2E05CCD5C401BF8D030BD0321001D13
:1082E000401E037812021A43491EF9D51046704702
:1082F000034603220870000A491C521EFAD518468C
:108300007047024670B54A40D30FDB0740002DD0BE
:108310004A002AD0010E140E000212020919400A66
:10832000520A8418E50104465443000A120A2E0436
:108330005043A4194219200CC543AA18120C012558
:10834000AD03521C521912047F39240400D0521C70
:10835000104301D44000491EC2B20C06C0092018C7
:10836000401C4008802A02D003E0002070BD400875
:108370004000002900DA0020184370BD70B50246A5
:108380004A40D50F40004A00ED0740085208002837
:1083900014D0002A12D0C40DD30D41020120C00513
:1083A0005202490A520AE41A091812187D349142FD
:1083B00001D3641C00E04900002C01DA002070BDEC
:1083C0000023914201D3891A034340084900002841
:1083D000F7D100290AD0914202D10121C90705E055
:1083E000914201D2012101E00121C943E005C018F9
:1083F000401900F05CF870BD10B5002296231146BC
:1084000000F05DF810BDC20FD207400040080BD04D
:10841000C10D0723DB01C91840020905400A1143B9
:10842000C208400711437047002001467047000012
:1084300010B5002904DB0124E40740428C412146A9
:10844000002B04DB1C460123DB075242A341994267
:1084500000D1904210BD00000122D207002800DBAD
:10846000101A002900DB511A8842704710B5202AE3
:1084700004DB0146203A9140002010BD91402023AA
:108480009C1A0346E3401943904010BD10B5202AC2
:1084900004DB0846203AD040002110BD0B46D340F3
:1084A000D0402024A21A91400843194610BD00294B
:1084B00004DA401C490001D140084000704770B404
:1084C0000024050C05D11024000402D1002921D07C
:1084D0001124050E01D100020834050F01D100015D
:1084E000241D850F01D18000A41C002801DB400061
:1084F000641C002908D020252E1B0D46F540A14004
:1085000000D001212943084301061B1B000ADB1D83
:1085100002D5002070BC7047DB05181880180029B0
:10852000F8DA401C4900F5D170BC400840007047A3
:10853000064C0125064E05E0E36807CC2B430C3CB6
:1085400098471034B442F7D3FFF7C6FD0028020065
:108550003028020070B58C180578401C6B075B0F43
:1085600001D10378401C2A1106D10278401C03E097
:1085700006780E70401C491C5B1EF9D12B0705D4F0
:108580000023521E0DD40B70491CFAE70378401CDF
:10859000CB1A921C03E01D780D70491C5B1C521E07
:1085A000F9D5A142D8D3002070BD70B507F0F8F915
:1085B0000524204618F0B2FE0025284607F0E6F90B
:1085C000204618F0ABFE0126304607F0BDF92046E4
:1085D00018F0A4FE284607F0B7F9204618F09EFED2
:1085E000304607F0D3F9204618F098FE70BDB0B5BC
:1085F00007F0D6F90524204618F090FE01252846FC
:1086000007F0C4F9204618F089FE284607F09CF9C7
:10861000204618F083FE002007F096F9204618F057
:108620007DFEB0BDF0B581B007F0A8F9052018F0C7
:1086300075FE08270026012007F086F9052420464C
:1086400018F06CFE204618F069FE07F08DF905461B
:10865000204618F063FE002007F076F9204618F057
:108660005DFE76002E437F1E3806E4D1F0B201B0E5
:10867000F0BD70B50446002007F066F907F090F9E8
:10868000052018F04BFE0826E0B2C00907F07EF97D
:108690000525284618F042FE012007F055F9284626
:1086A00018F03CFE002007F04FF9284618F036FE7F
:1086B000284618F033FE6400761E3006E4D105200B
:1086C00018F02CFE012070BDF0B583B00193144664
:1086D0000E460746012038430290032504E000F0CF
:1086E0008EF86D1E280631D000F067F83846FFF787
:1086F000C0FF00F0A7F80028F1D13046FFF7B9FF1E
:1087000000F0A0F80028EAD100F057F80298FFF72F
:10871000B0FF00F097F80028E1D1019802280BD3B0
:10872000451E0026FFF77EFF2070FFF73EFF641C0A
:10873000761CF0B28542F5DCFFF774FF2070FFF77E
:1087400056FF00F05CF8202003B0F0BD102003B00D
:10875000F0BDF0B583B01C46009201910290032554
:1087600004E000F04CF86D1E280623D000F025F838
:108770000298FFF77EFF00F065F80028F1D101981C
:10878000FFF777FF00F05EF80028EAD1002C0CD04C
:108790000026009F3878FFF76CFF00F053F80028A0
:1087A000DFD1761C7F1CA642F4D300F028F8082005
:1087B00003B0F0BD102003B0F0BDB0B507F0F0F885
:1087C0000524204618F0AAFD0125284607F0BCF82C
:1087D000204618F0A3FD284607F0D8F8204618F0E8
:1087E0009DFD0025284607F0D1F8204618F096FD9B
:1087F000284607F0A9F8642018F090FDB0BDB0B588
:1088000007F0CEF80524204618F088FD00252846FC
:1088100007F09AF8204618F081FD284607F0B6F8D0
:10882000204618F07BFD0125284607F08DF82046EC
:1088300018F074FD284607F0A9F8642018F06EFDC2
:10884000B0BD0000B0B507F099F80524204618F037
:1088500065FD012007F078F8204618F05FFD0B4D0C
:1088600007F082F8044607F069F8002C02D06D1E6C
:108870002804F5D10525284618F050FD002007F002
:1088800063F8284618F04AFD2046B0BD33210000A9
:10889000034801780B2901D8491C01707047C04674
:1088A000832F002070B584B00025039502950195B3
:1088B000009507F043F80F20C6430E4C1036F1B276
:1088C000A0206A461023FFF744FF204618F026FD3B
:1088D000204618F023FD912EF0D3A020B0216A4647
:1088E0001023FFF736FF204618F018FD02480580D8
:1088F00004B070BD581B0000762F002070B502290F
:1089000002D2EB24E0B270BD891EEB250022134693
:1089100005E0401C5B1CDDB2A94225460EDB047855
:108920006C40154604E034466E1C072D3546F0D2E7
:108930006608E407F7D09A246640F4E7E0B270BD19
:10894000F0B591B00C91417810AA117083781B0298
:108950005918C37804792402E3181B0459180B0E24
:10896000D3700C0C94700D0A55700B910895691812
:10897000099409190A93C9180278D24389184279CF
:1089800083791B029A18C379047A2402E3181B0422
:108990009A188918130A0693C918130C0593C91855
:1089A0000792120E04928918827AC37A1B029A18CF
:1089B000037B0F90447B2402E3181B0498180918CA
:1089C000020A02928918020C019289180D910390F3
:1089D000000E0E9000200346014606E032409A4009
:1089E000D2B211435B1C082B0ED0012635469D40A8
:1089F0000746024602E07F1C042FEFD010ACE45D76
:108A00002542F8D0521CF6E70E9C0D980019C3B20F
:108A10000F98827B934205D0427A914202D1002086
:108A200011B0F0BD1021FFF769FF0C99CC72019ACB
:108A30008A72029A4A72039A0A72049ACA71059A51
:108A40008A71069A4A71079A0A710A9ACA70099A33
:108A50008A70089A4A700B9A0A7011B0F0BDF0B58E
:108A60008DB055220270002747720B784370CA7987
:108A7000059202728A790492C2714A7903928271D4
:108A80000A7902924271CA7A089242738A7A0192F2
:108A900002734E7AC6720C7A84720CAA13704D78E7
:108AA0002D02EB188D78C978090249190904CB18F1
:108AB000190E01711D0CC57009931B0A0B90837070
:108AC00038460A91D170079595700693537031021C
:108AD0000919089A1202019BD21812045118089120
:108AE00003990902029A8918059A1202049BD21866
:108AF0001204511805913D463A4605E02640AE4025
:108B000032436D1C082D0ED001242146A940034696
:108B1000064602E05B1C042BF0D00CAFFF5C394230
:108B2000F8D0761CF6E70B9B5A7209980699401804
:108B3000079940180A994018059A8018110A401898
:108B4000110C4018110E4018089A8018110A40188C
:108B5000110C4018110E4018563898731021184601
:108B6000FFF7CCFE0DB0F0BDF0B58FB00446FF208E
:108B7000E070A07060700F20C04302900F30207032
:108B8000704818F0CBFB70490868632801D864204E
:108B900008606E4F002038806D4E0190308008E0F4
:108BA0000B99814222D338881030388080B2A128B6
:108BB0006DD206F0C3FE3978A02003AA1023FFF778
:108BC00083FD30802028EED103AD0BA92846FFF7A6
:108BD000B7FEE97B8842E6D128785528E3D15D4885
:108BE000017800290298DBD10846D9E73888A02807
:108BF0004DD8C0B20021019105E006F09FFE3988F2
:108C0000C8B2A12943D2C1B2A02003AA1023FFF702
:108C10005BFD3080398810313980202837D103AD91
:108C200007A92846FFF78CFEE97B8842E5D1287822
:108C30005528E2D1474800780028029900D1014622
:108C400007988842D9D240490A68962151430B9A25
:108C5000824208D90818904219D30BA90E22204647
:108C6000FFF70BFBC9E78918814210D307A90E2231
:108C70002046FFF702FB0BA80A99818107980B9009
:108C800008980C9009980D9038880190B5E72078E5
:108C9000617809020818A178E278120251180904D3
:108CA0000818401C24D1002001903880A020B02159
:108CB00003AA1023FFF708FD3080202818D103AD48
:108CC0000BA92846FFF73CFEE97B884210D12878A3
:108CD00055280DD11F480078002800D102900B982C
:108CE0000299884204D20BA90E222046FFF7C5FA4A
:108CF0002078617809020818A178E27812025118E8
:108D000009040818401C0CD10020E072A0726072A7
:108D10002072E071A07160712071E070A0706070CD
:108D20002070019838802078617809020818A178AD
:108D3000E2781202511809040818074908603088BF
:108D40000FB0F0BD70110100702F0020762F0020B1
:108D50006C2F00206F2F00207C2F0020F0B581B0F9
:108D600000910646214800250570002A2ED01446A1
:108D7000C036631B71190F2008401022101A83425D
:108D800000D303461A480278102A01D0042A1AD1C7
:108D9000C809FE2707405F2F13D80127B843603862
:108DA000C0B29E3282420CD3009A5219C9B2DFB2CD
:108DB0003B46FFF789FC0F490880ED19A542D8D33F
:108DC00004E0082000E004200A49088009480188DE
:108DD0000020042902D0082900D00120034908708E
:108DE000411E8841400001B0F0BDC046822F0020E6
:108DF0006E2F0020802F00200A4A012313700A4A98
:108E000010700A4A11600A4A00211160042801D139
:108E100005218901102801D11D208101054801800B
:108E20007047C0466F2F00206E2F0020702F00204B
:108E30007C2F0020742F0020F0B587B0994D0026BC
:108E40002E80994B1B688B4224D1994C2188202974
:108E500025D1029000920196964C00272760964DEE
:108E6000964E2878062809D806F068FD2068401C30
:108E70002060B042F5D38D48042101802F70904CC2
:108E800020880107029B31D0884820210180854D30
:108E9000019E0BE0012040028449088006E003A8FF
:108EA000FFF762FE20808148802101807F48008892
:108EB0003F2807DD874988420BDC402812D08028F4
:108EC00010D010E004280DD008280AD0202809D09E
:108ED00009E001214A02904204D0C902884201D02F
:108EE00001E002262E80288807B0F0BDA128019E4F
:108EF00000D32780009A012A6A4D1ED1187B0128D1
:108F000056D1DF719F715F711F711F73587B0128EC
:108F100004D1DF729F725F721F725F7303AF3846B6
:108F20001946FFF79CFDF8732088002846D01038BA
:108F3000C1B2A02003AA102344E0002AB6D16148A0
:108F400001780029B2D002701878597809020818FF
:108F50009978DA7812025118090408185A490978E0
:108F6000002901D00F21C943884233D2274603ACE0
:108F700020461946FFF773FDE0733978A0201023CF
:108F80002246FFF7E6FB029A4849088008288DD15F
:108F90003888103038801078517809020818917894
:108FA000D2781202511809040818484908607DE770
:108FB000597B012911D10128A3D0A7E7A02003AA3A
:108FC00010230146FFF7C5FB384908803D4800994A
:108FD00001706BE70120C0025EE73D480078012880
:108FE00012D103AC20461946FFF739FDE073A020EB
:108FF000B02110232246FFF7ACFB2C49088008283B
:10900000E4D133480770E1E7187859780902081865
:109010009978DA7812025118090408182B4909685E
:10902000214A12685118884203D220484021018009
:10903000CCE725490978002901D00F21C94388428E
:109040002DD203AF384619461C46FFF708FDF873CA
:109050001B480178A02010233A46FFF77AFB1349FA
:1090600008800828B2D11649088810300880207876
:10907000617809020818A178E278120251180904EF
:1090800008181249086008490A6815215143FFF77A
:109090005DF800299AD101200D49087096E701205A
:1090A000C00291E7882F0020702F0020862F00201B
:1090B0006C2F00208C2F0020832F0020818D5B00DF
:1090C000762F0020782F00206F2F00207C2F00208B
:1090D000842F0020FF010000F0B585B00646434C08
:1090E0000027278004921018414A1288904241D2EA
:1090F00001910397404F0020029038603F4C404D53
:109100002078052809D806F019FC3868401C38601A
:10911000A842F5D3374804210180029820703948CD
:10912000018839480278102A01D0042A32D18819DE
:109130000346C033049C651A0F2404401020001B12
:10914000854200DB0546DC09603C01263002E7B2BF
:109150007F09052F12D3B443E6B29E32B242234CAC
:10916000039F0DD301984218D9B2EBB23046FFF7F6
:10917000F0FA05E01F482021018011E01B4C039FFD
:109180001C49088008280BD1E8B21E4A118808182B
:10919000108005E00120800216490880134C039FCF
:1091A000144800881F2809DD202813D001210A0255
:1091B00090420FD0890288420CD00CE0042809D0DC
:1091C000082808D10F4800880499884201D3022753
:1091D00000E001272780208802210143022902D1D3
:1091E000084900220A8005B0F0BDC046882F002043
:1091F000742F0020862F00208C2F0020832F00202A
:10920000818D5B00902F00206E2F0020F0B585B07F
:10921000044600200190042C6FD20CF09FFA002825
:1092200001D10CF01BFB0020009000BF0098401CF7
:1092300000900CF093FA03900398002803D048495B
:1092400000988842F2D30398002856D1042145485B
:109250000CF066FA4448454908802101444A515CB3
:109260004900404A505A41490A880121090300F047
:1092700055F902900120049020013D4940184078A2
:10928000002801D100264BE02001394940184078E0
:10929000012802D13548068842E0200134494018AF
:1092A000407802282AD12001401805792901304A46
:1092B000515C49002B4A505A2C490A880121090364
:1092C00000F02CF9064628012A49431828012849AC
:1092D00040180289280140180021C7683046B84765
:1092E00006462801224BC018C2882801C018817880
:1092F000304600F087F8064612E02DE020011C49B8
:1093000040184078032804D02001401840781328E2
:1093100004D1200116494018868801E000200490FD
:109320000498002818D02001124943182001104940
:1093300040180289200140183146C7680298B84792
:10934000019020010A4BC018C2882001C018817802
:10935000019800F057F80190019805B0F0BD0000A9
:1093600050C300000201002088130000FC00002010
:109370009C1E0200DC1E0200F8B505460E4614468F
:109380000020009001211C4801751C48007888438A
:109390001A490870084680780821084317498870E0
:1093A000002088710846007801210843134908709D
:1093B00008460572002717E010480078802108430E
:1093C0000E49087000BF0E48007D0028FBD0002029
:1093D0000B4908750948C0892080A41C0748C18929
:1093E0000098081800907F1CB742E5D331460098DA
:1093F000FEF7ACFE80B2F8BD406100400050044072
:109400004060004010B50346012908D1094CA41A58
:109410009C4202D99C18A0B20BE0064809E0022940
:1094200006D1934202DD9C1AA0B202E0002000E0C7
:10943000184610BDFFFF000010B504460121202092
:1094400002F08CF800203249087001213148017582
:10945000002031490875152017F048FC2C48807809
:10946000E17808432A4988700846807821780843C3
:10947000274988702078802806D108460079E1794C
:10948000490008432249087121488078E17A08435D
:109490001F498870A078002803D108460079087118
:1094A0000FE0A078012806D119480079602108430F
:1094B0001749087105E016480079802108431449CE
:1094C0000871134880792179084311498871084649
:1094D0008079617908430E498871207AC872607A70
:1094E0008872084600783821884309490870084680
:1094F00000786178C900084305490870A07A0873AC
:1095000008460078012108430149087010BD000099
:10951000005004404061004040600040F8B50446FF
:109520000E461746002E01D100250FE0A64201DCB1
:109530003D460BE00094009C204678430090314665
:109540000098FEF703FE0090009885B22846F8BD0B
:109550000146042904D28A00024BD218508800E048
:10956000002070473C2900200146042903D28A00CC
:10957000024B985C00E00020704700003C2900206E
:10958000FFB587B004460898844203DA0A988068D9
:10959000002802D12448019042E00898001B82B2C2
:1095A0000292002625460A98806800212F463A46F6
:1095B0003346049605910690FEF722FE05460E46B8
:1095C000002328463146029AFEF7EAFD05460E467C
:1095D000304600210A4649405040014302D012481B
:1095E00001901DE003950A98C068039DA84202D32C
:1095F0000020019014E00A98C1680398401A039073
:1096000009990398FEF7A2FD03900398000C00044B
:10961000002802D00448019002E0039880B2019033
:1096200001980BB0F0BD0000FFFF000010B5084826
:10963000007880218843064908700121054801759A
:10964000002005490875152017F050FB10BD0000DB
:10965000005004404061004040600040F8B50546BD
:109660000E4614461F4621462846FEF785FD80B269
:10967000F8BD0000FFB587B006460A98406800288C
:1096800001D1029035E00A980168406808180390FB
:10969000002534460021274603980695049105903D
:1096A00038462946049B059AFEF7AAFD04460D4656
:1096B0000A98406802460023019020462946FEF79A
:1096C0006FFD04460D46002320462946099AFEF701
:1096D00067FD04460D4628460749214000235940AE
:1096E0005840014303D00448C043029001E0A0B2B7
:1096F000029002980BB0F0BD0000FFFF10B5FE48CD
:1097000000688079030017F0D7FA07059ED8F5F4B2
:10971000F3F2F100F84800684079030017F0CCFA42
:109720000805138A2A8A468A638A13F00FFB0020F1
:10973000F1490968C873F04800684079401CEE4957
:10974000096848717DE0ED494969EB4A1268D27AAF
:10975000885C13F073FBE84800684079401CE649D8
:1097600009684871E44800684079401CE24909688A
:10977000487166E00AF002FA002810D113F05EFB8F
:10978000DD4800684079401CDB4909684871DA48C7
:1097900000684079401CD8490968487105E013F019
:1097A000FFFA0020D449096848714AE00AF0E6F956
:1097B000002811D1112013F041FBCF4800684079F7
:1097C000401CCD4909684871CB4800684079401C6D
:1097D000C9490968487105E013F0E2FA0020C6495A
:1097E000096848712DE00AF0C9F900281BD1C24868
:1097F0000068C07A401CC0490968C872BE48006849
:10980000C07ABE49097888420DDB0020BA49096850
:10981000C872B94909684862B74800688079401C35
:10982000B5490968887113F0BBFA0020B24909688C
:10983000487106E013F0B4FA0020AF490968487196
:1098400000BF00BF32E3AC480068407C002817D05E
:10985000AA48C068002803D0A848C16819208847D2
:109860000020A54909684862A34800688079401C27
:10987000A1490968887100209F49096848711BE067
:109880009D480068406A282807D29B480068406AC3
:10989000401C9949096848620EE000209649096811
:1098A0004862954800688079401C9349096888712E
:1098B0000020914909684871F8E28F4800684079B2
:1098C000030017F0F9F9080518A42FA44CA480A4EC
:1098D00013F03CFA002088490968C873864800687C
:1098E0004079401C84490968487197E0D4E2C7E296
:1098F00030E25DE194E0814949697F4A1268D27A99
:10990000885C13F09BFA7C4800684079401C7A49D7
:1099100009684871784800684079401C76490968B0
:1099200048717BE00AF02AF9002811D1012013F0D8
:1099300085FA714800684079401C6F490968487190
:109940006D4800684079401C6B490968487105E022
:1099500013F026FA00206849096848715EE00AF0B1
:109960000DF9002828D164490968C97A2422514395
:10997000634A12688918604A1268D27B885C13F0C7
:109980005DFA5D480068C07B401C5B490968C8738C
:1099900059480068C07B242814D357480068407990
:1099A000401C554909684871534800684079401C7B
:1099B00051490968487105E013F0F2F900204E4959
:1099C000096848712AE00AF0D9F8002818D14A48F5
:1099D0000068C07A401C48490968C8724648006857
:1099E000C07A4649097888420ADB00204249096862
:1099F000C872414800688079401C3F4909688871F5
:109A000013F0CEF900203C490968487106E013F0D4
:109A1000C7F9002038490968487100BF00BF45E216
:109A2000354800684079030017F046F90A0614B972
:109A30002BB948B978B995B913F088F900202E49A7
:109A40000968C8732C4800684079401C2A49096895
:109A50004871ABE029494969274A1268D27A885C83
:109A600013F0ECF9244800684079401C2249096849
:109A70004871214800684079401C1F4909684871B5
:109A800094E00AF07BF8002811D14A2013F0D6F9AF
:109A9000194800684079401C174909684871164800
:109AA00000684079401C14490968487105E013F0CA
:109AB00077F9002010490968487177E00AF05EF8EC
:109AC000002824D1FF2013F0B9F90B480068C07BAF
:109AD000401C09490968C87307480068C07B2428EE
:109AE0001BD3054800684079401C03490968487148
:109AF00001480068407905E0E8070020542F002065
:109B0000E4070020401CEA490968487105E013F0A9
:109B100047F90020E6490968487147E00AF02EF845
:109B2000002811D1FF2013F089F9E148006840793D
:109B3000401CDF4909684871DD4800684079401CD5
:109B4000DB490968487105E013F02AF90020D8497B
:109B5000096848712AE00AF011F8002818D1D448A1
:109B60000068C07A401CD2490968C872D0480068B1
:109B7000C07AD049097888420ADB0020CC490968BC
:109B8000C872CB4800688079401CC949096888714F
:109B900013F006F90020C6490968487106E013F081
:109BA000FFF80020C2490968487100BF00BF7DE18D
:109BB000BF4800684079030017F07EF80C0715C312
:109BC0002CC349C366C382C39FC313F0BFF80020F0
:109BD000B7490968C873B64800684079401CB44961
:109BE00009684871B4E0B3494969B14A1268D27A48
:109BF000885C13F023F9AE4800684079401CAC49FA
:109C000009684871AA4800684079401CA849096859
:109C100048719DE009F0B2FF002811D1772013F0C0
:109C20000DF9A34800684079401CA14909684871B2
:109C30009F4800684079401C9D490968487105E0CB
:109C400013F0AEF800209A490968487180E009F0E5
:109C500095FF002811D10C2013F0F0F8944800680B
:109C60004079401C924909684871914800684079E0
:109C7000401C8F490968487105E013F091F80020F5
:109C80008B490968487163E009F078FF002810D11A
:109C900013F0D4F8864800684079401C844909686C
:109CA0004871834800684079401C814909684871BF
:109CB00005E013F075F800207D490968487147E018
:109CC00009F05CFF002811D1132013F0B7F8784891
:109CD00000684079401C76490968487174480068FA
:109CE0004079401C72490968487105E013F058F842
:109CF00000206F49096848712AE009F03FFF0028F9
:109D000018D16B480068C07A401C69490968C8725C
:109D100067480068C07A6749097888420ADB0020F2
:109D200063490968C872624800688079401C6049CC
:109D30000968887113F034F800205D49096848719A
:109D400006E013F02DF8002059490968487100BF5A
:109D500000BFABE0564800684079030016F0ACFF46
:109D6000080513872A874787638712F0EFFF0020D3
:109D70004F490968C8734E4800684079401C4C49F7
:109D8000096848717AE04B494969494A1268D27AB0
:109D9000885C13F053F8464800684079401C4449F9
:109DA00009684871424800684079401C4049096888
:109DB000487163E009F0E2FE002811D1492013F058
:109DC0003DF83B4800684079401C394909684871B2
:109DD000374800684079401C35490968487105E0FA
:109DE00012F0DEFF002032490968487146E009F0B0
:109DF000C5FE002810D113F021F82D4800684079E5
:109E0000401C2B4909684871294800684079401C6A
:109E100027490968487105E012F0C2FF0020244973
:109E2000096848712AE009F0A9FE002818D12048E5
:109E30000068C07A401C1E490968C8721C48006846
:109E4000C07A1C49097888420ADB00201849096851
:109E5000C872174800688079401C154909688871E4
:109E600012F09EFF002012490968487106E012F0C6
:109E700097FF00200E490968487100BF00BF15E038
:109E800000200B4909688871094909684871062052
:109E900007490968C87009E012F082FF00200449F0
:109EA0000968487102490968887100BF00BF10BD88
:109EB000E8070020542F002010B56A480068407958
:109EC000030016F0F9FE090610C627C644C6608EC8
:109ED000C60012F03BFF634800684079401C6149AE
:109EE00009684871BCE0604949695E4A1268D27AE3
:109EF000885C12F0A3FF5B4800684079401C594918
:109F000009684871574800684079401C55490968FC
:109F10004871A5E009F032FE002811D17F2012F02F
:109F20008DFF504800684079401C4E4909684871CF
:109F30004C4800684079401C4A490968487105E06E
:109F400012F02EFF002047490968487188E009F0A7
:109F500015FE002810D112F071FF424800684079C8
:109F6000401C4049096848713E4800684079401CDF
:109F70003C490968487105E012F012FF0020394998
:109F8000096848716CE009F0F9FD002822D13548D4
:109F90000068C07A401C33490968C87231480068BB
:109FA000C07A3149097888420FDB00202D490968C1
:109FB000C8722C4800684079401C2A4909684871D9
:109FC000002028490968486208E0002025490968FE
:109FD000487103E0002023490968487112F0E0FE4F
:109FE0003EE020480068407C002816D01E48C0682B
:109FF000002803D01C48C16819208847002019494F
:10A0000009684862174909684871164909688871E2
:10A01000052014490968C8701AE012480068406AAF
:10A02000282807D20F480068406A401C0D4909687B
:10A0300048620DE000200B49096848620949096837
:10A040004871084909688871052006490968C8707F
:10A0500006E012F0A5FE002002490968487100BF21
:10A0600000BF10BDE8070020542F002010B50024C9
:10A07000F7480068807A01287ED1F5480068C079E9
:10A0800000287AD0F24800688079002804D001289E
:10A0900074D0022873D191E1ED480068007B242838
:10A0A0006ED2EB480068C07901287AD1002475E0AF
:10A0B000E7480068C07A24214843E6490968401807
:10A0C000E3490968097B415CE1480068C07A2422C1
:10A0D0005043E14A12688018DD4A1268127B805CA6
:10A0E000814229D0DA480068C07A24214843DA49FD
:10A0F00009684018D6490968097B415CD448006862
:10A10000C07A24225043D34A12688018D04A126879
:10A11000127B8154CE480068407B242805D3CC486C
:10A120000068007BCA4909684873C9480068007B19
:10A13000C7490968887308E0C5480068407B24283F
:10A1400003D20120C24909688871C1480068007BB8
:10A15000401CBF4909680873BD480068007B24287B
:10A1600008D3BB480068407B242803D20120B849AB
:10A1700009688871B64805E0D3E1CDE169E0BAE14C
:10A1800038E00EE00068007B242804D2B048006864
:10A190008079012800D103E0601CC4B2242C87D34D
:10A1A00056E0002413E0AA480068C07A24214843FE
:10A1B000A94909684018015DA5480068C07A2422B1
:10A1C0005043A44A126880180155601CC4B2242C64
:10A1D000E9D300209E490968487323209C490968F7
:10A1E000887301209A490968887124209849096870
:10A1F00008732DE0002096490968087394480068A8
:10A20000C07A401C92490968C87291480068C07AB7
:10A2100092490978884217DB8D480068007C012844
:10A2200004D102208A490968887106E00020884923
:10A230000968887186490968C871002084490968DD
:10A24000C872834909680874002081490968487107
:10A2500061E17F4800684079030016F02DFD080594
:10A2600013A62AA651A68EA601207949096808746A
:10A2700012F06CFD764800684079401C744909680A
:10A28000487199E075494969714A1268D27A885CC7
:10A2900012F0D4FD6E4800684079401C6C49096892
:10A2A00048716B4800684079401C694909684871E9
:10A2B00082E009F063FC00281BD165490968497BED
:10A2C000491CC8B212F0BAFD61480068407B604981
:10A2D0000968C8735E4800684079401C5C49096899
:10A2E00048715B4800684079401C594909684871C9
:10A2F00005E012F055FD00205549096848715BE002
:10A3000009F03CFC00282BD151490968C97A242264
:10A310005143504A126889184D4A1268D27B885CB2
:10A3200012F08CFD4A480068C07B401C484909680F
:10A33000C87347480068C07B45490968897B8842E3
:10A340001ADD434800684079401C4149096848715A
:10A350003F4800684079401C3D49096848710BE05E
:10A3600012F01EFD3A480068407B39490968C873FD
:10A3700000203749096848711EE009F0FFFB0028FA
:10A380000CD1334909688871242031490968C873A0
:10A390002F49096848732E490968887312F000FD37
:10A3A00000202B490968487106E012F0F9FC0020F2
:10A3B00027490968487100BF00BFACE02448006825
:10A3C0004079030016F078FC08050F8E268E4C8E1F
:10A3D000688E12F0BBFC1E4800684079401C1C4986
:10A3E0000968487185E01D494969194A1268D27A9D
:10A3F000885C12F023FD164800684079401C14491F
:10A4000009684871124800684079401C1049096881
:10A4100048716EE009F0B2FB002811D1492012F01A
:10A420000DFD0B4800684079401C094909684871D6
:10A43000074800684079401C05490968487105E0F3
:10A4400012F0AEFC002002490968487151E000009A
:10A45000E8070020E4070020E0070020542F002038
:10A4600009F08CFB002810D112F0E8FC9C48006831
:10A470004079401C9A4909684871994800684079B8
:10A48000401C97490968487105E012F089FC0020DA
:10A490009349096848712CE009F070FB00281AD133
:10A4A0008F480068C07A401C8D490968C8728C4882
:10A4B0000068C07A8B49097888420CDB0020884903
:10A4C0000968C872864909688871854909684871B0
:10A4D00083490968C87112F063FC0020804909684B
:10A4E000487106E012F05CFC00207D490968487163
:10A4F00000BF00BF0FE012F053FC0020784909684C
:10A500004871774909688871754909680873744901
:10A510000968C87200BFE2E00020714909688872CA
:10A52000DDE06F480068807A0228F4D16C4800684A
:10A53000007A002879D06A4800684079030016F054
:10A54000BBFB0B0711BB25BB41545EBB7590BB0029
:10A5500012F0FCFB624800684079401C60490968C1
:10A560004871B7E05F494969087812F067FC5C48B8
:10A5700000684079401C5A49096848715848006889
:10A580004079401C564909684871A3E009F0F6FA81
:10A59000002810D112F052FC514800684079401C4C
:10A5A0004F49096848714E4800684079401C4C4941
:10A5B0000968487105E012F0F3FB0020484909687A
:10A5C000487187E009F0DAFA002807D144480068AA
:10A5D0004079401C42490968487103E00020404925
:10A5E0000968487112F0DCFB74E012F0AFFB3C48E4
:10A5F00000684079401C3A49096848716AE0394965
:10A6000049690978491CC8B212F018FC344800683E
:10A610004079401C324909684871314800684079E6
:10A62000401C2F490968487154E054E009F0A6FA2B
:10A6300000280FD112F05CFB2949096888700120BD
:10A6400012F0D0FB264800684079401C2449096874
:10A65000487105E012F0A4FB002021490968487107
:10A6600038E01F480068807811280CD100201C4970
:10A6700009680872AA201A490968887000201849D8
:10A680000968487011E0164800684078401C144979
:10A6900009684870124800684078032805D309F01B
:10A6A0000DFB00200E490968487012F079FB00206C
:10A6B0000B49096848710DE012F072FB002008494F
:10A6C00009684871064909684870AA200449096860
:10A6D000887000BF03E0002001490968887210BD3E
:10A6E000E8070020542F0020F0B505460C4616461A
:10A6F0001F462088482806DA3A462946304605F0A3
:10A7000057F9012800D0F0BD2088C0002E502088C5
:10A71000401C208000BFF6E710B502469000074BB2
:10A72000C018405C002802D00320C04310BD0120A7
:10A730009300024C1B1958540020F7E7D02A002040
:10A7400070B5002508E06D1C1B48854202D20BF055
:10A75000B1F801E0002503E00BF000F80028F2D189
:10A7600000BF022100200BF007F8032100200BF0AE
:10A7700003F8052100200AF0FFFF072100200AF05E
:10A78000FBFF002408E00020A1000C4A5054A10067
:10A7900089184880601CC4B2042CF4D301200849F5
:10A7A000087000204870052088700020C870054897
:10A7B0000549088070BD000050C300003C290020FE
:10A7C000FE00002088130000FC000020F8B58D4832
:10A7D0000078030016F070FA060405163D5EFDFCD5
:10A7E0000EE10BF03BF800208649C870487008461F
:10A7F0008078002802D10320087002E002208149FD
:10A800000870FDE07F488078002804D07D4880787B
:10A81000401E7C4988700AF0A1FF00280BD10BF084
:10A820001DF800207749C8700846807800280FD1AD
:10A83000032008700CE07348C078401C7149C87050
:10A840000846C078052803D3052008700BF032F8BD
:10A85000D6E00AF083FF00280ED104216A480AF0EE
:10A860005FFF00206749C8704870684868490880E1
:10A870000420644908700CE06248C078401C6149BB
:10A88000C8700846C078052803D3052008700BF06F
:10A8900011F8B5E05B49497809015E4A515C49000D
:10A8A000594A505A5A490A8801210903FEF736FECF
:10A8B00000900125534840780001564940184078DF
:10A8C000002801D100243CE04E4840780001514965
:10A8D00040184078012802D14D48048831E04948A9
:10A8E000407800014B4940184078022812D1454970
:10A8F00049780901474A89180879FEF729FE044674
:10A90000404949780901434A89180879FEF72CFE25
:10A91000054616E03B48407800013E494018407823
:10A92000032806D0374840780001401840781328A3
:10A9300006D134484078000136494018848800E048
:10A940000025002D2FD02F484078000132494318B0
:10A950002C48407800012F49401802892948407846
:10A96000000140182146C7680098B84706462548A8
:10A9700040780001274BC018C28822484078000167
:10A98000C01881783046FEF73DFD06461D484078E8
:10A99000800022494018468001201A4949788900E0
:10A9A0001E4A50540AE000201649497889001B4A83
:10A9B00089184880134949788900505411484078D3
:10A9C000401C1049487008464078042809D301E02B
:10A9D00013E007E00AF042FF00200A494870032014
:10A9E00008700DE00AF0BAFE002803D101200549E5
:10A9F000087001E00AF05EFF02E0FFF7A1FE00BF71
:10AA000000BFF8BDFE0000200201002088130000F6
:10AA1000FC0000209C1E0200DC1E02003C290020DD
:10AA200010B50AF065FE002405E00020A100074AE9
:10AA30005054601CC4B2042CF7D3002004490870A1
:10AA40000520887003480449088010BD3C29002077
:10AA5000FE00002088130000FC00002010B5034613
:10AA6000002000F0D7F8002000F03AF9002000F0B4
:10AA7000AFF8002000F012F9002000F087F8002065
:10AA800000F0EAF800BF012000F0A2F8012000F079
:10AA900005F9002421E0002000F09AF8002000F0E1
:10AAA000FDF880201840002806D0012000F0B2F800
:10AAB000012000F015F905E0002000F0ABF80020BF
:10AAC00000F00EF900BF012000F082F8012000F034
:10AAD000E5F85806030E601CC4B2082CDBDB01202D
:10AAE00000F054F8012000F0B7F810BD30B503466F
:10AAF0000C46012000F08EF8012000F0F1F8002053
:10AB000000F066F8002000F0C9F8002000F03EF8E0
:10AB1000002000F0A1F800BF012000F059F801204A
:10AB200000F0BCF8002528E0002000F051F80020DB
:10AB300000F0B4F880201840002803D0012000F075
:10AB400069F802E0002000F065F88020204000282D
:10AB500003D0012000F0C4F802E0002000F0C0F8AB
:10AB600000BF012000F034F8012000F097F85806EB
:10AB7000030E6006040E681CC5B2082DD4DB01204C
:10AB800000F004F8012000F067F830BD00280ED076
:10AB90000E490978082211430C4A11700B492031E3
:10ABA000097808229143094A203211700DE00749C3
:10ABB000097808229143054A117004492031097827
:10ABC00008229143014A203211707047000304406B
:10ABD00000280ED00E490978102211430C4A11703A
:10ABE0000B492031097810229143094A2032117013
:10ABF0000DE00749097810229143054A1170044974
:10AC00002031097810229143014A20321170704797
:10AC10000003044000280ED00E4909780422114395
:10AC20000C4A11700B492031097804229143094ADA
:10AC3000203211700DE00749097804229143054A3A
:10AC4000117004492031097804229143014A2032CD
:10AC5000117070470003044000280ED00E49C979D6
:10AC6000022211430C4AD1710B492031C9790222C9
:10AC70009143094A2032D1710DE00749C979022276
:10AC80009143054AD17104492031C9790222914387
:10AC9000014A2032D17170470003044000280ED0D1
:10ACA0000E49C979012211430C4AD1710B49203157
:10ACB000C97949084900094A2032D1710DE0074994
:10ACC000C97949084900054AD17104492031C97937
:10ACD00049084900014A2032D171704700030440FD
:10ACE00000280ED00E49C979042211430C4AD171B3
:10ACF0000B492031C97904229143094A2032D1718C
:10AD00000DE00749C97904229143054AD1710449EC
:10AD10002031C97904229143014A2032D171704710
:10AD20000003044010B5F920FFF798FE3221424895
:10AD300005F080FE8820FFF791FE9020FFF78EFE41
:10AD40009820FFF78BFE08210846FFF7CFFEE8208A
:10AD5000FFF784FE12210846FFF7C8FEA020FFF788
:10AD60007DFE70210846FFF7C1FEA820FFF776FEA2
:10AD700070210846FFF7BAFEB020FFF76FFE702182
:10AD80000846FFF7B3FEB820FFF768FE002108462B
:10AD9000FFF7ACFEC020FFF761FE00210846FFF779
:10ADA000A5FEC820FFF75AFE00210846FFF79EFEC9
:10ADB000D020FFF753FE2F210846FFF797FED8203B
:10ADC000FFF74CFE2F210846FFF790FEE020FFF72B
:10ADD00045FE2F210846FFF789FE4020FFF73EFE83
:10ADE00000210846FFF782FE0A20FFF737FE002405
:10ADF00005E000210846FFF779FE601CC4B25A2C1A
:10AE0000F7DB00240AE000200C4908550C490855DE
:10AE10000C4908550C490855601CC4B25A2CF2DB89
:10AE20008120FFF71BFE0020084908708870C87059
:10AE30000871487010BD0000204E000064260020FC
:10AE4000BE2600201827002072270020D4000020F2
:10AE500000B58020FFF702FE00BD0000002004497D
:10AE600008700120034908700020487070470000F6
:10AE7000D9000020D400002000B548480078002800
:10AE80007AD046488078030015F016FF0604434A3E
:10AE9000535A687E414800794149085C3F49097925
:10AEA000404A515C884209D13C4800793E49085CDF
:10AEB0003A4909793D4A515C88421BD037480079AC
:10AEC0003749085C35490979364A50543348007986
:10AED0003549085C31490979344A50542F48C078C3
:10AEE000002803D004202D49887011E001202B494F
:10AEF00088700DE000202949C87008460079401C80
:10AF00000871084600795A2802DB00200871087091
:10AF100041E04020FFF7A2FD0220204988703AE07E
:10AF20001E4A11791079FFF7E1FD03201B49887053
:10AF300031E00A20FFF792FD0420184988702AE0CA
:10AF4000164A1279194B995C144A1279154B985C80
:10AF5000FFF7CCFD0520114988701CE00F480079EF
:10AF6000401C0E490871084600795A2805DB00206C
:10AF700008710870C87003E00EE001200749C8702E
:10AF800000200649887006E0002004490870887097
:10AF9000C870087100BF00BF00BD0000D4000020D1
:10AFA00064260020BE2600201827002072270020DB
:10AFB00010B512F011FB01281ED101F093FD1149CB
:10AFC000884212D3072009F003FC002806D04B2248
:10AFD000D2000021012014F02DF812E07D22D200D1
:10AFE0000021012014F026F80BE07D22D200002180
:10AFF000012014F01FF804E000221146012014F093
:10B0000019F810BDB80B0000002003490872487001
:10B010008870486070470000680A0020582211526A
:10B02000704710B504460121022000F097FA002174
:10B03000022000F093FA10BD014600205322525C1A
:10B0400010231A40002A08D05322525C0C231A40C5
:10B050009210032A18D1032016E05422525A0123D9
:10B06000DB031A40002A0ED05322525C0C231A40F4
:10B070009210032A05D05322525C9207920F032AA2
:10B0800001D1022000E00120704702460020582331
:10B090009B5A0B40002B01D0012000E0002070479C
:10B0A000014600226020405AFF231B021840000581
:10B0B000020F1001014BC0187047000000550440FA
:10B0C00010B5002A0AD056231B5A0C0223435624DB
:10B0D000235256231B5A8B43235209E056231B5AF3
:10B0E0000C02A3435624235256231B5A0B432352CC
:10B0F00010BD0000F8B504460D460127002634486F
:10B10000844203D10121022000F028FA2878401E51
:10B11000A0702088FF21013108432080208840084A
:10B1200040002080A878401EC1B25A20015568799D
:10B130000007000CE97909020843A97908435C215A
:10B140000853288981B240200153A868C000C10C6F
:10B1500042200153A88981B244200153E868C0000D
:10B16000C10C46200153288A81B248200153286926
:10B17000C000C10C4A200153A88A81B24C2001535F
:10B180006869C000C10C4E2001535020005B297932
:10B1900009020843502108535020005B2979884355
:10B1A0005021085300E0761C5020005B4007400F00
:10B1B0002979884202D007488642F4D15020005BAA
:10B1C0004007400F2979884200D000273846F8BD53
:10B1D00000540440FFFF000030B5034600201C89E6
:10B1E0008C4209DD082A05D218244C431D682C190D
:10B1F000A05C02E0002000E0002030BD10B5024657
:10B2000013898B4205DD18234B431468E318987C9F
:10B2100000E0002010BD0146FF22C889C007C00F12
:10B2200000280AD00120C88100E0521EC889C0074A
:10B23000C00F002801D0002AF7D1C889C007C00F6D
:10B2400000280FD10220C8810420C881487A400814
:10B2500040004872487A3823984348720020487268
:10B26000012070470020FCE70246507A0123184372
:10B270005072507A0B78DB0018435072087A01281C
:10B2800008D1888850814868000C0123DB031843EB
:10B29000908108E0087A002805D150814868800034
:10B2A0001A4B18409081487A012804D1507A4023E3
:10B2B0001843507206E0487A002803D1507A4023A0
:10B2C000984350720878002811D1C87A1072087B10
:10B2D0001070487B5070887B9070CB7BD370087C5B
:10B2E00010714B7C5371887C9071CB7CD371887AC0
:10B2F000002803D00120C002D08101E00820D081C5
:10B30000FF200130D081012070470000FC1F0000A9
:10B31000002904D0427A80231A43427203E0427A21
:10B3200080239A434272704730B5024600200F4B8B
:10B330005024A45A0D022C435025AC525024A45A38
:10B340008C43AC5200E05B1E5024A45A6407640F87
:10B350008C4201D0002BF6D15024A45A6407640F0C
:10B36000002C01D0002000E0012030BDFFFF0000D4
:10B37000827A80231A40802A00D0817270470000B0
:10B3800070B5044600250023002D02D00126602060
:10B3900006530420C88188890126F603304000281E
:10B3A00008D0012010728889C004C0084E8930433B
:10B3B000506006E00020107288890F4E30408010E7
:10B3C0005060087AD072002304E0CE5C10460C3046
:10B3D000C6545B1CD07A9842F7DCC88904263040FA
:10B3E000002804D1C889F6023040002801D000208E
:10B3F00070BDD07AFCE70000FC1F0000002002496D
:10B400000880024908807047780000207A000020F8
:10B4100010B5A0210848FCF749FF074807494860D4
:10B42000074B05220749054800F037FE0021034875
:10B4300000F00AF810BD0000300900207408002058
:10B4400051B700002C1A0200027C80231A40802A87
:10B4500000D00174704710B50246FF23D089C007A1
:10B46000C00F002802D00120D0815B1ED089C00708
:10B47000C00F002801D0002010BD507A01242043C5
:10B480005072507A3824A0435072C87A1072487AA9
:10B4900000280FD1087B1070487B5070887B90701B
:10B4A000CC7BD470087C10714C7C5471887C90717A
:10B4B000CC7CD471FF200130D0814000D081107A43
:10B4C000DAE70000FFB581B004460D460020012CEC
:10B4D00003D140262E43304306E0002C00D103E088
:10B4E000022C01D1C0263043012A06D1049E7600E9
:10B4F00010273E430643F0B206E0002A00D103E0E5
:10B50000022A01D130263043134E307076788027DE
:10B51000BE43114F7E70012C08D1FF2100BF0E4E9B
:10B52000B3781E460E4033468B42F8D10A4E7678E9
:10B530004027BE43084F7E70012A0BD1002600969B
:10B5400003E000BF009E761C0096FF276937009E2F
:10B55000BE42F6D905B0F0BD00040240002905D076
:10B56000054A12780243044B1A7004E0024A12782A
:10B570008243014B1A70704720040240002905D015
:10B58000054A927E0243044B9A7604E0024A927E78
:10B590008243014B9A7670470008024070B503461B
:10B5A00014460020002B01D1C0B202E005468035D0
:10B5B000E8B2012902D1051DE8B206E0022903D153
:10B5C00005460835E8B200E0C0B2012C02D1851C66
:10B5D000E8B200E0C0B2084DA870AD78012635434E
:10B5E000054EB570002201E000BF521C7D252D01E3
:10B5F000AA42F9D970BD0000000C024070B50024C9
:10B600002448007920210840002801D0224D3FE045
:10B6100000F046F8054621480078802108400028BF
:10B6200036D01E4880780840002801D01A4D02E02C
:10B6300000F036F80546194880780007840F022C80
:10B6400001DBAD0804E0012C01D16D0800E000BF72
:10B65000124880788007C00F002801D02D0101E03A
:10B660000C2045430D4800784007840F002C02D180
:10B67000601CC4B207E0032C03D1601C4006040E1A
:10B6800001E06006040E21462846FCF75FFD0546F2
:10B69000284670BD0004024000127A00000C0240EF
:10B6A00000B5C0229178F82211401C4A127811434B
:10B6B000EA2923D00ADC0A46E03A130015F0FCFA26
:10B6C0000A181C20242A2A2A2A161A2AED291FD0F1
:10B6D00004DCEB2916D0EC291CD117E0F02903D0AB
:10B6E000F82917D10E4817E00E4815E00E4813E070
:10B6F0000E4811E00E480FE00E480DE00E480BE03A
:10B700000E4809E00E4807E00E4805E00E4803E049
:10B710000E4801E00D4800BF00BF00BD201C0240E4
:10B720000090D003006CDC020048E80100366E0196
:10B730000024F400001BB70000127A00808D5B002B
:10B7400000093D00C0C62D0080841E0040420F004D
:10B7500070B586B004460025002620680290A179C5
:10B760006846C1736179417300210173017100BFA3
:10B7700005E020460830415D04A841556D1C68462F
:10B78000C07BA842F5D80B22D2010299881A9142B7
:10B7900037D007DC2C48081A1FD023210901401A92
:10B7A00048D113E0FF386F38002802D0012841D17A
:10B7B00005E001A92548FFF74EFE06463BE001A93A
:10B7C00022484030FFF747FE064634E001A91F48F3
:10B7D0005030FFF740FE06462DE001A91B482030FF
:10B7E000FFF739FE06461A480088072805DA184888
:10B7F0000088401C1649088002E000201449088097
:10B8000019E005F0A1FD002813D012480178007856
:10B81000401C104A1070022906DC01A90B48603058
:10B82000FFF719FE064604E000200A4908700A499D
:10B83000087000E000BF00BF002E02D1012006B05A
:10B8400070BD0020FBE7000020020000805504408E
:10B850007A00002076000020F000002010B5A8211A
:10B860000A48FCF723FD094809490860094848606F
:10B87000072008810020887207220649044800F04A
:10B880008FFA00210248FFF773FD10BD88080020E1
:10B8900068080020B81A02000C4A127812060B4BF6
:10B8A0005B781B041A43094B9B781B021A43074B16
:10B8B000DB781A43104642084240D20083085A40BF
:10B8C0001146034A5140034A116070472B0700207C
:10B8D0000102000030070020F8B504460F46A07AA8
:10B8E0004006400E002874D10025ACE018206843C3
:10B8F00021680818407C01283CD1012118206843A8
:10B9000022681018017400260CE018206843216892
:10B9100008180830815D1820684322681018815586
:10B92000701CC6B2082EF0D300211820684322688C
:10B9300010180174182068432268101841741820E8
:10B940006843226810184161182068432268101863
:10B9500081742C20684361680818406A002809D067
:10B9600018236B432268D0182C236B436268D218CB
:10B97000516A884718206843216808184069FF21E8
:10B98000C94388425DD81820684321680818406977
:10B99000C1191820684322681018416118206843B3
:10B9A0002168081841692C20684362681018806972
:10B9B000814246D31820684321680818807C5528A6
:10B9C0003FD0552118206843226810188174002642
:10B9D00024E03CE01820684321680818805D2C2191
:10B9E0006943626851181031895D08401821694324
:10B9F0002268511888551820684321680818805D0E
:10BA00002C216943626851180831895D0843182167
:10BA10006943226851188855701CC6B2082ED9D3C4
:10BA20002C20684361680818806A002809D0182310
:10BA30006B432268D0182C236B436268D218916A3A
:10BA40008847681C85B22089A84200DD4EE7F8BD12
:10BA500001200149087070478C00002010B5044691
:10BA6000002015F08DFC02284DD1FFF7C7FC2D48B2
:10BA70000078002802D101202A490870294800785E
:10BA8000012823D127484078401C26494870214688
:10BA90005A20FCF75BFB23494978884241D80020B3
:10BAA0002049487008468078401C88700846807895
:10BAB0000A2803D30020887002200870FFF79EFC3C
:10BAC00000F068F8002015F08BFC2AE0154800789B
:10BAD000022826D113484078401C1249487021465C
:10BAE0007D20C000FCF732FB0E494978884218D807
:10BAF00000200C494870FFF781FC00F04BF8002053
:10BB000015F06EFC0DE00748C078401C0549C87070
:10BB10000846C078042804DB0020C870087048700C
:10BB2000887010BD7200002000B587B00021684603
:10BB30000171042141710C480290411003910B499D
:10BB4000049105910A480690FFF788FE01A815F0B8
:10BB5000ABFC00F059FB00F033F80021054809F078
:10BB6000A7FF07B000BD0000FFFF1F00FFFFFF1F82
:10BB700029BE00000205000030B5034600201C89E4
:10BB80008C4204D94D015C686419626000E00220B7
:10BB900030BD000010B5002400BF09E01C20604348
:10BBA00005494018214682680448FFF7E5FF641CF8
:10BBB000052CF3D310BD00002C1A020074080020DD
:10BBC00010B5FF2002307249486000200872012041
:10BBD000087000204872012088726E48FFF71BFB36
:10BBE0006B496C48FFF740FB01216A48FFF790FB67
:10BBF00069486749486000200872012008700020E9
:10BC000048720120887263481030FFF704FB6049D6
:10BC100060481030FFF728FB01215E481030FFF725
:10BC200077FB5D48401E5A49486000200872012099
:10BC30000870002048720120887256485030FFF783
:10BC4000EAFA534953485030FFF70EFB012151489F
:10BC50005030FFF75DFB5048C1384D494860002027
:10BC6000087201200870002048720120887249483B
:10BC70004030FFF7D0FA464946484030FFF7F4FA23
:10BC8000012144484030FFF743FBFF201230404978
:10BC900048600020087201200870002048720120CE
:10BCA00088723C486030FFF7B6FA3949394860304D
:10BCB000FFF7DAFA012137486030FFF729FBFF2050
:10BCC00021303349486000200872012008700020AC
:10BCD0004872012088722F48A030FFF79CFA2C4947
:10BCE0002C48A030FFF7C0FA01212A48A030FFF706
:10BCF0000FFB29488F382649486000200872012030
:10BD0000087000204872012088722248E030FFF756
:10BD100082FA1F491F48E030FFF7A6FA01211D48AB
:10BD2000E030FFF7F5FA1D48194948600020087215
:10BD300001200870002048720120887215482030C8
:10BD4000FFF769FA124913482030FFF78DFA0121F5
:10BD500010482030FFF7DCFA1048CB300C4948601F
:10BD600000200872012008700020487201208872AB
:10BD700008483030FFF74FFA054906483030FFF7E2
:10BD800073FA012103483030FFF7C2FA10BD0000FA
:10BD9000942A0020105504400204000014070000FB
:10BDA000F0B50B46144643600481002136E00022C2
:10BDB00016E02C254D4346687519AD5C18274F4396
:10BDC0000668F619B5542C254D4346687519AD5CC7
:10BDD00018274F430668F6190836B554551CEAB2C1
:10BDE000082AE6D3002518274F430668F61935744C
:10BDF00018274F430668F619757418274F430668CD
:10BE0000F619B57418274F430668F619F574182704
:10BE10004F430668F61975614D1CA9B205898D421C
:10BE2000C5DC00258572F0BD70B50446606800F081
:10BE3000F5FD0546E27A23460C332946094800F011
:10BE4000B5FD09496068884204D00749CB3960686C
:10BE5000884206D1E17AA28890B222460C3203F0E1
:10BE6000E7F870BD68080020DF070000F8B5054658
:10BE700000262C46002C29D000BF03E00020A0554E
:10BE8000701CC6B2082EF9D305F00CF8C0000821CA
:10BE9000084007462078884338432070E079E02145
:10BEA00088430B4909884901E02211400843E071A9
:10BEB00004F0F8FF012801D1082000E00020C706A7
:10BEC000FF0EE079400940013843E071F8BD000001
:10BED0007A000020F8B505460026002700200090D3
:10BEE0002C46002C5BD000BF03E00020A055701C46
:10BEF000C6B2082EF9D305F0D3F800280DD005F00E
:10BF000017FA022809D106212548FFF777F95528A5
:10BF100003D005F0BFF8002803D100202070607026
:10BF200011E005F0D3F892307D21C900884204D891
:10BF300005F0CCF8923087B201E07D27FF0038048D
:10BF4000000E2070677005F0AFF900280DD005F0E5
:10BF5000F5F9022809D106211148FFF74FF95528B4
:10BF600003D005F09BF9002803D10020A070E070F9
:10BF700015E005F0AFF992307D21C900884205D85F
:10BF800005F0A8F9923080B2009002E07D20C00058
:10BF9000009000980004000EA0700098E070F8BDBA
:10BFA0006808002070B5054600262C46002C24D0D9
:10BFB00000BF03E00020A055701CC6B2082EF9D3C4
:10BFC00005F0C2F901280AD13120207001206070EB
:10BFD0005920A0700820E070002020710DE005F0CD
:10BFE000B3F9022809D13120207001206070592056
:10BFF000A0700820E0700120207170BDFEB50546DC
:10C0000000260020019001F079FD074604F07AFF38
:10C010000A210090FCF7B0F880B201902C46002C69
:10C0200018D000BF03E00020A055701CC6B2082E37
:10C03000F9D33802000E60713804000EA071E77168
:10C0400005F05AF8FF2802DDFF20A07002E005F09D
:10C0500053F8A070FEBDFEB50546002600200190F5
:10C06000002704F045FD64210090FCF785F880B2BC
:10C070000190002001F064FD87B22C46002C0BD00B
:10C0800000BF03E00020A055701CC6B2082EF9D3F3
:10C090003804000EA070E770FEBDFFB581B0044605
:10C0A0000F4600250026002000902760039820817D
:10C0B0000498E0600020207400BF9DE01C206843CD
:10C0C000216808586A01616888501C20684321680B
:10C0D000081880686A016168891848601C206843F4
:10C0E0002168081840686A016168891888601C2006
:10C0F000684321680818C0686A0161688918C860C7
:10C100001C20684321680818007C6A01616889184E
:10C1100008741C20684321680818407C6A01616823
:10C12000891848741C20684321680818807C6A01BB
:10C130006168891888831C20684321680818C07CBE
:10C140006A0161688918887400206A016168891829
:10C15000C8741C206843216808184068002813D060
:10C160001C20684321680818C07C002805D1401EA7
:10C170006A0161688918C8831AE00020C0436A0117
:10C1800061688918C88313E01C2068432168081877
:10C19000C07C002805D000206A0161688918C88326
:10C1A00006E000206A0161688918C88301200090B8
:10C1B000002607E000216A0160688018143081556C
:10C1C000701CC6B2690160684018808BB042F1DC17
:10C1D0001C20684321680818406900280AD06B01B8
:10C1E0006268D218104614301C236B432268D218A0
:10C1F00051698847681CC5B22089A84200DD5DE707
:10C20000009805B0F0BD000000B58BB068480790FD
:10C21000002108A801706846017608A84170002036
:10C2200064498872082108A8C170002004E0002237
:10C2300009A90A54411CC8B208A9C9788142F6DC90
:10C240005D48FEF7E8FF06A95B48FFF70DF8584880
:10C25000401C0790002108A801706846017608A8D4
:10C260004170002053498872082108A8C17000203D
:10C2700004E0002209A90A54411CC8B208A9C978DF
:10C280008142F6DC4C484030FEF7C5FF06A94A481B
:10C290004030FEF7E9FF452000010790002108A883
:10C2A00001706846017608A84170002041498872F3
:10C2B000082108A8C170002004E0002209A90A543E
:10C2C000411CC8B208A9C9788142F6DC3A4850300E
:10C2D000FEF7A1FF06A938485030FEF7C5FF112030
:10C2E00040010790002108A801706846017608A85F
:10C2F000417000202F498872082108A8C1700020D1
:10C3000004E0002209A90A54411CC8B208A9C9784E
:10C310008142F6DC28482030FEF77DFF06A926483A
:10C320002030FEF7A1FF0B20C0010790002108A8D4
:10C3300001706846017608A8417000201D49887286
:10C34000082108A8C170002004E0002209A90A54AD
:10C35000411CC8B208A9C9788142F6DC1648603091
:10C36000FEF759FF06A914486030FEF77DFF10481C
:10C37000A6300290002168460173017141738173F8
:10C380000821C173002004E0002204A90A54411CC2
:10C39000C8B26946C97B8142F6DC07481030FEF717
:10C3A0003AFF01A904481030FEF75EFF0BB000BD54
:10C3B000EE060000942A002080550440F0B585B0B8
:10C3C00004460F4600250026207C4006400E5528D6
:10C3D0007ED100BF76E1690160684018807C00284A
:10C3E00077D169016068401840686A0161688918FE
:10C3F0008968884209D26901606840184068C0199C
:10C400006A016168891848605AE1690160684018EA
:10C41000C068AF49884208D8690160684018C068A0
:10C42000401C6A0161688918C86069016068401829
:10C43000C07C002821D1002607E000216A01606845
:10C44000801814308155701CC6B2690160684018AC
:10C45000808BB042F1DC1C206843216808184069D9
:10C4600000280AD06B016268D218104614301C23D1
:10C470006B432268D2185169884769016068405847
:10C480000090690160684018017C684601710021D4
:10C490004171690160684018017F684681716901D6
:10C4A00060684018417C6846C171002608E0690157
:10C4B000606840181430815D02A88155701CC6B2B6
:10C4C000690160684018808BB042F0DCE06801E0F0
:10C4D000FCE01DE0002806D06846E16888476A0154
:10C4E00061688918C874690160684018C07C0028B8
:10C4F00004D16A01616889184860E1E069016068F7
:10C5000040184068C01B6A01616889184860D7E01C
:10C5100069016068401880680028EED06901606891
:10C520004018C08B0028E8D0690160684018C08BB3
:10C530006A0161688918C968884207D16901606821
:10C540004018C08B6249C94388427DD16901606847
:10C55000401840686A01616889188968884209D270
:10C560006901606840184068C0196A0161688918EB
:10C570004860A5E000206A01616889184860690187
:10C5800060684018C0685249884208D869016068EC
:10C590004018C068401C6A0161688918C86000269C
:10C5A00007E000216A016068801814308155701C12
:10C5B000C6B2690160684018808BB042F1DC1C2073
:10C5C000684321680818406900280AD06B01626836
:10C5D000D218104614301C236B432268D2185169BC
:10C5E0008847690160684058009069016068401898
:10C5F000017C684601710021417169016068401841
:10C60000017F68468171690160684018417C684615
:10C61000C171002608E06901606840181430815D2E
:10C6200002A88155701CC6B2690160684018808BF1
:10C63000B042F0DCE068002808D06846E16888472E
:10C640006A016168891800E015E0C87469016068D2
:10C650004018C07C002804D16A01616889184860CC
:10C660002EE06901606840184068C01B6A0161687B
:10C670008918486024E01C20684321680818406835
:10C6800000280FD00020C0436A0161688918C88360
:10C690001C2068432168081840686A01616889188D
:10C6A000886008E000206A0161688918C8836A010F
:10C6B00061688918886000206A0161688918C8600B
:10C6C000681CC5B22089A84200DD84E605B0F0BD33
:10C6D0000000FFFF7CB500BF19212C480078FBF754
:10C6E00035FD04462A4860432A4A81180022012069
:10C6F0000DF03CFA20460A2250436430001981B202
:10C70000002201200FF0A4FA01200A22624312192C
:10C71000D1B20A22624312190090D0B201231A4604
:10C7200009F0DAFCFF220721002007F0BFF8012002
:10C73000009001900B20604382B20B20604381B2D5
:10C74000002301200EF0A0FF6F20604381B2012082
:10C750000FF024FD104860430246032101200BF036
:10C760007FFF002505E0012128460BF0B3FE681C81
:10C77000C5B20F2DF7DB21460B2251436431C8B2FD
:10C780000FF076FF0FF05EFF7CBD00006F00002011
:10C79000672B0000A0860100FCB1010000200549C4
:10C7A0000870054908700549087005490870054971
:10C7B0000870704770000020710000206F0000209A
:10C7C0006E0000206D000020F0B589B000BF00BFF2
:10C7D00000BF00BF00BF00BF00BF00BF00BF00BF61
:10C7E00000F080F91E2822D35D4800783C2805DA45
:10C7F0005B480078401C5A49087002E03C205849C8
:10C800000870574800781D2805DC56480078401C01
:10C81000544908700BE053480078002802D1514970
:10C82000087004E04F480078401E4E49087003210C
:10C830004C480078FBF7A0FC4B4948430390052186
:10C8400048480078FBF782FC0446032145480078FD
:10C85000FBF792FC0B214843643080B206904149BB
:10C8600009788A0088180621FBF786FCFF21F5313C
:10C87000484380B2079003213A480078FBF77CFCDC
:10C880000B214843643080B208900321354800787A
:10C89000FBF772FC354948433549401804900321A1
:10C8A00030480078FBF768FC0B2106464E43032115
:10C8B0002C480078FBF760FC0B2107464F4303210F
:10C8C00028480078FBF758FC6F21484380B2059058
:10C8D00003210120039A0BF0C3FEE1B201200BF00B
:10C8E0008BFCE1B201231846069A09F0CFFEFF2126
:10C8F000F5310798FBF740FCC0B2014602900120D9
:10C900000AF0A6FB0022012008990FF0A1F90022ED
:10C91000012004990DF02AF9012005990FF03EFC41
:10C920000120F9B20090F0B201231A46029009F0FA
:10C93000D3FBFF220721002006F0B8FF032109489E
:10C940000078FBF719FC0B21484385B201200090C9
:10C9500000232A46294601900EF096FE09B0F0BD4C
:10C960007100002070000020FCB10100672B000066
:10C97000A0860100002000BF06E00021044A1154F7
:10C98000044A1154411CC8B25A28F6DB7047000013
:10C9900064260020182700200348007A002801D1CF
:10C9A0000149487070470000680A0020FFB581B057
:10C9B00004460F463D462089A8422DDD18206843D5
:10C9C00021680818007C002826D1002609E0049878
:10C9D000815D182068432268101808308155701C4A
:10C9E000C6B2082EF3D3012118206843226810181C
:10C9F00041742C20684361680818006A00280BD035
:10CA000018236B432268D218104608302C236B433E
:10CA10006268D218116A884705B0F0BD0146072048
:10CA2000124BCA1A994211D008DCCA1FFA3A002ADE
:10CA300014D0102A0CD01F2A14D10DE0322A0FD0A6
:10CA4000C02A07D0C12A0DD100200DE001200BE043
:10CA5000022009E0032007E0042005E0052003E0B0
:10CA6000062001E0072000BF00BF7047410300001F
:10CA700010B504467D21C90061430846322103F008
:10CA8000D9FF10BDFF200B4908700020C0430A49A0
:10CA900008800A490880FF20094908700949087080
:10CAA00009490870002009490860094908600949D6
:10CAB00008607047540000205600002058000020F5
:10CAC0005A0000205B0000205C000020480000208D
:10CAD0004C00002050000020014800687047000012
:10CAE0004C0000200148006870470000480000200A
:10CAF00010B5054909886522514308466421FBF7B2
:10CB00003BFB80B210BD00005600002001480078B9
:10CB1000704700005B00002001480078704700006B
:10CB20005400002010B510F057FD01282CD100F062
:10CB300063F8012000F066F803F0E0FF044600F01F
:10CB400043F804F0BDF9044600F04AF804F01EFC76
:10CB5000012805D100F03EF8012000F047F805E07B
:10CB6000002000F037F8002000F040F800201349C2
:10CB7000086013480068134988421ED210480068B4
:10CB8000801C0F49086018E000200D4908600B4820
:10CB900000680C49884204D208480068801C074994
:10CBA0000860002000F028F8012000F02BF8002099
:10CBB00000F00AF8002000F013F810BD4C0000202F
:10CBC00048000020FFFFFF7F0149088070470000F8
:10CBD0005600002001490870704700005B000020EB
:10CBE0000149088070470000580000200149087082
:10CBF000704700005C000020014908707047000089
:10CC00005400002001490870704700005A000020BD
:10CC10000021014A11717047006000400022014963
:10CC20004A75704700600040002201494A7670470B
:10CC3000006000400021014A11727047006000400E
:10CC40000021014A11737047006000400021014A31
:10CC500011747047006000400021014A117570474F
:10CC6000006000400021014A1176704700600040DA
:10CC7000002201494A7370470060004000220149C8
:10CC80004A7470470060004010B51C4C1C49206875
:10CC900088421ED106221B49201DFBF712FB0028EB
:10CCA00017D11222184920460A30FBF70AFB002848
:10CCB0000FD10622154920461C30FBF702FB002845
:10CCC00007D10622124920462230FBF7FAFA002843
:10CCD0000DD000F059FF0A480E490860074814F0CB
:10CCE000B0FC0C4A2C21054814F0D6FC04E02C22A0
:10CCF00021460848FBF7C1FA10BD000000025000B1
:10CD00007AA7A55A41070020470700203B070020CB
:10CD100035070020A02E002000200849087008498F
:10CD2000087001200749087000200749087007486B
:10CD30000749086000200749087070472307002052
:10CD400022070020250700202A07002025060000D2
:10CD50005C0700203407002070B5044600BF912016
:10CD6000604305460A212846FBF7F0F905462846A8
:10CD700070BD000070B5A8B0054600240026A021B3
:10CD80006846FBF793FA00F06FFD1E490A6814210C
:10CD90006943505000211B48026814206843101852
:10CDA00041601848026814206843101881601548D3
:10CDB0004068002824D000BF17E06006060E282E29
:10CDC00000D316E00F480168142060430858B100F2
:10CDD0006A4650500B4801681420604308184168A7
:10CDE000701C80001150601CC4B20648007AA0423A
:10CDF000E3DC00BF620003486946436802209847AD
:10CE000028B070BD1C2F002030B5A9B0002400252B
:10CE1000A02101A8FBF74AFA00BF25E06006050E35
:10CE200000F022FD1F490A6814216143505000217F
:10CE30001C480268142060431018416019480268B9
:10CE40001420604310188160282D0BD2154801680A
:10CE5000142060430858A90001AA50500021681C02
:10CE600080001150601CC4B20E48007AA042D5DC8C
:10CE70000C484068002813D00A48007A400028284F
:10CE800006D30848282201A943680220984707E0F2
:10CE90000448007A4200034801A9436802209847E9
:10CEA00029B030BD1C2F0020FFB585B005460E46C9
:10CEB0001F460020049003900024029001900097E8
:10CEC000681C80004149085A0490002D05D0681E56
:10CED000800040184088039003E0A8003B49085AAE
:10CEE000039003990E98884205D304990E988842BE
:10CEF00001D80E9C08E0012E01D1049C04E0002E14
:10CF000001D1039C00E00E9C31480068052805D241
:10CF10002F480068401C2E49086053E000202C492F
:10CF2000086005210798FBF711F902900298002884
:10CF300044D028480068A04215D226480068201A2C
:10CF4000019002990198FBF701F9019021480168CD
:10CF5000019808181F49086008460068A04217D9C0
:10CF60000846046014E01B480068001B0190029909
:10CF70000198FBF7EBF80190164801680198081A30
:10CF80001449086008460068A04201D208460460BF
:10CF9000104800680090002E14D10E4800686330DD
:10CFA000B84201D300970DE064210A48006863305D
:10CFB000FBF7CCF864214843009003E00548046087
:10CFC00000680090009809B0F0BD00000A1E020041
:10CFD000C8000020D000002008B510F0FDFA01289C
:10CFE0007ED1FFF77FFD8D49884216D20F208C49F4
:10CFF0008871C87108468078002801D105204870E2
:10D0000087488078052802D1002085494870002093
:10D01000834948728872087047E0FA208049887115
:10D02000C8718049088803F091FE7E488078002806
:10D0300015D17B49087008468079C8700846C079C8
:10D040004871002088704870887276480088642192
:10D05000484375490860FA207149087125E00120AC
:10D060006F4908700846807A022805D1012088722D
:10D070000020C870487118E06948807A002814D1EF
:10D08000022067498872084640788870084680798F
:10D09000C8700846C07948716248008864214843D6
:10D0A00061490860FA205E490871FFF71BFD5B4982
:10D0B0001E3188427FD35A4880785949497888423E
:10D0C00029DD584800886421484355490090C979B2
:10D0D000534B5B79CA1A5249887853490B6800E070
:10D0E0008FE00021FFF7E0FE4F49086000204C4927
:10D0F000C870087108464079401C4871084640795C
:10D10000C97988425DDB002045494871084680782E
:10D11000401E887055E042488078414949788842ED
:10D1200027DA40480088642148433D4900908979C6
:10D130003B4BDB78CA1A3A4988783B490B68012196
:10D14000FFF7B2FE38490860002035494871087180
:10D150000846C078401CC8700846C0788979884263
:10D160002FDB00202E49C87008468078401C88704C
:10D1700027E000202A494871C87008460079401C01
:10D18000087108460079FA2801DBFA200871254861
:10D19000008864214843224900900979FA235A1AE9
:10D1A0001F49887820490B680221FFF77DFE1E4940
:10D1B000086006E0FFE71B480088642148431A49DD
:10D1C000086018488078002803D10120144948726B
:10D1D00023E003F0B3F8732803DB02201049487200
:10D1E0001BE003F0ABF8702803DC00200C49487208
:10D1F00013E00B48407A01280FD1002008494872FB
:10D200000BE000200649087008468079C87008467F
:10D21000C079487100204872887208BDB80B0000C0
:10D2200058260020C4000020CC0000200020044923
:10D2300088704870C87048714872887270470000E2
:10D24000582600200020064908808870054988700B
:10D250004870FA20C8704871002048728872704780
:10D26000C400002058260020F8B500240025002620
:10D27000002703F073FC044603F082FC054610F01F
:10D28000ABF901282ED105211A48FDF7B7FF552823
:10D2900004D1002018498870088027E0012D04D1AE
:10D2A000002015498870088020E00120124988700C
:10D2B0001248844202DB201A84B200E000240A21D2
:10D2C0002046FAF759FF052901DB601D84B20C489E
:10D2D000844200DD04460A212046FAF74DFF064944
:10D2E000088003E00020044988700880FFF774FE7E
:10D2F000F8BD000068080020C4000020AA0A000051
:10D30000C60700001CB500200090019000F0ACFAA8
:10D310000B49086000200B49096808600A4800684A
:10D3200000280CD00749096808680A21FAF70EFF9F
:10D330000090012269460520034B1B6898471CBDDD
:10D34000F8070020EC070020F4070020002008491F
:10D350004880084908800849088008490870084939
:10D3600088720849088048800120087170470000D1
:10D370002C0000201C0000201E00002020000020A7
:10D380004C08002024000020F8B503F0C9FB074634
:10D3900003F0D8FB0090FFF7BFFB012860D1052107
:10D3A000C548FDF72BFF552802D00098012807D16A
:10D3B0000020C2490870C2490880C249887256E0FC
:10D3C000BE480078002810D10120BC4908703D46B5
:10D3D0002846E917890F091889030D0CBA488542B8
:10D3E00000DD0546B648058041E0B648807A400039
:10D3F000B4490F520846867A0EE07000B1490D5AC2
:10D40000701E4000085A7100AE4A5052701E400013
:10D4100011460D52701EC6B2002E08DD7000A949DB
:10D42000095A701E4000A74A105A8142E5DBA54800
:10D43000807A401CA34988720846807A052816DB4A
:10D44000002088720846C5882846E917890F091800
:10D450008D109D48854200DD05469948058006E00F
:10D460000020964908709649088096498872944829
:10D47000058896480088A84257DA94480088281AF8
:10D4800084B292480079012827D190484088A04270
:10D490000BDA8E4840880A308C494880084640881C
:10D4A000A04204DD0846448001E088484480874863
:10D4B000448803212046FAF75FFE84B2192C00DA73
:10D4C000192482480088001980490880084600888D
:10D4D000A84201DD08460580CDE07C48408814283C
:10D4E00005DD7A48408814387849488002E00020F9
:10D4F000764948807548448803212046FAF73CFE67
:10D5000084B2192C03DA012070490871B3E06F4826
:10D510000088A04205DD6D480088001B6B4908802B
:10D52000A9E0002069490880A5E068480088A84271
:10D5300059DD66480088401B84B2644800790128A0
:10D5400027D162484088142805DD60484088143897
:10D550005E49488002E000205C4948805B4844887E
:10D5600003212046FAF708FE84B2192C03DA0220C0
:10D57000564908717FE055480088001953490880D2
:10D58000084600885049884275DD08464F490880A2
:10D5900071E04E484088A0420BDA4C4840880A307F
:10D5A0004A49488008464088A04204DD0846448035
:10D5B00001E0464844804548448803212046FAF764
:10D5C000DBFD84B2192C00DA19244048008829199F
:10D5D000884202DA3D4805804DE03C480088001B47
:10D5E0003A49088047E03948448803212046FAF741
:10D5F000C3FD84B2192C3EDD34484088142805DD73
:10D600003248408814383149488002E000202F49D0
:10D6100048802E48448803212046FAF7ADFD84B2A5
:10D620002A480079012813D1192C03DA022027494E
:10D63000087120E025480088001924490880084620
:10D6400000882149884216DD08462049088012E0FA
:10D65000192C03DA01201D4908710CE01B480088D1
:10D66000A04205DD19480088001B1849088002E027
:10D6700000201649088016480088502804DC13480A
:10D6800000881349088016E010480088104909886E
:10D69000884204DD0D4800880D4908800BE00B48E6
:10D6A00000880B490988081A84B2502C03DB07480C
:10D6B000008807490880F8BD680800202000002085
:10D6C0001C0000204C080020E02E00002400002058
:10D6D0001E00002010B5044664204443A1212046CA
:10D6E000FAF734FD0446204610BD000010B50120B5
:10D6F0000F49087000200F49096808600D49096842
:10D7000048600C490968886000F07EF9FFF7FAFD6F
:10D71000FFF77AFB08480068002807D00122054877
:10D72000016808310020044B1B68984710BD0000B9
:10D73000C5070020C0070020BC07002010B518480E
:10D7400000681849884229D117480068002804D089
:10D75000154800688047154908701548006800287A
:10D7600004D01348006880471249087012480068C6
:10D77000002804D0104800688047104908801048ED
:10D780000068002805D00E48006880470D490880D1
:10D7900002E00D480B49088000F078F810BD000049
:10D7A000D007002078563412AC070020C4070020B0
:10D7B000B0070020C6070020B4070020C8070020DB
:10D7C000B8070020CA0700201027000010B500236A
:10D7D000174C2360174C2370174C2370174C237081
:10D7E000174C2380174C2380174C2370174C136859
:10D7F0002360174C53682360164C93682360164CC3
:10D80000D3682360154C1369236000280CD0144B97
:10D810001860134C0B682468A3600023104C246824
:10D8200023600F4C246863600E4B014C236010BDD5
:10D83000D0070020CC070020C4070020C607002026
:10D84000C8070020CA070020C5070020AC07002039
:10D85000B0070020B4070020B8070020BC07002054
:10D86000C0070020785634120548006805498842F0
:10D8700003D105480068806870470020C043FBE77B
:10D88000D007002078563412C007002070B500245D
:10D89000002500263048007801285CD12F48007808
:10D8A000002858D12E480078012854D12D480588E9
:10D8B0002D490988694308462C49FAF747FC85B287
:10D8C000E1200001854207D8192169430846092152
:10D8D000FAF73CFC044600E0244C25480068006848
:10D8E0000019234909680860214800680068204938
:10D8F00009684968884207D31D48006800681C49C8
:10D9000009684968461A0AE0194800684068002119
:10D91000C943081A1649096809684018461C154881
:10D92000864218D3344601462046FAF70FFC0446D7
:10D930000F48006841680F48604308180C4909689F
:10D94000486001200C490870094800688068001987
:10D9500007490968886070BDC4070020C50700201A
:10D96000C6070020C8070020CA07002010270000B3
:10D97000C0070020A0860100CC07002000220C4B2D
:10D980001A600C4B0A681A600B4B4A681A600B4B02
:10D990008A681A600A4BCA681A600A4B0A691A60D8
:10D9A000002801D0084A1060084A014B1A607047ED
:10D9B000D0070020AC070020B0070020B4070020EB
:10D9C000B8070020BC070020C0070020785634129A
:10D9D00010B50A48006800280ED0094800780128D0
:10D9E0000AD1002006490870012206480168083162
:10D9F0000020024B1B68984710BD0000BC070020A8
:10DA0000CC070020C00700201CB50020009001902A
:10DA10000024FFF729FF04460E4800680460002038
:10DA20000C49096848600B49096888600A48006821
:10DA300000280DD00748006800680090054800687D
:10DA400040680190022269460120034B1B689847F9
:10DA50001CBD0000D4070020D8070020F8B50546FB
:10DA60000C4616460027002D17D00E480560FFF71C
:10DA7000FBFE07462068B84203D90A4800680760E1
:10DA800003E0084920680968086006496068096879
:10DA900048600449A0680968C8600348066000F04F
:10DAA00005F8F8BDD4070020D807002070B5002481
:10DAB0000025FFF7D9FE04460F4800680068A04221
:10DAC00000D903E00C4800680068251A0A4800687D
:10DAD00040684019084909688860074800688068FC
:10DAE00005490968C968884205D903480068C068C3
:10DAF00001490968886070BDD407002001480068AA
:10DB000080687047D4070020002801D0024A1060C6
:10DB1000024A116070470000D4070020D807002097
:10DB20000549002005E00A1D135C044A1354421CF9
:10DB3000D0B21528F7DB704700065000D02E002029
:10DB400001461048026814204843101882680D48A6
:10DB50000368142048431818C06882420BD909484A
:10DB60000268142048431018C2680648036814204D
:10DB7000484318188260034802681420484310186C
:10DB8000806870471C2F002010B500210022002063
:10DB900005E01B4B1C5C1B4B1C54431CD8B20628D5
:10DBA000F7DB1221002006E0174B1C5C154B9B1D78
:10DBB0001C54431CD8B28842F6DB002006E0134B0D
:10DBC0001C5C104B18331C54431CD8B20628F6DBDF
:10DBD000002006E00E4B1C5C0A4B1E331C54431CF9
:10DBE000D8B20628F6DB0422002005E00024054B0D
:10DBF00024331C54431CD8B29042F7DB10BD000004
:10DC000041070020A42E0020470700203B070020EA
:10DC10003507002038B5044600200090009401220A
:10DC20006946052000F05EFC38BD000008B5002004
:10DC3000009001226946062000F014FC6846007836
:10DC40000F4908736846407848730846007B0D49C1
:10DC500048730B48407B88730948807BC873084829
:10DC6000C07B0874002008730749086007490860F2
:10DC700007490860074908600749087008BD0000A7
:10DC800054280020D00900207C00002080000020C3
:10DC900084000020880000208C00002008B50020AF
:10DCA000009001226946062000F0DCFB68460078FF
:10DCB000124908736846407848730020104908608C
:10DCC00048600872487288720C48007B48730B48A1
:10DCD000407B88730948807BC8730848C07B087400
:10DCE0000020087307490860074908600749086071
:10DCF000074908600749087008BD00005428002043
:10DD0000D00900207C00002080000020840000203A
:10DD1000880000208C00002038B500240025002059
:10DD200000900121F848FDF769FA55280AD002F061
:10DD30006BFFF649487302F07BFFF44988730120BA
:10DD4000087308E0F248007BF0494873F048407BD4
:10DD50008873002008730621EB48FDF74FFA552819
:10DD600030D002F099FF002808D002F095FF401C47
:10DD7000002803D00120E549087502E00020E349AE
:10DD8000087502F06BFF002808D002F067FF401C06
:10DD9000002803D00120DD49C87402E00020DB49DF
:10DDA000C87402F079FF002808D002F075FF401C0B
:10DDB000002803D00120D549087507E00020D34989
:10DDC000087503E00020D149C8740875CF48407B2E
:10DDD00000282BD1CF490860CF480068CF4988423E
:10DDE00008D8CD480068401CCB4908600020C749CE
:10DDF00048736CE0C648007B022812D0C448007B00
:10DE000003280ED00121C048FDF7F8F9552803D0AA
:10DE10000320BE4948735AE0BD48007BBB494873A4
:10DE200055E0BB48007BB949487350E0B748407B98
:10DE300001282CD10020B8490860B6480068B749CD
:10DE4000884208D8B3480068401CB24908600120E5
:10DE5000AE4948733BE0AE48007B022812D0AC4884
:10DE6000007B03280ED00121A748FDF7C7F95528EC
:10DE700003D00320A549487329E0A548007BA349A6
:10DE8000487324E0A248007BA04948731FE09F48E4
:10DE9000407B022805D100209F4908609D49086009
:10DEA00015E09A48407B032808D100209A49086071
:10DEB0009849086003209549487308E00020964976
:10DEC0000860944908609248007B904948738F48E5
:10DED000807B00282BD192490860924800688F49C6
:10DEE000884208D88F480068401C8E49086000208E
:10DEF000864988736CE08648407B022812D08448AB
:10DF0000407B03280ED001217F48FDF777F9552883
:10DF100003D003207D4988735AE07D48407B7B49CC
:10DF2000887355E07A48407B7849887350E0774899
:10DF3000807B01282CD100207A490860784800684D
:10DF40007649884208D876480068401C74490860C1
:10DF500001206E4988733BE06D48407B022812D057
:10DF60006B48407B03280ED001216748FDF746F936
:10DF7000552803D003206549887329E06448407B15
:10DF80006249887324E06248407B604988731FE0DF
:10DF90005E48807B022805D1002062490860604904
:10DFA000086015E05948807B032808D100205D49AE
:10DFB00008605B49086003205449887308E000202A
:10DFC00058490860564908605148007B4F4988739A
:10DFD0004E48407B4E49097B884205D14B48807BA7
:10DFE0004B49497B88424FD04848407B4849097B90
:10DFF000884202D001204549C8734448807B444987
:10E00000497B884202D00120404908743F48407B48
:10E01000022803D03D48407B032816D13B48407B73
:10E020003B49097B884210D03848407B3849087307
:10E030000846017B684601703548417B684641705F
:10E0400001226946062000F04DFA3048807B022804
:10E0500003D02E48807B032816D12C48807B2C4986
:10E06000497B884210D02948807B2949487308465B
:10E07000017B684601702648417B68464170012259
:10E080006946062000F02EFA02F0C8FD044602F0B0
:10E09000DBFD054601211C48FDF7B0F8552807D1E6
:10E0A00000201A4908724872086048608872B9E016
:10E0B000FF2C01D0FF2D77D1FF2C3FD1FF2D3DD07C
:10E0C000002012490872012048721748086017485A
:10E0D0006843486048686621FAF738F80B49486099
:10E0E000084640681249884202D9084607494860F4
:10E0F00003F0E0F8112803DB03F0DCF8192819DD40
:10E100000120024988728DE068080020D0090020B3
:10E1100054280020800000207C00002070170000A0
:10E120008800002084000020DE030000BE0A0000FA
:10E13000AC26000000205949887273E0FF2C29D0DA
:10E14000FF2D27D1012055490872002048725448FC
:10E15000486054486043086008686621F9F7F6FF94
:10E160004E490860084600684F49884202D908466F
:10E170004A49086002F09AFF112803DB02F096FF7B
:10E18000192803DD0120454988724BE000204349EE
:10E19000887247E04448414908604860002088721E
:10E1A000087248723EE0FFE701203C49087248725D
:10E1B0003C486043086008686621F9F7C7FF3749A3
:10E1C0000860084600683849884202D90846334941
:10E1D0000860344868433149486048686621F9F767
:10E1E000B5FF2E494860084640682F49884202D949
:10E1F00008462A49486002F059FF11280BDB02F05B
:10E2000055FF192807DC03F055F8112803DB03F04C
:10E2100051F8192803DD01202049887202E000200E
:10E220001E4988721D48407B002802D11B49C873D3
:10E2300015E01A48407B012802D11849C8730EE046
:10E240001648407B022802D11449C87307E01348DE
:10E25000407B032803D11149C873134808600F4855
:10E26000807B002802D10D49087415E00B48807BA3
:10E27000012802D1094908740EE00848807B022871
:10E2800002D10649087407E00448807B032803D1C3
:10E29000024908740448486038BD0000D0090020D5
:10E2A000DE030000BE0A0000AC260000FFB583B00C
:10E2B00006460D46174600240020029000BF142099
:10E2C000784380190190002E57D00198002854D02F
:10E2D0002B4806602A49069848600846077200BF26
:10E2E00045E0FFF7C1FA02902001295802988142C7
:10E2F00004D820012858401C002806D12049029843
:10E300000A6814216143505006E0200129581C4836
:10E310000268142060431150200140194068401CDD
:10E32000002807D100211648026814206043101805
:10E33000416008E02001401941681148026814203A
:10E340006043101841602001401981680C48026840
:10E35000142060431018C16020014019017B084857
:10E3600002681420604310180161601CC4B20448A4
:10E37000007AA042B5DC00F005F807B0F0BD00005F
:10E380001C2F002070B5002400250026FFF76CFA32
:10E39000054600BF4EE02A48016814206043085833
:10E3A000A84239D8264801681420604308582E1A1C
:10E3B00023480168142060430818406881192048E8
:10E3C000026814206043101881601D480168142001
:10E3D0006043081881681A480268142060431018C6
:10E3E000C068814224D91648016814206043081887
:10E3F0000069002803D02046FEF7BCFC18E0104856
:10E400000168142060430818C1680D480268142090
:10E410006043101881600BE00948016814206043D4
:10E420000818406806490A68142161435118886039
:10E43000601CC4B20248007AA042ACDC70BD00008F
:10E440001C2F002010B500BF14244C4323180028B3
:10E4500005D0002B03D0024C20606260217210BDF9
:10E460001C2F0020F8B505460E4614462B0012F06E
:10E4700023FC0705131A3131212931001748FAF717
:10E4800073FB174908701548F9F728FF0746642100
:10E49000F9F75CFE30601EE0A004020C314620203B
:10E4A000FAF75CFC17E0A004020C31466020FAF792
:10E4B00055FC10E0A004020C3146FF202130FAF791
:10E4C0004DFC08E06004020C3146FF204130FAF7B1
:10E4D00045FC00E000BF00BF0020F8BD462800203A
:10E4E000DD00002070B505460E4614462B0012F0E4
:10E4F000E3FB07051D243A3A2B323A003068002826
:10E5000002D1FAF7CFF910E064223168514308468E
:10E510001649F9F7EDFE0020154908700122642123
:10E520001248FAF789FC124908701DE0A004020C99
:10E5300031462020FAF7D0FD16E0A004020C314647
:10E540006020FAF7C9FD0FE0A2B23146FF2021306A
:10E55000FAF7C2FD08E06004020C3146FF204130AA
:10E56000FAF7BAFD00E000BF00BF70BD38280020F8
:10E57000DC00002000B5AFB050211BA8F9F796FED3
:10E5800000201A90142115A8F9F790FE002012908F
:10E59000139014901190402101A8F9F787FE0020F4
:10E5A00000904849086001221BA9FFF75BFF1B98F8
:10E5B000401C002801D11A9001E01B981A90424893
:10E5C00015904248169042481790002018904148F4
:10E5D000199015AA1AA94048FFF7F8F802221CA9B9
:10E5E0000120FFF73FFF1C98401C002801D112902A
:10E5F00001E01C9812901C98401C002801D1139037
:10E6000001E01D9813903548149012A93448199AC6
:10E61000FFF724FA08221EA90220FFF723FF1E9805
:10E62000401C002801D1019001E01E9801901F9824
:10E6300002902C480390012069460874801E0590C2
:10E6400029490791012101A80177881E09902649CF
:10E650000B91012109A80173881E0D9022490F9189
:10E6600001210DA80173042201A92048199BFFF77D
:10E670001DFE01221BA90520FFF7F4FE1B98401C7C
:10E68000002807D101201A4988600122083105209D
:10E69000FFF728FF01221BA90620FFF7E3FE1B98C6
:10E6A000401C002808D100216846017041700122F9
:10E6B00069460620FFF716FF0E48024908602FB092
:10E6C00000BD0000E000002019CB00000DCB0000D1
:10E6D000F1CA0000E5E40000CC27002076841E008B
:10E6E000D82700200F2700009F860100E827002080
:10E6F00054280020A33AA55A00B585B014216846D5
:10E70000F9F7D4FD00200F4908600F4800900F482A
:10E7100001900F480290002003900E480490694633
:10E720000D48FFF72BF90D480499FFF7EDF9042187
:10E730000B48049AFFF786FE0A480249086005B0B4
:10E7400000BD0000E000002019CB00000DCB000050
:10E75000F1CA0000E5E40000CC270020D827002003
:10E76000E8270020A33AA55A00200C4908800C494C
:10E7700008800C49088001200B49087000200B49D3
:10E7800008730B4908804880012008710020074960
:10E790004880088007490860704700003400002066
:10E7A000360000203C0000203E00002058080020D9
:10E7B0004000002038000020F8B502F0EBF90646D2
:10E7C00002F0F2F90746FEF7A7F9012865D1052105
:10E7D000AB48FCF713FD552807D10020A949087064
:10E7E000A9490880A94988805FE0012F07D100204E
:10E7F000A4490870A4490880A449888055E0A1482C
:10E800000078002808D101209E49087035460A206A
:10E8100068439D49088048E09C48007B42009B4833
:10E82000801D8652801F047B11E061009748801D87
:10E83000455A601E41009548801D415A6200815230
:10E84000601E41009148801D4552601EC4B2002CDC
:10E850000ADD61008D48801D415A601E42008B48D0
:10E86000801D805A8142E0DB8848007B401C87493C
:10E8700008730846007B032807DB0020087308465E
:10E8800005890A206843804908807F4800887F49BD
:10E89000888001207B49087007E0002079490870D2
:10E8A00079490880794908738880774800887849D1
:10E8B000086074480078002815D0084600686C216C
:10E8C000484373490860642171480068F9F73EFCC9
:10E8D0006F490860084600686E49884206D90846B4
:10E8E0006B49086002E000206949086068480068D8
:10E8F00069490988884203D2654800680F2804D214
:10E9000063480088644908800AE0634800886049D9
:10E910000968401A0F2803D35D4800885E490880C3
:10E920005A480088401C59490880084600880A282F
:10E930002CDB002008805948008857490988884204
:10E9400003DA01205649087108E05448008852490A
:10E950000988884202DD0220514908715048007937
:10E96000012840D14C4800884C49098888420DDB79
:10E970004948018849480088FF309130814206DDCE
:10E9800046480088FF3073304449088077E04248A9
:10E990000188424800889630814205DD3F48008862
:10E9A00078303E4908806AE03B4801883B4800884F
:10E9B0003230814205DD394800881E3037490880F1
:10E9C0005DE035480188354800880A30814205DD20
:10E9D000324800880A303149088050E02E480088CB
:10E9E0002E4908804BE02E480079022847D12A485A
:10E9F00000882A490988884239DA27480088FF3088
:10EA0000913026490988884206DA24480088FF3870
:10EA10007338224908802AE01F48008896301F4931
:10EA20000988884205DA1D48008878381B49088023
:10EA30001DE019480088323018490988884205DAF3
:10EA4000164800881E381549088010E012480088D2
:10EA50000A3012490988884205DA104800880A38C5
:10EA60000E49088003E00C4800880C4908800B48D8
:10EA700000880849884202DB084608490880F8BD3A
:10EA8000680800203E0000203400002058080020C4
:10EA900038000020C60700003C000020360000209F
:10EAA00040000020002008490880084908800849E3
:10EAB00008804880012008710020064948800880AD
:10EAC0000549086070470000360000203C00002027
:10EAD0004000002058080020380000200020044991
:10EAE000087004490870002103480176704700004F
:10EAF0008D0000208E000020480A002070B50025FF
:10EB00000024FEF709F8012863D103213448FCF7FB
:10EB100075FB552808D10020324908703249087029
:10EB200000213248017659E02F480078002807D1AB
:10EB300002F0D0F82B49087001202B4908704DE0F5
:10EB400001202949087002F0C5F82849097E89008A
:10EB5000264A603A50502548047E10E0A000234920
:10EB600060390D5C601E80000858A1001F4A603AA1
:10EB70005050601E800011460D50601EC4B2002C23
:10EB80000ADDA000194960390958601E8000174A43
:10EB9000603A10588142E1D31448007E401CC1B253
:10EBA00012480176007E1E2818DB00210F480176EE
:10EBB00001466039896B0246603AD26B8918024679
:10EBC000603A126C88180321F9F7C0FA05490870F9
:10EBD00004E00020034908700349087070BD00007C
:10EBE000680800208D0000208E000020480A0020C8
:10EBF000F0B5A9B004460E46002500270020289055
:10EC0000A0216846F9F752FBFEF72EFE26490A6856
:10EC100014216143505024480168142060430818AF
:10EC2000C068B0420CD22048016814206043081824
:10EC3000C1681D480268142060431018416005E057
:10EC40001948016814206043081846601648406857
:10EC5000002826D0002517E06806070E282F00D3CD
:10EC600016E011480168142068430858B9006A4644
:10EC700050500D4801681420684308184168781CFA
:10EC800080001150681CC5B20748007AA842E3DC36
:10EC900000BF6A0004486946436802209847012083
:10ECA0002890289829B0F0BD1C2F002010B500F046
:10ECB000F9FD00F0D7F810F01DFF00F00DFB00F09B
:10ECC00001F810BD70B541480078912800D070BDA2
:10ECD00000F0BEF8012876D13D4800883D49088003
:10ECE00008468078F021884320303A4988700846E9
:10ECF0008078000900013549097A0907090F08439E
:10ED0000344988703148807A401E304988720846FC
:10ED10000089401C088108460089C988884216DAA3
:10ED200008202C49887200240EE028484188284891
:10ED3000001D415C2748C01C015524484088401CE8
:10ED400022494880601CC4B2072CEEDB2DE01F482E
:10ED500000891E49C98888421CD11C4800791B497A
:10ED60008978401AC5B2681C1A49887200240EE0DE
:10ED7000164841881648001D415C1648C01C0155C4
:10ED800012484088401C11494880601CC4B2AC4203
:10ED9000EEDB0AE000F012FD00200C4908700C497F
:10EDA0000888092100F0B8F991E7012000F0C8FCBB
:10EDB000084A917A1088921C00F070F90549088879
:10EDC000002100F0C1F800BF81E70000542C0020B2
:10EDD000F02B0020802B00201B49097E002932D017
:10EDE0001949897E0C225143174A515A174A1180FA
:10EDF00000200CE01449897E0C225143124A8918E4
:10EE0000891C0A5C1149891C0A54411CC8B2082893
:10EE1000F0DB0D49897E0C2251430B4A8918897A0F
:10EE20000A4A91720121D1720749097E491E064A98
:10EE300011761146897E491C91761146897E0229F8
:10EE400001DB0021917670474C2B0020742B0020B1
:10EE50000349487B012802D10021014A51737047C0
:10EE6000642C002010B533484068002861D1314837
:10EE7000007B030011F020FF07590512212E3D4AA7
:10EE800059002D480078002807D000202A49087032
:10EE90002A490888012100F03FF947E02648007818
:10EEA000002809D000202449087025494A8808888C
:10EEB0000123091D00F040F938E01F4800780028C0
:10EEC00007D000201C4908701C490888022100F066
:10EED00023F92BE018480078002809D000201649B3
:10EEE000087017494A8808880923091D00F024F989
:10EEF0001CE011480078002807D000200E49087057
:10EF00000E490888092100F007F90FE00A48007847
:10EF1000002809D000200849087009494A88088853
:10EF20000323091D00F008F900E000BF00BF00F056
:10EF300045FC10BD642C0020542C0020F02B002038
:10EF40008C2B00207047000070B504460D463448F5
:10EF50000088A04263D1002D61D132480078222878
:10EF60004ED004DC20283DD0212856D141E0902805
:10EF700002D0912851D115E02A48C08801280AD131
:10EF800000202849087000F019FC27490888002152
:10EF900000F0C2F805E0032000F0D2FBA0202149D8
:10EFA00008703BE01F4800891E49C98888420AD181
:10EFB00000201C49087000F001FC1B490888002152
:10EFC00000F0AAF80DE01748807A002806D000F07B
:10EFD000F5FB1449087B00F095FB02E0032000F0EC
:10EFE000AFFB1BE0062000F0ABFB11200D490870C1
:10EFF00014E0062000F0A4FB11200A4908700DE07F
:10F0000000200849087000F0D9FB08494A880888A0
:10F010000923091D00F090F800E000BF00BF70BD9B
:10F02000682B0020542C0020F02B00208C2B00207B
:10F0300070B50346184C247E022C00DB70BD164CC4
:10F04000647E0C256C43144D2B5300200AE0155CA4
:10F05000114C647E0C2674430F4EA419A41C255435
:10F06000441CE0B28842F2D30B4C647E0C267443FD
:10F07000094EA419A1723446247E641C35462C76B0
:10F080002C46647E641C6C762C46647E022C01DB6C
:10F0900000246C7600BFD1E74C2B0020F0B585B082
:10F0A00007460D4616461A480780002406E03178C8
:10F0B0001748801C0155761C601CC4B2AC42F6DBBC
:10F0C0002C4605E0AA211248801C0155601CC4B2E0
:10F0D000082CF7DB0E480088019008216846C172B1
:10F0E0000021417201720170002406E00848801C72
:10F0F000015D03A80155601CC4B2082CF6DB69460B
:10F100000448FCF7A8F901200149887205B0F0BD58
:10F11000682B00209055044070B504460D462946E2
:10F12000204610F009FC70BD70B504460D46294616
:10F13000204610F00FFC70BDF8B504460D4616468B
:10F140001F463B4632462946204610F004FCF8BDD7
:10F15000F8B507460E4615465C480078002804D0EE
:10F1600009213846FFF7D8FFF8BD002D01D0602DEA
:10F1700004DD09213846FFF7CFFFF5E75448078043
:10F180004580002406E031785148001D0155761C69
:10F19000601CC4B2AC42F6DB00204C494870084603
:10F1A0008580FF2088727F200873084680880828A1
:10F1B0002EDA0120C8800846808848800120088116
:10F1C000434800884349088008468078F0218843F6
:10F1D0004049887008468078000900013B49097958
:10F1E0000907090F08433B49887038480079401CDB
:10F1F0008872002407E03648001D015D3548C01CB8
:10F200000155601CC4B231488088A042F3DC4AE05A
:10F210000721681CF8F7B0FF002907D0072128460E
:10F220000830F8F7A9FF2949C88005E00721681CC4
:10F23000F8F7A2FF2549C88006202449488001200C
:10F240000881234800882349088008468078F021F7
:10F25000884310301F4988700846807800090001F3
:10F260001A4989880905090F08431A498870084610
:10F270004088FF2109028843144989880902FF2236
:10F280001202114008431349488008208872002464
:10F2900007E00F48001D015D0E48001D0155601C70
:10F2A000C4B2062CF5DB012000F04AFA094A917A33
:10F2B0001088921CFFF7F2FE90200449087005495F
:10F2C00008880021FFF740FE00BF4DE7542C0020C6
:10F2D000F02B0020802B002010B5FFF77DFD144897
:10F2E000C07A002822D0124880780009002806D071
:10F2F000012807D002280AD0032810D10CE000F022
:10F30000A7F90FE000F09EF800F066FA0AE000F0BE
:10F3100011F800F061FA05E000F000F902E0FFF7F3
:10F3200011FE00BF00BF00200149C87210BD0000DF
:10F33000742B002010B53F480078112800D010BD74
:10F340003D4800883D49884200D0F8E73A48807837
:10F350000007000F3749097A0907090F88420CD0C6
:10F3600000203449087000F029FA35494A88088895
:10F370000423091DFFF7E0FEE1E72E480089401C49
:10F380002C4908810846807A401E88720846008908
:10F39000C98888421BDA2848807A082800D0CEE73E
:10F3A00000240EE02448C01C015D22484288244805
:10F3B000001D81541F484088401C1E494880601C25
:10F3C000C4B2072CEEDB062000F0BAF930E0194891
:10F3D000808818494988401A1749897A884203DA8F
:10F3E0001548807A082800D0A9E700240EE01248CA
:10F3F000C01C015D0F4842881148001D8154601CEB
:10F40000C4B20C484088401C0A49488009484088DA
:10F41000084989888842EADB00200649087000F024
:10F42000CDF907494A8808880023091DFFF784FEA3
:10F4300000BF84E7542C0020742B00201407000028
:10F440008C2B002070B5314800788021084080283E
:10F4500000D170BD2E4800882E49884200D0F8E7C0
:10F460002B48807A082800D0F3E7294880780507E0
:10F470002D0F2D0226484088000A0543082D00DA8A
:10F48000E7E700202149487006204880084685802B
:10F4900001200881082088720020C8728988481CD1
:10F4A0000721F8F769FE002909D01849898808461C
:10F4B00008300721F8F760FE1449C88007E01349B7
:10F4C0008988481C0721F8F757FE1049C880104862
:10F4D00000881149088008464580002407E00C4850
:10F4E000001D015D0C48001D0155601CC4B2062CB6
:10F4F000F5DB042000F024F9102004490870064AC6
:10F5000051881088FFF710FE00BFA2E7542C00209E
:10F51000742B0020140700008C2B002010B54848E5
:10F520000078A02808D046480078912804D04448A4
:10F530000078A12800D010BD424800884249884286
:10F540000AD0424908880921FFF7E6FD00F036F9A4
:10F5500000203B490870EEE73A48807A08280AD034
:10F560003A4908880921FFF7D7FD00F027F9002064
:10F5700033490870DFE7334880780007000F002820
:10F5800004D001282DD002284BD136E02C484078F9
:10F59000002800D050E02B48C078002803D101207B
:10F5A0002749487003E02748C078254988722448D5
:10F5B000007891280BD023480079002803D101203E
:10F5C0001F49087303E01F4800791D490873912003
:10F5D0001B49087000F0F2F81949087B00F092F816
:10F5E0002AE017484078002800D025E0A1201449DF
:10F5F0000870032000F0A4F81EE0114840780028AD
:10F6000000D019E00E480078A02809D10F490888D9
:10F610000821FFF781FD00F0D1F8002008490870AB
:10F620000AE00A4908880521FFF776FD00F0C6F8D0
:10F6300000200349087000BF00BF00BF7BE7000047
:10F64000542C0020742B002014070000F02B002005
:10F6500010B52848007880210840802800D110BDCE
:10F6600024480078002805D0234800882349884290
:10F6700000D0F4E72048807A1F4989780907090FEC
:10F68000884203DD1C48807A082800D0E7E71A4842
:10F6900080780007000F002805D017488078000701
:10F6A000000F072800DDDAE71348008814490880B6
:10F6B000114880780007000F4880002407E00E48BA
:10F6C000C01C015D0E48001D0155601CC4B20C48F1
:10F6D0004088A042F3DC00200649087000F06EF874
:10F6E00007494A8808880023091DFFF725FD00BF48
:10F6F000B5E70000542C0020742B002014070000F4
:10F700008C2B00207F2805DC7D21C90041430A4A5B
:10F7100091600DE0F12808DBF92806DC0107090FEC
:10F7200064225143044A916002E00449024A916014
:10F730000221014A51737047642C002018F0010027
:10F7400000B5030011F0B8FA0729050B11171D23A6
:10F7500029000121144A11731449516022E0022149
:10F76000114A1173114951601CE003210E4A1173B3
:10F770000F49516016E004210B4A11730D49516085
:10F7800010E00521084A1173002151600AE00621AA
:10F79000054A11730849516004E00021024A1173BF
:10F7A000516000BF00BF00BD642C0020A8610000B4
:10F7B000F824010028230000F0490200002001493C
:10F7C00008737047642C0020024909880918014A0F
:10F7D00011807047642C002010B52E480078102846
:10F7E00018D12D48408860280ADD2C48807800090F
:10F7F0000001801C2949887022202649087025E0D4
:10F800002648807800090001244988702020214979
:10F8100008701BE01F480078112816D11D48807A17
:10F82000002800D010BD1B484078002800D0F9E720
:10F830000820184988721948807800090001174982
:10F84000887020201349087000E0EBE71448134942
:10F85000088008468078F021884330300F4988704E
:10F860000846C0780020C870084600791420087146
:10F87000032088720220FFF763FF084A917A1088FC
:10F88000921CFFF70BFC054908880021FFF75CFB81
:10F8900000BFC7E7542C00208C2B0020802B0020B9
:10F8A00094070000244A118852888A4242D0224A92
:10F8B00052888A4204DA204A52888A1A90B207E0B3
:10F8C0001D4A52880023DB439A1A521C521890B2E8
:10F8D000194A5180127B002A10D0174A5268002A18
:10F8E0000CD0154A5268824205D9134A5268121A3E
:10F8F000114B5A6002E000220F4B5A600E4A527BB5
:10F90000022A17D10C4A9268002A0CD00A4A92683F
:10F91000824205D9084A9268121A074B9A6002E09F
:10F920000022054B9A60044A9268002A02D1012203
:10F93000014B5A7370470000642C002010B506F08C
:10F9400091F910BD00BF704710B504462146032051
:10F95000400206F0ADF810BD10B580210320400232
:10F9600006F03AF810BD000010B50224024806F077
:10F9700083F80446204610BD0106000010B50021A2
:10F98000014806F029F810BD0106000010B5044634
:10F990002146024806F08CF810BD00000106000068
:10F9A00010B58021014806F017F810BD01060000CF
:10F9B00030B503460C46002101250D48834201D095
:10F9C000002B01D1022030BD012A01D10120FAE72C
:10F9D000002108E0C8002058984202D1002528469E
:10F9E000F1E7481C81B29142F4DB2846EBE70000C6
:10F9F000FFFF0000002000BF14E00021C200134BF5
:10FA00009950C200D2189180C200114B9950C20087
:10FA1000D2189180C2000F4B9950C200D218918029
:10FA2000411C88B24828E8DB0B490C4A11600C499C
:10FA30005160002191600B4911610B49D160002197
:10FA40000A4A11800A4A117070470000981F00206E
:10FA5000D821002018240020250F0100841F002039
:10FA6000C10F01006B1001005D100100BE000020FD
:10FA7000C2000020F0B585B00646674F38460390B7
:10FA80000290002500240020019000906348006847
:10FA9000002803D061490868804707465F484068EE
:10FAA000002803D05D494868804703905B48806820
:10FAB000002803D059498868804702905748006958
:10FAC000002803D055490869804700905348C06812
:10FAD000002803D05149C86880470546482D00DDFD
:10FAE00048250098002876D0002D74DD4C48008809
:10FAF000A8420BDA2B463A4649494A48FAF7F4FD40
:10FB00002B4647494748039AFAF7EEFD44480088D8
:10FB1000002833DD42480088A84202D10020404935
:10FB20000880002415E0E0003F490858E1003D4A04
:10FB3000515888420BD0E00011460858E1003A4A7B
:10FB40005050E00011460858E100384A5050601CFF
:10FB500084B2AC42E7DB0120354908702C460BE04B
:10FB60000020E100314A5050E1002F4A5050E1009E
:10FB70002C4A5050601C84B2482CF1DB2B480068A2
:10FB80002549884246D0294880882A49884205DA92
:10FB9000264880888019254988803BE00020234939
:10FBA0008880084600680190012D33DD002408E0BC
:10FBB000601CC0001D490858E1001C4A5050601CE0
:10FBC00084B2681EA042F3DC691EC900174A01987E
:10FBD00050501FE0FFE7002015490870002414E092
:10FBE0000020E100114A5050E10089188880E100AE
:10FBF0000C4A5050E10089188880E1000A4A5050B0
:10FC0000E10089188880601C84B2482CE8DB002061
:10FC10000349088005B0F0BDFFFF0000841F0020ED
:10FC2000BE000020D821002018240020981F0020AA
:10FC3000C2000020881300002E480078401C2D4987
:10FC400008702D480078401C2B4908702B4800781C
:10FC5000401C2A4908702A480068401C284908604E
:10FC600008460068FF219131884202D900202449CA
:10FC7000086020480078C82802D900201D49087073
:10FC80001D480078842802D900201B4908701B48B1
:10FC90000078502802D900201849087019481849DE
:10FCA0000968405C18490870184812490978405C96
:10FCB00017490870174810490978405C16490870C0
:10FCC00016480E490978405C1549087015480949DD
:10FCD0000978405C14490870144806490978405C6A
:10FCE00013490870134803490978405C12490870A9
:10FCF000704700006B0700206C0700206D07002094
:10FD0000700700203722020064070020C72302008A
:10FD1000650700208F24020066070020DB25020013
:10FD20006807002013250200670700202B26020029
:10FD300069070020F32602006A07002010B5820040
:10FD4000054BD218525C012A04D100228300024CD8
:10FD50001B195A5410BD0000D02A002010B50446CB
:10FD6000204600F055FA204600F002F810BD0000D1
:10FD700010B50446B348007800287DD1B248008809
:10FD8000B249884278DAB248007800284FD0B148AA
:10FD90000078002803D0AC480088AF490880AF48FD
:10FDA0000078002818D1A8480188AB4800880A309C
:10FDB000814206D30120A9490870A3480088A649BA
:10FDC0000880A1480088A449098888421CDA9E4816
:10FDD0000088A149088017E09F4801889A48008858
:10FDE0000A30814206D300209C490870964800885A
:10FDF000994908809448008897490988884203DD1A
:10FE0000914800889449088094480078002858D187
:10FE100093480078042803D08E480078002807D043
:10FE200089480088822803DA05208D490870A3E0FC
:10FE30008B480078032803D086480078002809D032
:10FE400081480088FF211931884203DA042084495F
:10FE5000087091E082480078022803D07D4800783D
:10FE600000280AD078480088FF21AF31884204DAA0
:10FE700003207B4908707FE0E2E0794800780128A0
:10FE800003D074480078002809D06F480088AF215B
:10FE90008900884203DA0220714908706CE07048DA
:10FEA0000078002803D06B480078002864D06648AA
:10FEB0000088E121890088425EDA012068490870E3
:10FEC0005AE066480078012856D165480078012834
:10FED00003D060480078002809D05B480088E12101
:10FEE0008900884203DB00205D49087044E05C48DB
:10FEF0000078022803D057480078002809D05248DB
:10FF00000088AF218900884203DB01205449087032
:10FF100032E053480078032803D04E480078002888
:10FF200009D049480088FF21AF31884203DB022015
:10FF30004B49087020E04A480078042803D045481F
:10FF40000078002809D040480088FF2119318842F4
:10FF500003DB0320424908700EE041480078052881
:10FF600003D03C480078002806D037480088822813
:10FF700002DB04203A490870FCF7B4FD33496439C8
:10FF800088425DD337480068001936490860314817
:10FF90000078002808D000202E49087031490860F8
:10FFA0002F4800783049087000F0A8FD00281FD1C4
:10FFB0002C4800682D49884239D30020294908601F
:10FFC0002948007826490978884205DA26480078C9
:10FFD000401C254908702AE0234800782049097808
:10FFE000884224DD20480078401E1F4908701EE02A
:10FFF0001C4800681E49884219D30020194908602E
:020000040001F9
:100000001948007816490978884205DA16480078B8
:10001000401C154908700AE0134800781049097817
:10002000884204DD10480078401E0F4908700E48D1
:1000300000780B490978884202D1002009490860FC
:1000400010BD00000B000020020000201C0C00006E
:100050001200002008000020040000200A000020F8
:10006000060000201800002007000020C05D0000EE
:10007000407E050000200B4908700B4908700120E4
:100080000A4908700A49087000200A4908700A499C
:1000900008700A4908800A4908800A4908800A4904
:1000A00008707047060000200700002008000020AC
:1000B000090000200A0000200B0000200C00002096
:1000C0000E000020100000201200002000200B492C
:1000D00008700B49087001200A4908700A49087025
:1000E00000200A4908700A4908700A4908800A492C
:1000F00008800A4908800A490870704706000020F5
:100100000700002008000020090000200A0000204D
:100110000B0000200C0000200E000020100000202A
:1001200012000020F8B50646002700240025002014
:10013000009031480078002809D00320F9F714FA1C
:10014000002804D00320F9F703FA2C4908802C4832
:1001500000880A284AD300202949088029480078C5
:10016000282829D20320F9F7F3F90746002407E0ED
:1001700060002549085AB84200DD05E0601CC4B2A1
:10018000204800788442F3DB00BF1E48057808E071
:10019000681E40001C49085A69001B4A5052681EDC
:1001A000C5B2A542F4DC600017490F52154800782B
:1001B000401C1449087019E0002000900F2407E04B
:1001C00060001149095A009808180090601CC4B2D8
:1001D000192CF5D30A210098F7F7B8FF07490880D2
:1001E0000020084908700120084908700448008868
:1001F000801903490880F8BD090000200200002092
:100200001600002000000020FC0700201200002043
:10021000394909881E2928DA0021384A1180384ACC
:10022000118038490988384A914207DC37490978F2
:10023000002914D033490988914210DC0121344A45
:1002400011700021334A1170334A11702F4A117016
:100250000121324A11700021314A11704BE02949C5
:1002600009880918274A118045E023490988264A48
:10027000643291422ADB0021224A1180204A1180F7
:100280001E490988204A914207DC20490978002943
:1002900016D01A490988914212DC02211C4A1170B9
:1002A00000211C4A117005211B4A11700021174AB8
:1002B00011700121194A11700021194A11701AE0B8
:1002C0000E49098809180D4A118014E000210D4AD1
:1002D00011800A4A11800A4909880B4A914205DDBA
:1002E00000210B4A1170094A117004E00449098881
:1002F0000918034A118070470200002010000020F6
:100300000C0000200E000020B80B000009000020A7
:100310000B0000200600002007000020080000203D
:100320000A0000200148007870470000582600208D
:100330000148407A704700005826002010B564211B
:1003400002480068F7F702FF80B210BDCC00002021
:10035000014880787047000058260020F8B5002337
:10036000002500950024002200BF94E001259D4057
:10037000ACB20D8825400095009DA5426FD11A466C
:100380008D79012D0DD1464D03263602AD192D5C18
:10039000012696403543424E03273F02F619355455
:1003A0000CE03F4D03263602AD192D5C0126964028
:1003B000B5433B4E03273F02F6193554CD78002D47
:1003C0004ED1374D60352D5CCE78002E01D10126FF
:1003D00000E000269640B543314E603635548D78A6
:1003E000002D2ED12E4D19267601AD192D5C8E785B
:1003F000002E01D1012600E000269640B543284E8C
:1004000019277F01F61935540D79002D0ED1244D91
:1004100050352D5C0E79002E01D1012600E000261A
:100420009640B5431E4E5036355423E01C4D503592
:100430002D5C0E7996403543EEB2194D50352E5451
:1004400018E0174D19267601AD192D5C8E7896406F
:100450003543134E19277F01F61935540AE018E089
:100460000F4D60352D5CCE7896403543EEB20C4D85
:1004700060352E544D79012D0AD1094D30352D5C52
:10048000012696403543EEB2054D30352E5400E03E
:1004900000BF5D1CABB2082B00DA67E7F8BD0000B7
:1004A00000000440FFB5074615461E4600243846A6
:1004B000019900F01FF8002802D0012004B0F0BD1F
:1004C00000240CE00A2060430949085CB04204D1D2
:1004D0002946204600F05EF807E0601C84B20A203E
:1004E00060430349085C0028ECD100BF0020E5E729
:1004F000C00100200246002A03D1402901DD01206D
:100500007047032A03D1022901DD0120F8E7042AFC
:1005100003D1202901DD0120F2E7052A03D120299A
:1005200001DD0120ECE70C2A03D1102901DD0120B7
:10053000E6E70D2A05D1012903DD402901DA012072
:10054000DEE70E2A03D1202901D10120D8E70020BF
:10055000D6E7000010B5064A03231B02D218125C2E
:100560008A43034B032424021B191A5410BD0000B4
:100570000000044010B5064A03231B02D218125C87
:100580000A43034B032424021B191A5410BD000014
:100590000000044070B502460020B1E00A23534336
:1005A0005A4C1B195B1C440004191B199B788B4285
:1005B0007DD10A235343554C1B195B1C440004197D
:1005C0001B195B78082B33D10A2353434F4C1B195B
:1005D0005B1C440004191B574D4C4E4D6419E35CE1
:1005E000012423430A245443484D6419641C4500E4
:1005F00045196457464D474EAD192B550A235343B1
:10060000424C1B195B1C440004191B57404C3546D7
:100610006419E35C022423430A2454433B4D6419C8
:10062000641C450045196457394DAD192B5564E0DC
:100630000A235343354C1B195B1C440004191B1936
:100640005B78092B34D10A235343304C1B195B1CB4
:10065000440004191B572E4C2E4D6419E35C4024B2
:1006600023430A245443294D6419641C4500451949
:100670006457274D274EAD192B550A235343234C5E
:100680001B195B1C440004191B57214C3546641987
:10069000E35C8024A3430A2454431C4D6419641C66
:1006A0004500451964571A4DAD192B5525E025E035
:1006B0000A235343154C1B195B1C440004191B5798
:1006C000134C144D6419E35C0A2454430F4D641910
:1006D000641C45004519641965780124AC40234326
:1006E000DCB20A235343094D5B195B1C45004519D5
:1006F0005B57074D074EAD19EC5404E0431CD8B2CC
:10070000032800DA4AE700BF70BD0000C0010020E6
:100710000000044075080000F8B50024FCF7FCF95F
:10072000012861D100F0A6FB0446FF22072100202A
:1007300003F0BCF8012C21D100F09AFC00280ED067
:1007400000F0AAFB054600F09BFB0646012003468D
:10075000024629460090304605F0BEFC50E000F00D
:100760009BFB054600F08CFB064601200023024659
:1007700029460090304605F0AFFC41E0022C21D123
:1007800000F076FC00280ED000F086FB054600F055
:1007900077FB064601200346024629460090304674
:1007A00005F09AFC2CE000F077FB054600F068FBB2
:1007B0000646002001231A4629460090304605F0DF
:1007C0008BFC1DE000F054FC054600F065FB06467E
:1007D00000F056FB0746012003462A4631460090AA
:1007E000384605F079FC0BE000200346024601463E
:1007F000009005F071FC00220721104603F056F826
:10080000F8BD0000FEB5002481480078012827D1FA
:10081000FCF782F9012815D1FBF75CFF00BF0EE061
:10082000182C0AD0152C08D00D2C06D01A2C04D068
:10083000FF222146002003F039F8601CC4B2242CAA
:10084000EEDBE4E0FCF796F8002406E00022214607
:10085000104603F02BF8601CC4B2242CF6DBD6E063
:10086000FCF75AF901287BD1FCF73CF96949884229
:1008700078D300F00BFB064600F022FB07460A2166
:10088000F7F764FC05463246294601200BF0E0F9F3
:1008900000F060FD064600F0E1FC0A210290F7F747
:1008A00055FC054600F0F2FA07463246294609F0A3
:1008B0005DF9FFF731FF00F0CBFA0546294601202C
:1008C00007F09AFC00F0F6FA0646FF21F531F7F73B
:1008D00053FCC5B22946012006F0BAFBFFF722FD02
:1008E0000546FFF72BFD0646FFF732FD07462B4670
:1008F00032463946012005F0C9FE00F005F90546EB
:10090000294601200BF04AFC00F0CEFC054600F021
:10091000C7FB064600F0CEFC074600F0C7FB0023ED
:100920003A46014600960195029001200AF0ACFE7D
:10093000FF220321002002F0B9FFFF220421002042
:1009400002F0B4FF00F07EFC054600F075FC0646A0
:1009500000F07EFC07462A46314607F081FE56E04D
:100960000DE0FFE7FF220321002002F09FFFFF229E
:100970000421002002F09AFFFBF726FF47E0FBF777
:10098000F9FF00220321104602F090FF002204210B
:10099000104602F08BFF00222321104602F086FF52
:1009A00000222221104602F081FF0022072110467A
:1009B00002F07CFF00220821104602F077FF00229F
:1009C0000921104602F072FF00220A21104602F0AF
:1009D0006DFF00221321104602F068FF0022112152
:1009E000104602F063FF00221221104602F05EFF63
:1009F00000220E21104602F059FF00220F2110465E
:100A000002F054FF00221021104602F04FFFFEBDFD
:100A1000F9000020D60B0000014908607047000073
:100A20009807002002480068401C01490860704790
:100A300094070020F3B581B0064600200E490860F7
:100A400000F01EF8044600F01BF805462F1B304648
:100A5000029903F03DFF00900AE000F011F805460E
:100A60002F1B06480068002802D004480068804711
:100A700000988742F1D3FEBD94070020980700201C
:100A80000148006870470000940700200B4909786E
:100A9000012901D101200FE008490978022901D17B
:100AA000022009E005490978032901D1042003E067
:100AB0000121024A11700120704700002507002023
:100AC00010B5094B1B8899B20A12C8B2D34331330F
:100AD000064C2370C3432333637013465633A3700D
:100AE00003467133E37010BD5C0700202B07002024
:100AF00001480088704700001C0000200148008861
:100B00007047000034000020014800787047000062
:100B10008D00002001480078704700008E00002002
:100B200010B5002205210648FAF756FB04020122FF
:100B300005210348FAF750FB201880B210BD0000D1
:100B40006808002010B5062205210348FAF744FB87
:100B5000C006C00F10BD00006808002010B50422B8
:100B600005210648FAF738FB04020522114603481E
:100B7000FAF732FB201880B210BD00006808002090
:100B800010B5062205210248FAF726FBC01110BD58
:100B90006808002010B5022205210248FAF71CFB64
:100BA00010BD00006808002010B50622052103488A
:100BB000FAF712FB8006C00F10BD00006808002085
:100BC00010B5042202210348FAF706FBC007C00F44
:100BD00010BD00006808002010B50522022103485E
:100BE000FAF7FAFAC007C00F10BD0000680800202D
:100BF00010B5002204210348FAF7EEFA4006400F30
:100C000010BD00006808002010B504220121024830
:100C1000FAF7E2FA801110BD6808002010B5002232
:100C200001210248FAF7D8FA10BD00006808002038
:100C300010B5052201210348FAF7CEFA8007800F8C
:100C400010BD00006808002010B5012211460248BE
:100C5000FAF7C2FA10BD00006808002010B50022A3
:100C600006210C48FAF7B8FA0402012206210948C5
:100C7000FAF7B2FA20180402022206210548FAF710
:100C8000ABFA20180402032206210248FAF7A4FA5C
:100C9000201810BD6808002010B5042206210C4859
:100CA000FAF79AFA0402052206210948FAF794FA9B
:100CB00020180402062211460548FAF78DFA20187A
:100CC0000402072206210248FAF786FA201810BD0E
:100CD0006808002010B5022203210248FAF77CFAC6
:100CE00010BD00006808002010B503220021024852
:100CF000FAF772FA10BD00006808002010B5002253
:100D000011460248FAF768FA10BD00006808002092
:100D100010B5042200210248FAF75EFA10BD000067
:100D20006808002010B5012200210248FAF754FAA1
:100D300010BD00006808002010B5052200210248FF
:100D4000FAF74AFA10BD000068080020014632296F
:100D500015DA3E488078012803DD01203B4A5070B7
:100D600070E03A488078002805DD2F296ADC0020F1
:100D7000364A507066E00020344A507062E03E29E6
:100D800017DA322915DB31488078022803DD02208A
:100D90002E4A507056E02D488078012805DD3B2909
:100DA00050DC0120294A50704CE00120274A507045
:100DB00048E0502917DA3E2915DB244880780328BB
:100DC00003DD0320214A50703CE02048807802284F
:100DD00005DD4D2936DC02201C4A507032E002202D
:100DE0001A4A50702EE0622917DA502915DB17488D
:100DF0008078042803DD0420144A507022E0134850
:100E00008078032805DD5F291CDC03200F4A507021
:100E100018E003200D4A507014E073290FDA62299C
:100E20000DDB0A488078042805DD70290ADC0420DF
:100E3000064A507006E00420044A507002E0052083
:100E4000024A507001484078704700005826002040
:100E50000148007870470000070000200148006842
:100E600070470000981F002001480078704700007C
:100E7000ED0000200148007870470000EC000020E1
:100E80000148007870470000F10000200148007917
:100E90007047000054280020014840787047000047
:100EA000F10000200148007A70470000542800201B
:100EB0000020704701480088704700001E00002095
:100EC00010B50024FFF7E2FF00280AD10A48008885
:100ED0000A49884202DB0846074908800648048818
:100EE00008E005480088FCF7F5FB84B2044884421A
:100EF00000DB0446204610BD36000020C607000077
:100F0000CE040000002005490988054A914202DB11
:100F10001146024A118001490888704736000020B6
:100F2000C6070000F8B50027002500260024FFF7BB
:100F3000E5FE0546FFF7F6FE0646F02028400011C4
:100F40000A2805DBF02028400011C01C044303E000
:100F5000F02028400011044324022807000F0A282B
:100F600004DB2807000FC01C044302E02807000F21
:100F700004432402F020304000110A2805DBF02051
:100F800030400011C01C044303E0F0203040001149
:100F9000044324023007000F0A2804DB3007000F47
:100FA000C01C044302E03007000F0443002C01D1B1
:100FB0000248F8BD27463846FBE70000FFFF000067
:100FC000F8B50027002500260024FFF7A1FE0546FE
:100FD000FFF7B2FE0646F020284000110A2805DB84
:100FE000F02028400011C01C044303E0F0202840FA
:100FF0000011044324022807000F0A2804DB2807F5
:10100000000FC01C044302E02807000F0443240221
:10101000F020304000110A2805DBF020304000119C
:10102000C01C044303E0F0203040001104432402BC
:101030003007000F0A2804DB3007000FC01C0443F0
:1010400002E03007000F0443002C01D10248F8BD34
:1010500027463846FBE70000FFFF000010B50024DC
:10106000FFF742FE0446204610BD012070470000F5
:1010700001480078704700006507002001480078AB
:1010800070470000670700200148C07B70470000E0
:10109000D00900200148C07C70470000D009002022
:1010A0000148007A70470000D009002010B50024E4
:1010B00005480088323084B264212046F7F75CF896
:1010C00084B2204610BD0000D009002070B5002475
:1010D00007490868FBF740FE05466421F7F736F834
:1010E00084B20448844200DD0446204670BD0000FE
:1010F000D0090020DE03000010B5002400F014F831
:10110000012800D10CE000F00FF8022802D1FF24E2
:10111000373405E00A2103480088F7F72DF884B238
:10112000204610BD020000200148007870470000F2
:101130000B000020002005490968002903D003495D
:101140000968086800E00248704700007801002044
:101150003075000010B50024044804F08DFC002810
:1011600001D0012400E00024204610BD0407000047
:1011700010B50024044804F07FFC002801D00124AD
:1011800000E00024204610BD0507000010B5002433
:10119000044804F071FC002801D0012400E0002480
:1011A000204610BD0707000010B50024062004F0FB
:1011B00063FC002801D0012400E00024204610BD7B
:1011C00010B50024052004F057FC002801D00124AC
:1011D00000E00024204610BD10B50024044804F0AF
:1011E0004BFC002801D0012400E00024204610BD63
:1011F0000607000010B50024044804F03DFC002858
:1012000001D0012400E00024204610BD03050000A9
:1012100010B50024044804F02FFC002801D001245C
:1012200000E00024204610BD040500000148807A3B
:1012300070470000D0090020014880787047000006
:10124000680A00200148406870470000680A0020D2
:101250000148407870470000680A002070B50024FB
:10126000FFF714FE002803D1FCF748FC04460DE00C
:10127000FFF70CFE012806D1FCF740FC0546FCF701
:1012800029FA044602E0FCF739FC0446204670BD0A
:101290000148007C70470000D00900200148007D13
:1012A00070470000D00900200148407A70470000D4
:1012B000D009002010B5002405488088323084B25F
:1012C00064212046F6F758FF84B2204610BD000086
:1012D000D009002070B5002407494868FBF73CFDA1
:1012E00005466421F6F732FF84B20448844200DDEB
:1012F0000446204670BD0000D0090020DE03000037
:1013000070B50BF059FA05460BF056FA044908601F
:10131000002D01D1012400E00024204670BD000012
:10132000840100200148007B70470000D0090020A4
:101330000148407B70470000D00900200148807BB5
:1013400070470000D0090020014800787047000075
:10135000F000002070B50024FFF798FD002803D1AD
:10136000FCF7EEFB04460FE0FFF790FD012807D1E4
:101370000020FCF7E5FB0546FCF7ACF9044603E06A
:101380000020FCF7DDFB0446204670BD01480078D4
:10139000704700003E00002070B505460024032D74
:1013A00000D170BD002D01D0012D1BD18121032062
:1013B000800204F011FB8021134804F00DFB322160
:1013C0001248FFF737FB002409E0A200104BD218A7
:1013D0009178A200985A04F0FFFA601CC4B23B2C2A
:1013E000F3DB0FE0022D0DD1002409E0A200094B30
:1013F000D2189178A200985A04F0EEFA601CC4B298
:101400003B2CF3DB00BFCCE702060000A086010006
:101410005418020040190200F8B5002100240023EE
:10142000002200BF0AE001258D40ABB205881D40B7
:101430002C469C4200D10A464D1CA9B21029F2DB71
:101440000588FF2D1FDC284D6D7E0688B543264E8E
:10145000757635462D7E0688B543234E357635465E
:101460006D7E8678F607F60F964035431E4E7576EC
:1014700035462D7E867802273E40760896403543D5
:10148000194E357622E0184DED7E0688B543164E8E
:10149000F5763546AD7E0688B543134EB57685782C
:1014A000ED07ED0F1646083EB5400F4EF67E35436C
:1014B0000D4EF5768578022635406D081646083EB5
:1014C000B540094EB67E3543074EB57600250095EA
:1014D00005E000BF6D462D786D1CEEB200966D469E
:1014E0002D78012DF5D9F8BD206B0440C107C90F37
:1014F000002905D00021394A1171002238490A71AA
:1015000002210140002905D00021344A1172002235
:1015100033490A7204210140002905D000212F4AD5
:10152000117300222E490A7308210140002905D0B9
:1015300000212A4A1174002229490A74102101400D
:10154000002905D00021254A1175002224490A7579
:1015500020210140002905D00021204A11760022D7
:101560001F490A7640210140002904D000221B496E
:101570004A711B494A7180210140002904D0002290
:1015800016494A7216494A72FF2101310140002969
:1015900004D0002211494A7311494A7301214902BA
:1015A0000140002904D000220C494A740C494A74B5
:1015B000012189020140002904D0002207494A750F
:1015C00007494A750121C9020140002904D00022BF
:1015D00002494A7602494A7670470000006000409E
:1015E00000610040C107C90F002905D001223C4914
:1015F0000A7100213B4A117102210140002905D0E6
:10160000012237490A720021364A11720421014031
:10161000002905D0012232490A730021314A117391
:1016200008210140002905D001222D490A7400211A
:101630002C4A117410210140002905D001222849AB
:101640000A750021274A117520210140002905D083
:10165000012223490A760021224A117640210140C5
:10166000002905D001221E494A7100221D494A71F4
:1016700080210140002905D0012219494A72002227
:1016800018494A72FF2101310140002905D0012289
:1016900013494A73002213494A7301214902014048
:1016A000002905D001220E494A7400220D494A74CE
:1016B000012189020140002905D0012208494A750B
:1016C000002208494A750121C9020140002905D0BC
:1016D000012203494A76002202494A7670470000F7
:1016E000006100400060004010B50C480078002800
:1016F00003D00B4A50689168884708484078002812
:1017000003D0084A506891688847044880780028C8
:1017100003D0054A50689168884710BD00600040BA
:1017200010030020900400201006002010B5084887
:101730000079002803D0074A106951698847044896
:101740004079002803D0044A50689168884710BD4A
:1017500000600040100300209C04002010B50848E1
:10176000007A002803D0074AD069116A88470448E4
:10177000407A002803D0044A50689168884710BD19
:101780000060004010030020A804002010B50848A5
:10179000007B002803D0074A906AD16A8847044832
:1017A000407B002803D0044A50689168884710BDE8
:1017B0000060004010030020B404002010B5084869
:1017C000007C002803D0074A506B916B884704487F
:1017D000407C002803D0044A50689168884710BDB7
:1017E0000060004010030020C004002010B508482D
:1017F000007D002803D0074A106C516C88470448CC
:10180000407D002803D0044A50689168884710BD85
:101810000060004010030020CC04002010B50848F0
:10182000007E002803D0074AD06C116D8847044819
:10183000407E002803D0044A50689168884710BD54
:101840000060004010030020D804002010B50848B4
:10185000407F002803D0074A5068916888470448B1
:10186000007F002803D0044A906DD16D884710BDD9
:1018700000600040E40400201003002010B5084878
:101880004078002803D0074A506891688847044888
:101890000078002803D0044A506E916E884710BD2E
:1018A00020600040F00400201003002010B509481B
:1018B0000079002803D0084A106F516F8847054807
:1018C000001D4078002803D0044A5068916888477A
:1018D00010BD00002060004010030020FC04002028
:1018E00010B5034AD06F78329168884710BD000068
:1018F0001003002010B5024A50689168884710BD57
:101900009403002010B50948007C002803D0084A41
:10191000506891688847054810304078002803D007
:10192000044A50689168884710BD0000206000405C
:10193000A00300202005002010B5024A50689168DD
:10194000884710BDAC03002010B5024A506891686A
:10195000884710BDB803002010B50948007F002853
:1019600003D0084A50689168884705481C30407881
:10197000002803D0044A50689168884710BD0000D1
:1019800020600040C40300204405002010B50C482E
:101990000078002803D00B4A5068916888470848AF
:1019A0004078002803D0084A506891688847044866
:1019B0008078002803D0054A50689168884710BD98
:1019C00040600040D003002050050020D0060020D9
:1019D00010B50D480079002803D00C4A5068916872
:1019E00088470948001D4078002803D0084A5068FD
:1019F000916888470448001D8078002803D0054A74
:101A000050689168884710BD40600040DC030020AA
:101A10005C050020DC06002010B50D48007A002887
:101A200003D00C4A506891688847094808304078CC
:101A3000002803D0084A5068916888470448083055
:101A40008078002803D0054A50689168884710BD07
:101A500040600040E803002068050020E806002000
:101A600010B50D48007B002803D00C4A50689168DF
:101A7000884709480C304078002803D0084A50684D
:101A80009168884704480C308078002803D0054AC4
:101A900050689168884710BD40600040F403002002
:101AA00074050020F406002010B50D48007C0028C5
:101AB00003D00C4A50689168884709481030407834
:101AC000002803D0084A50689168884704481030BD
:101AD0008078002803D0054A50689168884710BD77
:101AE0004060004000040020800500200007002026
:101AF00010B5024A50689168884710BD0C04002058
:101B000010B50948007E002803D0084A5068916843
:101B10008847054818304078002803D0044A5068A8
:101B20009168884710BD0000406000401804002004
:101B30009805002010B50948007F002803D0084A06
:101B400050689168884705481C304078002803D0C9
:101B5000044A50689168884710BD0000406000400A
:101B600024040020A405002010B5084800780028AF
:101B700003D0074A50689168884704484078002895
:101B800003D0044A50689168884710BD60600040E7
:101B900030040020B005002010B509480079002865
:101BA00003D0084A5068916888470548001D40786E
:101BB000002803D0044A50689168884710BD00008F
:101BC000606000403C040020BC05002010B50948BE
:101BD000007A002803D0084A506891688847054871
:101BE00008304078002803D0044A5068916888473C
:101BF00010BD00006060004048040020C8050020BF
:101C000010B5024A50689168884710BD54040020FE
:101C100010B5024A50689168884710BD60040020E2
:101C200010B50948007D002803D0084A5068916823
:101C30008847054814304078002803D0044A50688B
:101C40009168884710BD0000606000406C0400206F
:101C5000EC05002010B50948007E002803D0084A92
:101C6000506891688847054818304078002803D0AC
:101C7000044A50689168884710BD000060600040C9
:101C800078040020F805002010B50948007F0028DE
:101C900003D0084A50689168884705481C3040784E
:101CA000002803D0044A50689168884710BD00009E
:101CB00060600040840400200406002010B5FE4847
:101CC00000688079002806D001286ED002286DD0E7
:101CD00003286CD104E2F8480068407903000EF054
:101CE000EBFF0A0614BC2BBC47BC67BC9BBC0BF0CB
:101CF0002DF80020F0490968C873EF480068407962
:101D0000401CED4909684871AEE0EC490969EA4AAE
:101D10001268D27A885C0BF091F8E7480068407945
:101D2000401CE54909684871E34800684079401C57
:101D3000E1490968487197E001F020FF002810D1BF
:101D40000BF07CF8DC4800684079401CDA490968EF
:101D50004871D94800684079401CD74909684871E2
:101D600005E00BF01DF80020D349096848717BE0BD
:101D700001F004FF002811D101200BF05FF8CE48DC
:101D800000684079401CCC4909684871CA4800681D
:101D90004079401CC8490968487105E00BF000F81B
:101DA0000020C549096848715EE05FE0FEE0A3E1FC
:101DB00001F0E4FE002828D1BF490968C97A24222D
:101DC0005143BF4A12688918BB4A1268D27B885CAB
:101DD0000BF034F8B8480068C07B401CB64909686D
:101DE000C873B5480068C07B242814D3B248006883
:101DF0004079401CB04909684871AF480068407993
:101E0000401CAD490968487105E00AF0C9FF00208F
:101E1000A9490968487127E001F0B0FE002815D1F2
:101E2000A5480068C07A401CA3490968C872A24846
:101E30000068C07AA1490978884207DB00209E49E2
:101E40000968C87201209C49096888710AF0A8FFD6
:101E5000002099490968487106E00AF0A1FF0020B6
:101E600095490968487100BF00BF4FE1924800687A
:101E7000407903000EF020FF080513912A91479145
:101E800070910AF063FF00208B490968C8738A4883
:101E900000684079401C88490968487184E0874996
:101EA0000969854A1268D27A885C0AF0C7FF8248BD
:101EB00000684079401C8049096848717E48006884
:101EC0004079401C7C49096848716DE001F056FE7C
:101ED000002811D126200AF0B1FF77480068407928
:101EE000401C754909684871734800684079401C76
:101EF00071490968487105E00AF052FF00206E49F7
:101F00000968487150E001F039FE00281DD1012018
:101F10000AF094FF68480068C07B401C6649096865
:101F2000C87365480068C07B242814D362480068E1
:101F30004079401C6049096848715F4800684079F1
:101F4000401C5D490968487105E00AF029FF00203E
:101F500059490968487127E001F010FE002815D1A1
:101F600055480068C07A401C53490968C8725248F5
:101F70000068C07A51490978884207DB00204E4941
:101F80000968C87202204C49096888710AF008FF84
:101F9000002049490968487106E00AF001FF002065
:101FA00045490968487100BF00BFAFE0424800687A
:101FB000407903000EF080FE0805138B2A8B478BB7
:101FC000638B0AF0C3FE00203B490968C8733A4896
:101FD00000684079401C3849096848717EE03749FB
:101FE0000969354A1268D27A885C0AF027FF3248BC
:101FF00000684079401C3049096848712E480068E3
:102000004079401C2C490968487167E001F0B6FD31
:10201000002811D125200AF011FF274800684079D7
:10202000401C254909684871234800684079401CD4
:1020300021490968487105E00AF0B2FE00201E49F6
:10204000096848714AE001F099FD002810D10AF0B2
:10205000F5FE194800684079401C17490968487125
:10206000154800684079401C13490968487105E02B
:102070000AF096FE00201049096848712EE001F030
:102080007DFD002815D10C480068C07A401C0A4923
:102090000968C87208480068C07A08490978884207
:1020A00007DB002004490968C87203200249096857
:1020B00088710AF075FE05E0E8070020542F002023
:1020C000E4070020002012490968487106E00AF080
:1020D00067FE00200E490968487100BF00BF15E087
:1020E00000200B4909688871094909684871062070
:1020F00007490968C87009E00AF052FE0020044947
:102100000968487102490968887100BF00BF10BDA5
:10211000E807002010B56A480068407903000EF017
:10212000CBFD090610C627C644C6608EC6000AF05D
:102130000DFE634800684079401C61490968487198
:10214000BCE0604909695E4A1268D27A885C0AF08C
:1021500075FE5B4800684079401C59490968487120
:10216000574800684079401C554909684871A5E006
:1021700001F004FD002811D14F200AF05FFE504805
:1021800000684079401C4E49096848714C48006815
:102190004079401C4A490968487105E00AF000FE90
:1021A000002047490968487188E001F0E7FC0028F1
:1021B00010D10AF043FE424800684079401C404973
:1021C000096848713E4800684079401C3C490968EC
:1021D000487105E00AF0E4FD0020394909684871BA
:1021E0006CE001F0CBFC002822D135480068C07AB1
:1021F000401C33490968C87231480068C07A3149C7
:10220000097888420FDB00202D490968C8722C48E4
:1022100000684079401C2A49096848710020284913
:102220000968486208E0002025490968487103E010
:1022300000202349096848710AF0B2FD3EE02048B9
:102240000068407C002816D01E48C068002803D0D3
:102250001C48C1681920884700201949096848624C
:102260001749096848711649096888710520144999
:102270000968C8701AE012480068406A282807D226
:102280000F480068406A401C0D49096848620DE02B
:1022900000200B49096848620949096848710849E2
:1022A00009688871052006490968C87006E00AF0C7
:1022B00077FD002002490968487100BF00BF10BDCA
:1022C000E8070020542F002010B50024F7480068CC
:1022D000807A01287ED1F5480068C07900287AD03C
:1022E000F24800688079002804D0012874D00228C0
:1022F00073D191E1ED480068007B24286ED2EB4851
:102300000068C07901287AD1002475E0E7480068A8
:10231000C07A24214843E64909684018E34909681E
:10232000097B415CE1480068C07A24225043E14ABD
:1023300012688018DD4A1268127B805C814229D0C5
:10234000DA480068C07A24214843DA49096840180D
:10235000D6490968097B415CD4480068C07A2422C8
:102360005043D34A12688018D04A1268127B8154B5
:10237000CE480068407B242805D3CC480068007B09
:10238000CA4909684873C9480068007BC749096899
:10239000887308E0C5480068407B242803D20120E8
:1023A000C24909688871C1480068007B401CBF4968
:1023B00009680873BD480068007B242808D3BB481F
:1023C0000068407B242803D20120B849096888713D
:1023D000B64805E0D3E1CDE169E0BAE138E00EE0CE
:1023E0000068007B242804D2B04800688079012866
:1023F00000D103E0601CC4B2242C87D356E0002433
:1024000013E0AA480068C07A24214843A949096812
:102410004018015DA5480068C07A24225043A44AB0
:10242000126880180155601CC4B2242CE9D3002026
:102430009E490968487323209C49096888730120D4
:102440009A490968887124209849096808732DE021
:10245000002096490968087394480068C07A401CB7
:1024600092490968C87291480068C07A924909780F
:10247000884217DB8D480068007C012804D10220C7
:102480008A490968887106E00020884909688871CE
:1024900086490968C871002084490968C87283495F
:1024A00009680874002081490968487161E17F4822
:1024B0000068407903000EF0FFFB080513A62AA66A
:1024C00051A68EA601207949096808740AF03EFCDD
:1024D000764800684079401C74490968487199E061
:1024E00075490969714A1268D27A885C0AF0A6FCBB
:1024F0006E4800684079401C6C49096848716B4817
:1025000000684079401C69490968487182E001F01F
:1025100035FB00281BD165490968497B491CC8B2B5
:102520000AF08CFC61480068407B60490968C87308
:102530005E4800684079401C5C49096848715B4806
:1025400000684079401C59490968487105E00AF063
:1025500027FC00205549096848715BE001F00EFB3B
:1025600000282BD151490968C97A24225143504A85
:10257000126889184D4A1268D27B885C0AF05EFCAA
:102580004A480068C07B401C48490968C8734748EE
:102590000068C07B45490968897B88421ADD434849
:1025A00000684079401C4149096848713F4800680B
:1025B0004079401C3D49096848710BE00AF0F0FB86
:1025C0003A480068407B39490968C8730020374998
:1025D000096848711EE001F0D1FA00280CD1334996
:1025E00009688871242031490968C8732F4909682E
:1025F00048732E49096888730AF0D2FB00202B49E2
:102600000968487106E00AF0CBFB002027490968F9
:10261000487100BF00BFACE0244800684079030067
:102620000EF04AFB08050F8E268E4C8E688E0AF03F
:102630008DFB1E4800684079401C1C4909684871A0
:1026400085E01D490969194A1268D27A885C0AF046
:10265000F5FB164800684079401C14490968487128
:10266000124800684079401C1049096848716EE0C2
:1026700001F084FA002811D125200AF0DFFB0B4875
:1026800000684079401C094909684871074800689A
:102690004079401C05490968487105E00AF080FB53
:1026A000002002490968487151E00000E807002055
:1026B000E4070020E0070020542F002001F05EFA1C
:1026C000002810D10AF0BAFB644800684079401C29
:1026D000624909684871614800684079401C5F4957
:1026E0000968487105E00AF05BFB00205B49096856
:1026F00048712CE001F042FA00281AD157480068CE
:10270000C07A401C55490968C87254480068C07AAC
:102710005349097888420CDB002050490968C87287
:102720004E49096888714D49096848714B490968E3
:10273000C8710AF035FB002048490968487106E075
:102740000AF02EFB002045490968487100BF00BF10
:102750000FE00AF025FB00204049096848713F4915
:10276000096888713D49096808733C490968C8725D
:1027700000BF71E000203949096888726CE0374871
:102780000068807A022867D134480068007A0028FF
:102790005ED0324800684079002804D001280CD06F
:1027A000032846D11BE00AF0D1FA2C480068407992
:1027B000401C2A490968487149E000200AF03EFBA4
:1027C000264800684079401C24490968487123481C
:1027D00000684079401C21490968487137E00AF0D7
:1027E0007FFA002812D11D4800684078401C1B4920
:1027F00009684870194800684078032812D301F02E
:102800005DFA00201549096848700BE00020134963
:1028100009680872AA2011490968887000200F49C8
:10282000096848700AF0BCFA00200C490968487130
:102830000DE00AF0B5FA0020084909684871074917
:1028400009684870AA2005490968887000BF03E03C
:10285000002002490968887210BD0000E8070020C6
:10286000542F0020F8B504460D4600260C20604386
:102870001D49085C002801D00120F8BD0C206043F0
:102880001949401885600C20604340188068002872
:1028900001D10120F1E701210C206043124A1154BB
:1028A00000222046E317DB0E1B185B115B01E31AC5
:1028B0009B000E4FDB19E717FF0E3F197F11DA550A
:1028C0000EF02CFA00222046E317DB0E1B185B11DA
:1028D0005B01E31A9F00064BFB18E717FF0E3F1939
:1028E0007F11DA553046C8E7100300200060004031
:1028F0000061004000BFFEE709480088401C08490D
:102900000880084600880749884208DD06480078A4
:10291000002804D0084602490880012088707047CA
:10292000E8000020DC050000EC00002010B5154890
:102930008078012824D11448007801280CD113484C
:102940000078012808D1002011498870084602F05B
:1029500061FE00200D4908700B48007802280CD158
:102960000C480078012808D10020094988700846E1
:1029700002F050FE0020074908700020024908704C
:1029800010BD0000E8000020EC000020EE00002058
:10299000F1000020EF0000207047000010B500F0AB
:1029A0005DFE012803D1002001490880887010BD18
:1029B000E8000020F0B505460E46174600243A46CA
:1029C0003146284600F058FE00BF42E000202101B9
:1029D000394A126850522101374A126889184880D2
:1029E00000212001344A1268801881802001324A77
:1029F00012688018C18020012F4A12688018017265
:102A000020012D4A12688018417220012A4A12685A
:102A1000801881722001284A12688018C172002033
:102A20002101254A12688918087300212001224AD1
:102A3000126880184173002021011F4A126889180A
:102A40008873002120011C4A12688018C173601C21
:102A5000C4B21A484078A042B8DC6420184909681A
:102A600008807D20C000164909684880154814492F
:102A7000096888807D20000111490968C8801049D3
:102A80000968088110480E49096848810F480C49B7
:102A90000968888140000A490968C88132200849CC
:102AA00009680882FF20F530054909684882044911
:102AB00009688882F0BD0000A80700209C0700205C
:102AC000A40700204C04000010270000307500000F
:102AD00038B5002404E0002013490855601C84B276
:102AE000282CF8D301216846417001706A460F49CD
:102AF0000D48FFF75FFF7D21C900322000F0ACF9DF
:102B00000B490C4800F0C6F90948643000F058F948
:102B10000748C83000F064F9074800F077F9074823
:102B200000F08AF938BD000064280020281E020049
:102B300028230000B80B00005424000010270000D8
:102B400010B524480078002803D1012021490870DD
:102B50003EE020480078012810D11F480078012865
:102B600008D100201D498870084602F053FD00205E
:102B70001949087002201749087029E015480078A3
:102B8000022810D116480078012808D100201349E6
:102B90008870084602F03EFD0020114908700320AD
:102BA0000C49087014E00B480078032803D1052075
:102BB000084908700CE007480078052803D005484C
:102BC0000078062804D100200249087005490870E1
:102BD00010BD0000EC000020EE000020F1000020FD
:102BE000EF000020F0000020F8B5002400250026AA
:102BF0003548007800281ED134480078002803D1D9
:102C000001203249087016E030480078012803D1CD
:102C100002202E4908700EE02C480078022803D1CB
:102C200003202A49087006E028480078032802D1CA
:102C30000020264908702448007801280ED101247C
:102C400017250026224801233246294600902046B7
:102C500001F09CFE01201F49087034E01A480078FA
:102C600002280FD101243B2500261948401C0123CE
:102C7000324629460090204601F088FE0120164980
:102C8000087020E01048007803280DD1FEF7FEF808
:102C9000002803D101201149087102E000200F49EA
:102CA00008710DF0DBFF0EE007480078052803D11E
:102CB00006200549087006E003480078062802D17E
:102CC000052001490870F8BDEC000020ED0000204F
:102CD000F1000020EE000020EF000020542800202A
:102CE00010B5044623000DF0E7FF095B060E16172A
:102CF0001819595A5E00F9F7F5FE2C49884201D39C
:102D0000FFF772FF50E0F9F7EDFE2849884201D342
:102D1000FFF716FF48E047E046E045E0F9F7E2FE3E
:102D20002249884239D301F0E1FD21480078032887
:102D300014D120480078002810D1FEF7B3F80028FD
:102D400006D101201C4988608868FAF763FF05E016
:102D50000020194988608868FAF75CFF14480078F9
:102D6000012805D113480078002801D1FAF74CF862
:102D700010480078052803D10120104908700AE0A6
:102D80000C480078062803D102200C49087002E0A4
:102D900000200A4908700BF0FFFC05E004E003E0A6
:102DA000FFF7AAFD00E000BF00BF10BDB80B000098
:102DB000ED000020EC00002054280020F00000204E
:102DC00001460020054A126852898A4201DC01202E
:102DD00002E0024A1268118170470000A407002037
:102DE00001460020084A126812898A4201DB01204C
:102DF00009E0054A126892898A4201DC012002E05A
:102E0000014A126851817047A40700200146002042
:102E1000084A126852898A4201DB012009E0054A0A
:102E20001268D2898A4201DC012002E0014A12685C
:102E300091817047A407002001460020054A1268CE
:102E400092898A4201DB012002E0024A1268D181A4
:102E500070470000A4070020024600200C4B1B68AE
:102E60001B8A934201DD012010E08A4201DB012030
:102E70000CE0074B1B689B888B4201DC012005E0BE
:102E8000034B1B681A80024B1B6859807047000077
:102E9000A4070020024600200C4B1B681B8A9342AB
:102EA00001DD012010E08A4201DB01200CE0074B2C
:102EB0001B685B88934201DB012005E0034B1B6824
:102EC0009A80024B1B68D98070470000A40700203D
:102ED00070B5044600250C206043FE49096840187F
:102EE0004068002807D00C216143FA4A126889180B
:102EF0004868804705460C206043F6490968085C2D
:102F0000002873D10C206043F2490968401880689A
:102F1000002874D02001F04909684018C07A0228BE
:102F20000AD1032D08D10C206043EA4A12688018A8
:102F300081680120884762E02001E749096840185C
:102F4000C07A02280AD1042D08D10C206043E14A3E
:102F50001268801881680220884750E02001DE490D
:102F600009684018C07A02280AD1052D08D10C2022
:102F70006043D84A126880188168032088473EE081
:102F80002001D54909684018C07A02280AD1062DC7
:102F900008D10C206043CF4A126880188168042051
:102FA00088472CE02001CC4909684018C07A0228E3
:102FB0000AD1072D08D10C206043C64A1268801838
:102FC0008168052088471AE02001C3490968401834
:102FD000C07A02280BD1082D09D10C206043BD4ACC
:102FE0001268801881680620884708E00DE00C20F0
:102FF0006043B84A12688018816800208847200121
:10300000B54909684018C5720CE30C206043B1490A
:103010000968085C012873D10C206043AD49096838
:1030200040188068002874D02001AB490968401816
:10303000C07A03280AD1022D08D10C206043A54A8A
:103040001268801881680120884762E02001A24947
:1030500009684018C07A04280AD1022D08D10C2032
:1030600060439C4A1268801881680220884750E0BB
:103070002001994909684018C07A05280AD1022D13
:1030800008D10C206043934A12688018816803209D
:1030900088473EE02001904909684018C07A062818
:1030A0000AD1022D08D10C2060438A4A1268801888
:1030B0008168042088472CE020018749096840186E
:1030C000C07A07280AD1022D08D10C206043814A1A
:1030D000126880188168052088471AE020017E491F
:1030E00009684018C07A08280BD1022D09D10C209C
:1030F0006043784A1268801881680620884708E093
:103100000DE00C206043734A12688018816800202B
:1031100088472001704909684018C57282E20C2076
:1031200060436C490968085C0228F7D1002D7DD105
:10313000200169490968085A68490968098A88426A
:1031400075DA200164490968085A0A3081B2200101
:10315000614A1268115220015F490968085A5F49A3
:103160000968098A884231DB20015B4909684018F7
:1031700040885A4909680988884227DB2001564956
:1031800009684018408855490968498888421DDC0B
:1031900000202101504A12688918488020014E49B8
:1031A00009684018807A0028B8D10C20604349494A
:1031B0000968401880680028B0D00C206043454A58
:1031C000126880188168012088472BE2200142495B
:1031D0000968085A41490968098A88429EDB20012A
:1031E0003D490968401840883C49096889888842F7
:1031F00094DB20013849096840184088374909683C
:10320000C98888428ADC00202101334A1268891863
:1032100048802001304909684018807A0028D4D1BC
:103220000C2060432B490968401801E063E00BE083
:1032300080680028C9D00C206043264A1268801894
:10324000816802208847EDE100202101224A1268AE
:10325000891848802101204A12688918C872002103
:1032600020011D4A12688018C18020011A4A126884
:10327000801841722001184A12688018817218481B
:1032800001782001144A126880180172002021017F
:10329000114A12688918888021010F4A126889181A
:1032A000087321010C4A12688918487321010A4ADF
:1032B00012688918887300212001074A1268801853
:1032C000C1730C20604303490968401880680028D6
:1032D000B9D007E0A0070020A8070020A40700201D
:1032E0009C0700200C206043CF4A12688018816838
:1032F0000020884796E1012DA5D12001CB4909681E
:103300004018C07AA84225D000212001C74A12687F
:103310008018418000202101C44A12688918C880A1
:103320002001C24909684018C572C14800782101CE
:10333000BE4A12688918487200202101BB4A1268EF
:1033400089188880BA4801782001B84A1268801824
:10335000017267E12001B54909684018007AB44953
:103360000978884220D0B24800782101AF4A12681B
:10337000891808722001AD4909684018407AAC49A3
:103380000978884209D02001A84909684018808836
:103390002101A64A12688918C88000212001A34A89
:1033A00012688018818012E02001A0490968401845
:1033B0008088A04988420AD220019C4909684018A7
:1033C00080880A302101994A126889188880200172
:1033D0009649096840184088964988420AD22001D7
:1033E00092490968401840880A3021018F4A1268C2
:1033F0008918488020018D4909684018407A8C4915
:103400000978884205D001202101884A126889186C
:1034100088722001854909684018408886490968F2
:103420000988884204DB00212001804A1268115279
:1034300020017E4909684018807A00287ED10C203E
:1034400060437949096840188068002877D02001D6
:10345000764909684018408877490968098988428F
:1034600014DB2001714909684018007B00280DD148
:103470000C2060436C4A12688018816803208847DA
:1034800001202101694A12688918087320016749DF
:10349000096840184088684909684989884214DBEE
:1034A0002001624909684018407B00280DD10C209A
:1034B00060435D4A126880188168042088470120B3
:1034C00021015A4A1268891848732001574909682E
:1034D00040184088584909688989884214DB2001CE
:1034E000524909684018807B00280DD10C206043A8
:1034F0004D4A126880188168052088470120210103
:103500004A4A126889188873200148490968401896
:10351000408849490968C989884210DB200143492C
:1035200009684018C07B00287CD10C2060433E4ACB
:103530001268801881680620884701E007E03BE0B8
:1035400001202101394A12688918C8736AE02001F4
:10355000364909684018407A01282ED1344800784D
:1035600002282AD12001314909684018C08832490F
:103570000968498A884255DB20012C4909684018AE
:1035800080882D490968898A88424BDB0C2060437A
:103590002549096840188068002843D00C20604302
:1035A000214A12688018816807208847002021017D
:1035B0001E4A12688918487234E020011B490968C4
:1035C0004018407A02282DD119480078012829D1C5
:1035D0002001164909684018C08817490968898A76
:1035E00088421FDB20011149096840188088124970
:1035F0000968498A884215DB0C2060430A4909683A
:103600004018806800280DD00C206043064A1268DC
:10361000801881680820884700202101034A126829
:103620008918487270BD0000A0070020A80700207C
:103630009C070020F0FF0000A407002010B5002424
:1036400000BF04E02046FFF743FC601CC4B2024800
:103650004078A042F6DC10BD9C07002010B5002485
:10366000044802F009FA002800D000E001242046B6
:1036700010BD00000304000010B5074B14781C7047
:1036800054785C70054B1960054B1860034618337D
:10369000044C236010BD00009C070020A007002000
:1036A000A4070020A807002010B50446012C09D16A
:1036B000FF220C21002000F0F9F80121022004F083
:1036C00009FF08E000220C21104600F0EFF800216D
:1036D000022004F0FFFE10BD10B5002404210848AC
:1036E000F7F78CFD552801D1012407E0042001F0F3
:1036F0006FF8002801D0002400E00124204610BD0E
:103700006808002010B50446012C09D1FF221C21B5
:10371000002000F0CBF80121062004F0DBFE08E0D9
:1037200000221C21104600F0C1F80021062004F000
:10373000D1FE10BD10B50024062001F049F8002884
:1037400001D0012400E00024204610BD10B504463D
:10375000012C09D1FF221721002000F0A7F8012138
:10376000042004F0B7FE08E000221721104600F004
:103770009DF80021042004F0ADFE10BD0020044996
:10378000097A002901D0012000E0002070470000E4
:10379000680A002010B50446022C1CD100220D211D
:1037A000104600F083F8FDF763FC002809D0FF22E3
:1037B0000B21002000F07AF801210D2004F08AFE90
:1037C00058E000220B21104600F070F800210D2077
:1037D00004F080FE4EE0032C1CD100220B21104689
:1037E00000F064F8FDF744FC002809D0FF220D2109
:1037F000002000F05BF801210D2004F06BFE39E0A1
:1038000000220D21104600F051F800210D2004F097
:1038100061FE2FE0042C0ED1FF220D21002000F0CC
:1038200045F800220B21104600F040F801210D2040
:1038300004F050FE1EE0012C0ED100220D21104696
:1038400000F034F8FF220B21002000F02FF80121B6
:103850000D2004F03FFE0DE000220D21104600F087
:1038600025F800220B21104600F020F800210D2041
:1038700004F030FE10BD000010B500240A480078A6
:10388000012801D101240CE0FCF752FD012801D1EF
:10389000032406E0FCF74CFD022801D1022400E0DD
:1038A0000424204610BD0000F900002010B5064B8E
:1038B0001B78834207DD242905D224234343034C8C
:1038C00024681B195A5410BD542F0020E007002013
:1038D00010B574480068407903000DF0EDF90B074E
:1038E00011D325D35A6D77D38DA8D30009F02EFAC2
:1038F0006C4800684079401C6A4909684871CFE00B
:1039000069494969087809F099FA66480068407978
:10391000401C644909684871624800684079401C4D
:10392000604909684871BBE000F028F9002811D10E
:103930007F2009F083FA5B4800684079401C5949B0
:1039400009684871574800684079401C5549096822
:1039500048711DE0534800684078401C514909688F
:10396000487050480068407803280BD300204D4928
:1039700009684870AA204B490968887003204949A2
:103980000968C87009F00CFA0020464909684871B6
:1039900086E000F0F3F8002807D14248006840793B
:1039A000401C40490968487103E000203D4909680E
:1039B000487109F0F5F973E009F0C8F93948006871
:1039C0004079401C37490968487169E036494969BE
:1039D0000978491CC8B209F031FA324800684079C8
:1039E000401C3049096848712E4800684079401CE5
:1039F0002C490968487153E000F0C0F800280FD145
:103A000009F076F9274909688870012009F0EAF978
:103A1000244800684079401C22490968487105E043
:103A200009F0BEF900201F490968487138E01D48B7
:103A30000068807818280CD102201A49096808709B
:103A40000020184909684870042016490968C870A0
:103A500011E0144800684078401C12490968487019
:103A6000104800684078032805D300F027F90020AB
:103A70000C490968487009F093F900200949096860
:103A800048710DE009F08CF9002006490968487179
:103A9000044909684870AA2002490968887000BF73
:103AA00000BF10BDE8070020542F002010B531489A
:103AB00000684079002804D001280CD0032848D1A0
:103AC0001DE009F043F92B4800684079401C294962
:103AD000096848714BE028490969087809F0AEF98E
:103AE000244800684079401C2249096848712148EF
:103AF00000684079401C1F490968487137E000F0B0
:103B00003DF800280CD101201A49096808700020EE
:103B1000184909684870042016490968C87011E0FE
:103B2000144800684078401C1249096848701148E0
:103B300000684078032805D300F0C0F800200D4944
:103B40000968487009F02CF900200A490968487191
:103B50000DE009F025F9002006490968487105497A
:103B600009684870AA2003490968887000BF00BF2F
:103B700010BD0000E8070020542F002010B509F008
:103B8000AFF804461F4800680078002838D01D4868
:103B90000068C078042833D3002C09D100211948CB
:103BA0000068C07A8200174800681430815027E00E
:103BB00014480068C07A81001248006814304058E8
:103BC0001149884211D20F480068C07A81000D481F
:103BD000006814304058401C0A490968C97A8A00B4
:103BE00008490968143188500AE000F067F800219C
:103BF00004480068C07A820002480068143081508E
:103C0000204610BDE8070020B80B000000B587B0C3
:103C10000120694608710848029008480390084846
:103C20000490084805900848069001A9074800F04C
:103C30000FF807B000BD0000753F0100655C010092
:103C4000450E0200951E0200941E0200CC280020A2
:103C5000F8B506460F46002400253946304600F0E8
:103C6000EFF900BF14E000250EE00021242060439E
:103C70000B4A12688018415524206043094A126893
:103C800080184155681CC5B2242DEED3601CC4B207
:103C900005480078A042E6DC00F010F8F8BD00000E
:103CA000E0070020E4070020542F002001200249F3
:103CB0000968087170470000E807002010B500F09F
:103CC00073F9002003490968087002490968C8703F
:103CD00010BD0000E807002007480068C0780628EB
:103CE00008D105480068C079002803D101200249A5
:103CF0000968C87170470000E807002010B55548F2
:103D00000068C07803000CF0D7FF08671D1A17146D
:103D1000110E056650484068002803D04E4841689F
:103D20000020884793E000F0E5F890E000F0C6F846
:103D30008DE000F0D1F88AE0FFF7B8FE87E0FFF7EA
:103D4000C7FD84E044484068002803D042484168E9
:103D5000012088473F480068407C00281AD03E4830
:103D6000C068002803D03C48C168C82088470020AC
:103D7000384909684862374800680078002804D04C
:103D8000042034490968C87024E0022031490968D8
:103D9000C8701FE02F480068406A401C2D49096820
:103DA00048622C480068406A7D21C900884211D3CE
:103DB00000202849096848622648006800780028E1
:103DC00004D0042023490968C87003E00220214977
:103DD0000968C8703BE000BF1F484068002803D056
:103DE0001D484168002088471A480068407C002828
:103DF00013D01948C068002803D01748C168C820EC
:103E00008847002013490968486212480068C07852
:103E1000401C10490968C87018E00E480068406AE4
:103E2000401C0C49096848620A480068406A7D21C4
:103E3000C90088420AD3002006490968486205483B
:103E40000068C078401C03490968C87000BF00BF03
:103E500010BD0000E8070020542F002010B51548C1
:103E60000068C078072824D00120124909684874E6
:103E700008E011488068002802D00F498868804710
:103E8000FFF73CFF0B480068C0780628F1D10948CD
:103E90000068007A0028ECD106480068C079002844
:103EA000E7D104480068807A0028E2D10149096816
:103EB000487410BDE8070020542F002010B50548B5
:103EC00000680078012802D1FDF7F8FE01E0F5F75F
:103ED00015FC10BDE807002010B505480068007803
:103EE000012802D1FEF716F901E0F5F7E5FF10BD54
:103EF000E807002010B51D480068807A002829D105
:103F00001A480068007A002803D00220174909687F
:103F1000887216480068C079002803D00120134930
:103F200009688872114800680079012812D10020C0
:103F30000E49096808710D490968887207200B4904
:103F40000968C8700A484068002803D008484168DA
:103F500000208847054800680078012802D1FEF754
:103F6000B3F901E0F6F782F810BD0000E807002081
:103F7000542F002010B504462146084801F098FD52
:103F800007480078002805D1002C03D032210548CD
:103F9000FCF750FD0248047010BD00000103000052
:103FA000FA00002050C3000000202449096848702E
:103FB000AA202249096888700020204909684862BF
:103FC0001E49096808711D49096848711B4909683B
:103FD00088711A490968C87118490968087217492F
:103FE0000968887215490968C87214490968087314
:103FF00024201249096848731049096888730F49D9
:104000000968C87300200D49096808740B490968DC
:1040100048740A490968887408490968C8740749D6
:10402000096848610021054800688161034800680B
:10403000C16102480068016270470000E807002083
:1040400010B50A780D4B1860034628330C4C2360DA
:1040500024235343044628341B190A4C23600A4C7A
:104060004B6863608B68A360CB68E3604B696361F6
:104070000B6923610B78237010BD0000E807002056
:10408000E0070020E4070020542F002007480068C4
:10409000C078062808D105480068007A002803D1B6
:1040A000012002490968087270470000E8070020F3
:1040B00010B50446012C09D1FF2220210020FFF772
:1040C000F5FB0121084604F005FA08E00022202152
:1040D0001046FFF7EBFB0021012004F0FBF910BDB7
:1040E00010B50024032000F073FB002801D0012448
:1040F00000E00024204610BD10B50446032C0ED16C
:10410000FF2215210020FFF7D1FB002214211046C9
:10411000FFF7CCFB01210E2004F0DCF939E0022C82
:104120001CD1FCF7A5FF002809D0FF221421002094
:10413000FFF7BCFB01210E2004F0CCF908E00022BF
:1041400014211046FFF7B2FB00210E2004F0C2F943
:10415000002215211046FFF7A9FB1AE0012C0ED111
:10416000FF2214210020FFF7A1FB01210E2004F003
:10417000B1F9002215211046FFF798FB09E0002253
:1041800015211046FFF792FB002214211046FFF77D
:104190008DFB10BD10B50024F8F7A4FC0949884236
:1041A0000DD3FCF7C1FF002807D1FCF751FE012811
:1041B00001DD032404E0022402E0022400E00124E3
:1041C000204610BDB80B000010B50446012C09D1E3
:1041D000FF221D210020FFF769FB0121002004F0D0
:1041E00079F908E000221D211046FFF75FFB00214E
:1041F000084604F06FF910BD10B50024022000F04D
:10420000E7FA002801D0012400E00024204610BD78
:1042100010B50446012C09D1FF221E210020FFF712
:1042200045FB0121092004F055F908E000221E2178
:104230001046FFF73BFB0021092004F04BF910BDAD
:1042400070B5002400250026FCF7BAFC0546FCF7F3
:10425000C3FC064602210848F6F7D0FF552800D1D6
:1042600008E0012E01D1002404E0012D01D1012438
:1042700000E00024204670BD6808002010B5044608
:10428000012C09D1FF221F210020FFF70FFB012184
:10429000082004F01FF908E000221F211046FFF754
:1042A00005FB0021082004F015F910BD70B50024AD
:1042B0000025FCF70FFD054603211A48F6F79EFF7F
:1042C000552806D101201849088000201749088088
:1042D00023E016480088012811D114490880FCF712
:1042E00013FC762803DA01200F49088015E0FCF75B
:1042F0000BFC782811DB00200B4908800DE0012021
:104300000A490880FCF700FC762803DA01200649F8
:10431000088002E000200449088003480488204601
:1043200070BD000068080020160100201801002060
:1043300010B50446012C09D1FF2221210020FFF7EE
:10434000B5FA0121072004F0C5F808E00022212178
:104350001046FFF7ABFA0021072004F0BBF810BDB0
:1043600010B50024FCF7CCFF012801D1012400E0A6
:104370000024204610BD10B50446012C09D1FF22AF
:1043800016210020FFF792FA0121032004F0A2F881
:1043900008E0002216211046FFF788FA00210320CA
:1043A00004F098F810BD10B50024052000F010FAB4
:1043B000002801D0012400E00024204610BD10B5E3
:1043C0000446012C09D1FF2219210020FFF76EFAC3
:1043D0000121052004F07EF83CE0022C17D1FCF707
:1043E00047FE002809D0FF2219210020FFF75EFABE
:1043F0000121052004F06EF82CE00022192110465E
:10440000FFF754FA0021052004F064F822E0032CA1
:1044100017D1FCF733FE002809D0FF221921002014
:10442000FFF744FA0121052004F054F812E00022BD
:1044300019211046FFF73AFA0021052004F04AF846
:1044400008E0002219211046FFF730FA002105206C
:1044500004F040F810BD000010B50024FCF722FD68
:10446000012839D104214048F6F7C8FE552803D168
:1044700001203E49087032E0FCF7BAFB01280BD05E
:10448000FCF7B6FB022807D0FCF7B2FB032803D0E9
:10449000FCF7AEFB052803D10120344908701EE06B
:1044A000FCF7A6FB042803D102203049087016E06F
:1044B000FCF79EFB062803D103202C4908700EE070
:1044C000FCF796FB002803D0FCF792FB072806D1E7
:1044D00000202649087002E0002024490870244882
:1044E0000078022813D123480078002807D1FCF770
:1044F000BFFD002803D01D4800781D490870FCF757
:10450000B7FD1C490870FCF7B3FD044616E01848D7
:104510000078032812D117480078002807D1FCF74B
:10452000ADFD002803D01148007811490870FCF750
:10453000A5FD10490870FCF7A1FD04460C48007861
:1045400002280ED00A48007803280AD007480078CD
:104550000749087008460078002801D0012400E0CF
:104560000024204610BD0000680800201A01002029
:104570001B0100201C01002010B50446012C0ED1A7
:10458000FF221B210020FFF791F900221A2110467B
:10459000FFF78CF901210A2003F09CFF1EE0022C9A
:1045A0000ED1FF221A210020FFF780F900221B21E3
:1045B0001046FFF77BF901210A2003F08BFF0DE085
:1045C00000221A211046FFF771F900221B21104624
:1045D000FFF76CF900210A2003F07CFF10BD0000FA
:1045E00010B5002410480078012801D1012418E0FA
:1045F000FCF74AFD022803D0FCF74AFE02280FD13F
:10460000FCF714FE012809D1FCF744FD012803D072
:10461000FCF744FE012801D1012402E0022400E05D
:104620000224204610BD0000F900002010B5F8F764
:1046300073FA0446204610BD10B5034B0822034907
:10464000034800F013F910BD2D460100341E02008E
:104650008C28002070B506465C488068002804D08D
:104660005A4988688047054600E000250024A6E0F6
:10467000564841680C20604308184088A84207D07B
:10468000524841680C2060430818408802287DD1B8
:104690004E4841680C2060430818806800280CD000
:1046A0004A494A680C216143511888688047474944
:1046B0000968E2008918487009E0444841680C2004
:1046C0006043095C41480068E200801841703F483F
:1046D0000068E100401840783C490968E200895CC4
:1046E00088420FD039480068E100401841783748C7
:1046F0000068E2008154002034490968E20089180A
:1047000048605AE031480068E100401841782F487D
:1047100042680C2060431018407881421FD12B481A
:104720000068E10040184168284842680C20604356
:104730001018808881420BD824480068E100401896
:104740004068801921490968E2008918486034E00E
:1047500001201E490968E200891848802DE01B48A5
:104760000068E10040184168184842680C20604326
:104770001018C08881420DD814480068E100401824
:104780004068811911480068E20000E009E08018E3
:10479000416012E000200D490968E2008918488054
:1047A0000BE0002009490968E200891848800021CF
:1047B00006480068E20080184160601C84B203482B
:1047C0008089A04200DD53E770BD00000C2F00205F
:1047D0000146064A92898A4205DD044A1268CB00E6
:1047E000D218508800E00020704700000C2F0020F5
:1047F000002000BF14E00D494A680C2141435118C4
:10480000498801290AD10021084A1268C300D21838
:104810005180064A1268C300D2185160411C88B208
:10482000024989898142E6DC704700000C2F002094
:10483000002000BF13E00C494A680C214143511885
:104840004988002909D1084A1268C300D21851804A
:10485000054A1268C300D2185160411C88B202494F
:1048600089898142E7DC70470C2F0020F0B50446AF
:104870000020164DAB6069602C60AA8100BF1FE06C
:10488000124D6E680C254543755D104E3668C700A5
:10489000F61975700D4D6E680C254543755D0B4E10
:1048A0003668C700F5550025084E3668C700F6196A
:1048B0007580064E3668C700F6197560451CA8B2AB
:1048C000024DAD898542DBDCF0BD00000C2F0020DD
:1048D00070B505460E46002E05D031462846F3F742
:1048E00035FC044600E02C46204670BD10B5FCF7B0
:1048F00007FD012817D10C480078012813D00A4879
:10490000007803280FD00948007800280BD1FCF765
:1049100011FC0749884202D108F0CBF803E07D2062
:10492000000108F0CDF810BDED000020EC000020E3
:104930008813000008B50020009001226946052078
:10494000F9F790FD05490098886000200449087037
:10495000044908700449087008BD0000542800206C
:10496000EC000020EE000020EF00002008B5002041
:104970000090012269460520F9F774FD00200249E4
:1049800008710098886008BD5428002070B5049C08
:104990002578914216DD01280AD18D4206DAFF26DC
:1049A000F61AAE420ED3EE18F5B20BE0154609E04A
:1049B000022807D1954204DD9D4203DBEE1AF5B2D1
:1049C00000E00D46257070BD0D4A41685160816957
:1049D0009161C168D160416A5162016A11620168E6
:1049E00011604169516181689160C169D16101695A
:1049F0001161816A91620021024A117070470000C2
:104A0000282F0020DC07002010B5FFF7F1FEF7F794
:104A1000C5FE10BD10B5F7F7C1FEFFF709FF0AF09C
:104A20002FF90AF0CBF9FBF725FBFAF757F8FFF758
:104A300081FFF8F7FBFBF6F7E7FAF9F7F7F85521EE
:104A40000548F6F701FDF8F71FF9F9F769F8FAF7E5
:104A5000D1FFF6F7D3FC10BD740800201CB5002070
:104A60003A49087008F022F90020FCF795FC0CF098
:104A70004BFCF7F759F8F9F711F9F6F7BFFC0221EB
:104A80003348F6F729FF02213148F6F725FF0221C6
:104A90002F48F6F721FFF9F73FF9F6F7B9FC552152
:104AA0002C48F6F7D1FCF8F7EFF8F9F739F8F5F7F5
:104AB00047FEF6F737F9E12040020CF067F800F006
:104AC000B9FAF6F7A1FA08F0DFFAF7F767FEF9F797
:104AD0004BFEF8F73BFCF8F7B5FBFFF7ADFDFDF734
:104AE000F7FFFFF793F8FFF7B9F9F9F743FDFBF785
:104AF000EDFAF9F7F3FF184A184901200AF024FAF1
:104B00000022114601200AF063F908F03DF80AF08E
:104B10009DF80AF053F9FFF729FF0020104988712A
:104B200048710871012088704870142008700722AD
:104B30006846F3F7A2FB0199009801F009F80221F9
:104B4000012000F0E1FEFAF755FF1CBDF90000203E
:104B500068080020740800200090D003EC040000D6
:104B60000A0100207047000010B50446552C03D1FF
:104B700005494869804702E00349086880470020EA
:104B80000249087010BD0000282F0020DC0700201B
:104B900010B54648007803000CF08EF80A06111B89
:104BA00026303B465051738141484068002802D06E
:104BB0003F494868804701203C49087000BF3C4895
:104BC0008068002804D03A498868804737490870CF
:104BD00069E03748C068002802D03549C868804776
:104BE00003203249087000BF31480069002804D012
:104BF0002F49086980472D49087054E02C484069C6
:104C0000002802D02A4948698047002027490870B7
:104C100049E027488069002802D0254988698047F3
:104C200006202249087000BF2148C069002804D02E
:104C30001F49C86980471D49087034E000BF1B4800
:104C4000007807280AD11A48006A002802D01849BB
:104C5000086A804709201549087011E01348007858
:104C600008280AD11248406A002802D01049486A30
:104C7000804709200D49087002E000200B490870A8
:104C800000BF0A480078002808D00948806A002838
:104C900004D00749886A80470449087003E000206F
:104CA0000249087000BF00BF10BD0000DC070020F3
:104CB000282F00207047000010B500200CF0E0FB0A
:104CC00009F0BCF809F010F909F026F900F010FD20
:104CD000F6F7BEF80220FCF75FFB002007490870DA
:104CE000FFF7BCF8FEF7E2FFFFF708F8F5F798FECC
:104CF00010200AF03FFD00F0FBFD10BDB0010020C8
:104D000010B5012408F068FC012801D1052407E052
:104D1000F7F7E2FE0349884201D2012400E00224B1
:104D2000204610BD204E000010B5062408F054FCAB
:104D3000002800D1002408F055FC012803D008F019
:104D400051FC072800D90924204610BD10B5F6F7FC
:104D50007FF80022114601200AF06CF900213C483E
:104D6000F6F772FB00203B490880002400BF00F0EA
:104D700079FF32217D200001FBF75CFE00203649DF
:104D800008700AE00022344801781046FEF78EFDD4
:104D900031480078401C304908702F48007824289A
:104DA000F0DB00202D49087009E000212B48007835
:104DB00009F054FD29480078401C2849087027480C
:104DC00000780D28F1DBFEF799FFF5F7FFFC08F0FE
:104DD00055FB23480078401C21490870084600789C
:104DE000052812D300200870FEF776FF1D480078D2
:104DF0000A2805D300201B490870FFF747F904E093
:104E000018480078401C1749087008F0EBFB01288F
:104E1000ADD908F0E7FB0728A9D200200F49087098
:104E200008E00E48007809F033FD0C480078401C7B
:104E30000A490870094800780D28F2DBF5F772FF7F
:104E400055210348F6F700FBF7F71CFE204610BD7E
:104E5000740800207A0000201301002011010020B6
:104E6000120100201401002010B5032408E000F016
:104E7000F9FE012000F000FE002801D0042400E02B
:104E8000F5E700BF204610BD10B50020314908608D
:104E900007F00CFF0120FCF77FFAF6F745FEF7F765
:104EA000F3FEF8F73DFE0CF02FFAF5F749FCF9F7A1
:104EB00023FCF5F737FF08F0F1FAF8F7B7FE022107
:104EC0002548F6F709FD02212348F6F705FD0221E2
:104ED0002148F6F701FDF8F71FFFF6F799FAF6F704
:104EE0008DFA55211D48F6F7AFFAF9F73DFCF9F7B1
:104EF000D9FDF8F72BFAFFF79FFBFDF7E9FDFFF768
:104F000097FCFFF717FDFEF781FEFEF7A7FF00F005
:104F100091F8E12040020BF039FEF6F775F8FBF747
:104F2000D5F8F9F7DBFD0E4A0E4901200AF00CF81E
:104F300000221146012009F04BFF09F087FE09F01D
:104F40003DFF0221012000F0DFFCFAF753FD07F0DE
:104F50003DFE10BD4C0000206808002074080020B1
:104F60000090D003EC04000010B50720400200F0D0
:104F700083FD012812D114480068C82808D30020F6
:104F80001249086000210720400200F091FD19E05D
:104F90000D480068401C0C49086013E00B4800688D
:104FA000022805D809480068401C0849086009E043
:104FB00000200649086004490860012107204002DA
:104FC00000F076FD10BD0000B4000020B800002005
:104FD00070B506460D4614460E4806600E4805603C
:104FE0000E49206808600E49606808600D49A06895
:104FF00008600D49206908600C49E06808600C49A8
:105000006069086005480068002802D0034800680D
:10501000804770BDA8000020B00000209000002054
:1050200094000020980000209C000020A000002098
:10503000A400002000B587B00C4801900C480290F5
:105040000C4803900020049005900B480690002027
:105050000A49086048600A490860486001AA0121BD
:10506000C9020848FFF7B4FF07B000BD895001002E
:1050700035540100BD530100E15201007C120020B3
:10508000740A00208417002001207047F3B5C3B0D4
:105090000446449E0020009057E002E0641C761E07
:1050A00000BF022E05D32078EB28F7D16078902836
:1050B000F4D1072E00D24AE0A778FD1CB54200D9F2
:1050C00045E0A81E205C0002691E615C0843429016
:1050D000042D38D9291FA01C0CF030F942998842C0
:1050E00026D11D480068002804D0B91EE01C1A4AC9
:1050F0001268904719480068002824D0E178684673
:105100000171207981116846417120798106890EEB
:1051100068468171381FC1B26846C171C279611D8C
:1051200002A8F3F7AAF801A80C49096888470AE021
:105130000020009002E00098401C00900098A842D7
:10514000F9D3002000906419761B072EA5D200BF6A
:105150004498801B45B0F0BD9C000020A4000020B6
:10516000F7B5C0B0154600260027E81DFF21013124
:10517000884202DD002043B0F0BDEB21684601709B
:1051800090214170281DC1B2684681700021C17014
:105190004098C1B2684601710524002605E0419897
:1051A000805D69460855641C761CAE42F7DBA11E83
:1051B00000A802300CF0C2F80746381269460855BC
:1051C000641C0F55641C06480068002805D0214661
:1051D0006846034A12689047CDE70020CBE70000FD
:1051E0009400002070B50024002500261B4840686C
:1051F0001A490968884200D170BD184840681749AB
:105200000968884205D91548406814490968451A53
:1052100007E01248006811494968401A01218902D3
:105220000D1AFF2D01D9FF2600E02E4600240DE0C7
:105230000A4801680830405C094908550748008859
:10524000401C8005800D05490860641CB442EFD302
:10525000B1B203480BF0F6FC00BFCDE77C12002092
:105260008416002070B500251A480068002830D048
:10527000194A1288FF230133991A184A1268164BEB
:105280001B88D018134A126890470546002D20D07D
:1052900011480088401910490880084601880F48C5
:1052A0000068FFF7F3FE0446002C0DDD0A48008875
:1052B000844209DA08480088021B0848006801197E
:1052C00006480068F2F7D9FF03480088001B02492E
:1052D000088070BD98000020AC000020A8000020CD
:1052E00038B504460020009030490860A0781028A6
:1052F0000CD120792E49087008460078012853D136
:10530000002211462020FFF72BFF4DE0A078122845
:1053100003D120792649087246E0A078052803D1F8
:105320002079234988723FE0A07802281DD1207996
:105330001F4948720846407A012806D10090012290
:1053400069460420FFF70CFF2EE01948407A022836
:105350002AD100BFBFF34F8F16481749C860BFF36B
:105360004F8F00BF00BF00BFFDE7A07801281BD111
:105370002079332803D101200D49487005E02079B8
:10538000352802D100200A494870607908498870A0
:10539000607A0006217A09040843E179090208438A
:1053A000A17908430249486038BD0000B4000020DC
:1053B000680A00200400FA0500ED00E070B503461D
:1053C0000022002400251A484068194E3668B04271
:1053D00001D1002070BD16484068154E3668B042B5
:1053E00005D913484068124E3668841B07E0104800
:1053F00000680F4E7668801B0126F602341AA1421F
:1054000001D9254600E00D4600220CE00848066858
:105410000830805D985406480088401C4005400DC7
:10542000034E3060521CAA42F0D32846D2E7000057
:10543000740A002070B50346002200241548406815
:10544000144D2D68A84208D312484068114D2D68AC
:10545000401B0125AD022C1A04E00E4800680D4DDA
:105460006D68441BA14201D9012070BD00220CE0EF
:105470009D5C084846680830855508388088401C7F
:105480008005800D034D6860521C8A42F0D30020D5
:10549000EBE700007C12002010B50248FFF794FAF9
:1054A00010BD00001C1F02000021014A1175704749
:1054B00040600040014600BFF020084000110A2370
:1054C000584302460807000F8018C0B270470146D3
:1054D000002204E0501CC2B208460A38C1B20A29B0
:1054E000F8DA1007000E08437047000010B50446B4
:1054F00001218020F6F732F8607A012805D1424870
:10550000C078102108434049C870607AA22805D1AC
:105510003E48007F802108433C490877607A3B4938
:10552000087700203A4948770846407F21780843A9
:1055300037494877E07B002805D00846407F202186
:105540000843334948773248407FC008C000A17AF9
:1055500008432F4948770846807FF72108402C49A7
:105560008877E078FFF7B3FF29498874A078FFF7C0
:10557000AEFF2749C8746078FFF7A9FF2449087572
:105580002078002805D10846007D2179084320496C
:105590000875E079FFF79BFF1D4988756079FFF773
:1055A00096FF1B494875A079FFF791FF1849C87508
:1055B000207AFFF78CFF164908760846807F400660
:1055C000400E8877E07A002806D00846807F402188
:1055D00008430F49887703E00D48807F0C4988779E
:1055E000A07BFFF774FF0A498876607BFFF76FFFA7
:1055F0000749C876207B08770846807F10218843BA
:105600000349887710BD0000200402406004044074
:10561000404F044010B504461B48807F01210843D9
:10562000194988772078FFF752FF17490875607885
:10563000FFF74DFF1449C874A078FFF748FF1249DF
:10564000887420780C2806DD0846407F082108432E
:105650000D49487709E00C48407F0B4948770846D8
:10566000007DE1780843084908750748807F4008B5
:1056700040000549887700BF0348807F0221084029
:105680000028F9D110BD0000404F044010B50020A3
:105690001449087616200BF035FB002112480176DC
:1056A0001248407F80210843104948770846807F90
:1056B000012108430D49887700BF0C48807F0221F3
:1056C00008400028F9D00948807F40084000074979
:1056D000887700BF0548807F022108400028F9D163
:1056E00010BD00004060004040610040404F044059
:1056F00010B500200749087000212020F5F72EFF83
:1057000001210548017500200449087515200BF09A
:10571000E1FA10BD0050044040610040406000408C
:1057200070B504460D46002C14D0002D12D0042D67
:1057300010D800F013F800280CD1002608E0064924
:10574000885D22460121F3F717FEA41C701CC6B227
:10575000AE42F4DB70BD0000981E02000020054937
:10576000897DC907C90F002901D0012000E0002070
:10577000704700000050044030B585B005460C4627
:10578000002003900490009001900290072C0BDC05
:105790000120A04081B2684681810121C17303A923
:1057A0000220FAF7DBFD3EE0082C01D0092C0BD1DA
:1057B0000120A04081B2684681810121C17303A903
:1057C0000120FAF7CBFD2EE00A2C03D00B2C01D0E0
:1057D0000D2C0BD10120A04081B2684681810121AE
:1057E000C17303A90020FAF7B9FD1CE00C2C01D00D
:1057F0000F2C0BD10120A04081B26846818101218C
:10580000C17303A90E20FAF7A9FD0CE00E2C0AD1F2
:105810000120A04081B2684681810121C17303A9A2
:105820000C20FAF79BFD002168460170C1704170A1
:105830000121817000210171C1720D218172FF214E
:10584000017200214172F3F7F7FD03491520FDF7BE
:1058500009F805B030BD0000A954010010B50020C2
:105860001049087515200BF035FA00210E48017516
:105870001520002809DB00BF00BFC206D20E01219F
:1058800091400A4A116000BF00BF00BF08488079FC
:105890008011032805D00648007880210843044978
:1058A000087010BD406000404061004000E100E031
:1058B0000050044010B5F3F7B9FE10BD10B5012338
:1058C0001A4600211846F5F7FDFD01221146104643
:1058D000F5F764FEF2F7F6FB03480BF007FD02480C
:1058E0000249086010BD00000090D003600700204E
:1058F00000BF04480069042108430249086130BF21
:1059000000BF704700ED00E0F3B585B00546002408
:1059100000270026002003900490EEB22804070E12
:105920000F2F54DA082E52DA002009E00C214143EF
:10593000284A515AA94201D1044603E0411CC8B289
:105940001728F3D300BF0120B04086B20C2060437B
:1059500020494018C3780C20604340188278F8B280
:1059600031460190FAF79EFD6846868101218173D8
:105970000021C17302214174F8B203A9FAF7EEFCC9
:105980000C216143134A8918C888FBF72BFE0C20B1
:10599000604310494018C1886846018169460698ED
:1059A000887202A8FBF738FD0C226243094BD2181B
:1059B00091680C226243D21804201056FCF752FF63
:1059C0000C216143034A8918C888FBF78FFD07B093
:1059D000F0BD0000B4200200FEB505460C460020D4
:1059E000C0430290EFB22804060E0F2E42DA082FB1
:1059F00040DA0120B8406946088080202040002815
:105A000016D101208870A007800F022801D14871AB
:105A100009E0A007800F012802D16946487102E021
:105A2000002069464871F0B26946FAF797FC1FE01A
:105A30000020694688700E202040002800D000BF5A
:105A400010202040002802D16946087102E00120A0
:105A500069460871E007C00F002802D169468871C5
:105A600002E0012069468871F0B26946FAF776FCD7
:105A7000002002900298FEBD30B50146CAB20C0467
:105A8000230E00200F2B0FDA082A0DDA0124944090
:105A9000A2B2064C03252D026419E45C1440002CCC
:105AA00001D0012000E0002030BD000000000440D3
:105AB000F8B504460F460020C0430090E6B220042B
:105AC000050E0F2D11DA082E0FDA0120B04086B234
:105AD000002F04D1E8B23146FAF73CFD03E0E8B20A
:105AE0003146FAF747FD002000900098F8BD00000D
:105AF0001649897F01221143144A917700BF134947
:105B0000897F022211400029F9D01049897C8170D7
:105B10000E49C97C41700D49097D01700B498A7D90
:105B20008271497D01710949CA7D42710A7EC27143
:105B3000897F49084900054A917700BF0349897F59
:105B4000022211400029F9D170470000404F044063
:105B500003B585B0002001900290039004900021CD
:105B600068464173817E01A8C1706846417E01A8E4
:105B700081706846017E4171002101A801710821F0
:105B800068460171817D01A8C1716846C17D41727D
:105B9000417D01A881716846017D01A80172002143
:105BA00068468173C17301A881730C21417341213F
:105BB000684601740021C17401A8FFF797FC1D20FD
:105BC0000449888204491620FCF74CFE00F006F8D0
:105BD00007B000BD204F04403914020010B5FFF794
:105BE00055FD10BD70B504460D46601E0D49884236
:105BF00000D90124002C00D1012440200A4908705A
:105C0000084600786043094948610321081F0BF0EA
:105C100091F8002005498861072008610448056063
:105C200070BD0000FFFFFF008C01002000E000E0DD
:105C3000880100200020C043002809DBC206D20EE4
:105C400001219140054A1160BFF34F8FBFF36F8F61
:105C500000BF0020024908618861704780E100E0D0
:105C600000E000E010B50BF00BF810BD1A20084959
:105C700008722B2048723C2088724D20C8727F2009
:105C8000044909680860AC20034948707047000067
:105C900000040240900100200010024010B51C4892
:105CA0000078012812D11B480078642809DB022003
:105CB0001949487108710020164908701449087084
:105CC00004E014480078401C12490870134800781A
:105CD00001281CD112480078012804D10020104965
:105CE0000870104908700F48007832280ADBF7F76F
:105CF00013F800210C48F5F73BFB55210B48F5F74D
:105D0000A3FB04E007480078401C0649087010BD5A
:105D1000290700202807002018070020220700205C
:105D200024070020230700206808002074080020B2
:105D3000F8B504460D46002700200090032000031C
:105D4000204000130090102C04D0122C02D01148D7
:105D5000844217D122202840222806D127073F0F4E
:105D600039460098F4F7D8FC06461220284012283D
:105D70000ED12007000F471C39460098F4F7CCFCE1
:105D8000064605E02107090F0098F4F7C5FC064612
:105D90003046F8BD10100000F8B504460D46002648
:105DA00000270120000320400713102C04D0122CE0
:105DB00002D00F48844215D122202840222805D144
:105DC0002607360F31463846F9F7B8FF122028402B
:105DD00012280CD12007000F461C31463846F9F72F
:105DE000ADFF04E02107090F3846F9F7A7FFF8BD1A
:105DF00010100000FFB58BB01C46002007900690E5
:105E000005903848049010210B980840002801D0D4
:105E1000022707E040210B980840002801D0012705
:105E200000E00027002C04D0149804700120089092
:105E300001E010200890002548E0002C08D02546FD
:105E40006000294A115A0C98F2F780F9079006E091
:105E50006800254A115A0C98F2F778F907903E46E7
:105E600030E0711C0798F2F771F9400806900D9820
:105E7000F2F7C2FA03900D9A0699881AF2F7BCFA63
:105E800018490190F2F73DFA02900399F2F776FA79
:105E900005900598F2F7B7FA490049080391029076
:105EA0000498F2F7B0FA4900490801910090039B69
:105EB000029AF2F7BDFA03D20A9509960598049062
:105EC000701CC6B27F2ECCDD681CC5B20898854216
:105ED000B3DB14990A9808701499099848700498CB
:105EE0000FB0F0BD0000C842C82102000246412A9E
:105EF0002ED010DC212A2AD006DC102A45D0122A06
:105F00004BD0202A59D11CE0222A26D0232A2AD07D
:105F1000402A52D116E081235B01D01A9A4228D040
:105F200008DC422A1AD0432A1ED02548101800281F
:105F300043D13AE0012822D020281BD021283CD18F
:105F40001EE000BF1F4803890B43038136E000BFFA
:105F50001C4843890B43438130E000BF19488389C3
:105F60000B4383812AE000BF1648C3890B43C381DA
:105F700024E000BF144883880B4383801EE000BFE9
:105F80001148C3880B43C38018E00E4843890B4374
:105F9000438103890B43038110E00A48C3890B4303
:105FA000C38183890B43838108E00748C3880B437F
:105FB000C38083880B43838000E000BF00BF70472D
:105FC000F0EFFFFF0011044000140440F0B5054657
:105FD0000E46412D30D010DC212D2CD006DC102DAA
:105FE00051D0122D56D0202D62D11CE0222D2AD066
:105FF000232D30D0402D5BD116E081214901681A54
:106000008D4230D008DC422D1ED0432D24D02A48AA
:10601000281800284CD144E001282CD0202823D077
:10602000212845D128E000BF244F3888314600F0B0
:1060300049F804463DE000BF204F7888314600F023
:1060400041F8044635E000BF1C4FB888314600F0E7
:1060500039F804462DE000BF184FF888314600F0AB
:1060600031F8044625E000BF154F3888314600F06E
:1060700029F804461DE000BF114F7888314600F032
:1060800021F8044615E00D4F7888314600F01AF8E3
:1060900004460EE0094FF888314600F013F8044634
:1060A00007E0074F7888314600F00CF8044600E01E
:1060B00000BF00BF2046F0BDF0EFFFFF001104401D
:1060C000001404400246002013460B40002B01D070
:1060D000012000E000207047FFB581B00E46174652
:1060E000012F07D1F748407D00090001C01DF54987
:1060F000487505E0F348407D00090001F149487505
:10610000049801287ED10A210198F2F71FF805466C
:10611000ED48445DE007C00F002807D0E948007C47
:1061200000090001C01DE749087405E0E548007C4E
:1061300000090001E349087402202040002807D02C
:10614000E048C07BF02188437030DE49C87305E029
:10615000DC48C07BF0218843DA49C8730420204022
:10616000002807D0D748807C00090001C01DD54910
:10617000887405E0D348807C00090001D149887407
:1061800008202040002807D0CE48407CF0218843DA
:106190007030CC49487405E0CA48407CF0218843FF
:1061A000C849487410202040002807D0C548407CCA
:1061B00000090001C01DC349487405E0C148407C86
:1061C00000090001BF49487420202040002807D062
:1061D000BC48007CF02188437030BA49087405E05F
:1061E000B848007CF0218843B6490874402020401C
:1061F000002808D0B348807CF02188437030B14932
:10620000887406E08BE0AF48807CF0218843AD497C
:1062100088740A210198F1F799FF0D46AA48445D58
:10622000E007C00F002807D0A648807BF0218843F4
:106230007030A449887305E0A248807BF021884330
:10624000A049887302202040002807D09D48807B09
:1062500000090001C01D9B49887305E09948807BB7
:10626000000900019749887304202040002807D0C6
:106270009448007DF021884370309249087505E00C
:106280009048007DF02188438E4908750820204001
:10629000002807D08B48007D00090001C01D8949F6
:1062A000087505E08748007D0009000185490875EB
:1062B00010202040002807D08248C07CF02188436D
:1062C00070308049C87405E07E48C07CF021884366
:1062D0007C49C87420202040002807D07948C07B22
:1062E00000090001C01D7749C87305E07548C07BEF
:1062F000000900017349C87340202040002807D0DE
:106300007048C07C00090001C01D6E49C87454E08B
:106310006C48C07C000900016A49C8744DE06948B6
:10632000007C00090001674908740846C07BF02121
:1063300088436449C8730846807C0009000188745A
:106340000846407CF02188435E4948740846407CFA
:106350000009000148740846007CF021884359492F
:1063600008740846807CF0218843564988740846A2
:10637000807BF0218843534988730846807B00095D
:10638000000188730846007DF02188434D49087557
:106390000846007D0009000108750846C07CF02110
:1063A00088434849C8740846C07B00090001C87387
:1063B0000846C07C00090001C8740A9801287DD1F4
:1063C0000A213046F1F7C2FE05463F48445DE0072A
:1063D000C00F002807D03B48407B00090001C01DCA
:1063E0003849487305E03748407B000900013549CA
:1063F000487302202040002807D03248007BF0215B
:10640000884370302F49087305E02E48007BF02147
:1064100088432C49087304202040002807D02948CD
:10642000807DF021884370302649887505E0254835
:10643000807DF0218843234988750820204000286A
:1064400007D02048807D00090001C01D1D498875C6
:1064500005E01C48807D000900011A49887510205C
:106460002040002807D01748407DF0218843703035
:106470001449487505E01348407DF02188431149CF
:10648000487520202040002807D00E48407BF0218E
:10649000884370300B49487305E00A48407BF0217F
:1064A0008843084948734020204000280ED0054802
:1064B000C07D00090001C01D024900E092E0C875DE
:1064C0000AE0000064260020EC1B02006D48C07D3D
:1064D000000900016B49C8750A213046F1F736FE04
:1064E0000D466948445DE007C00F002807D06548A5
:1064F000C07AF021884370306249C87205E0614873
:10650000C07AF02188435F49C872022020400028E9
:1065100007D05C48C07A00090001C01D5949C87203
:1065200005E05848C07A000900015649C8720420A5
:106530002040002807D05348407E00090001C01DBC
:106540005049487605E04F48407E000900014D491A
:10655000487608202040002807D04A48007EF021D5
:10656000884370304749087605E04648007EF021B0
:1065700088434449087610202040002807D041482D
:10658000007E00090001C01D3E49087605E03D4837
:10659000007E000900013B490876202020400028A9
:1065A00007D03848007B00090001C01D3549087339
:1065B00005E03448007B000900013249087340209F
:1065C0002040002807D02F48C07DF021884370303C
:1065D0002C49C87554E02B48C07DF02188432949D7
:1065E000C8754DE02748407B0009000125494873E4
:1065F0000846007BF0218843224908730846807DC5
:10660000F02188431F4988750846807D00090001F4
:1066100088750846407DF02188431A494875084628
:10662000407BF0218843174948730846C07D000924
:106630000001C8750846C07AF02188431149C87224
:106640000846C07A00090001C8720846407E000969
:10665000000148760846007EF02188430949087603
:106660000846007E0009000108760846007B000904
:10667000000108730846C07DF02188430149C875B0
:1066800005B0F0BD64260020EC1B0200FFB581B010
:106690000E461746019801287ED10498002826D17D
:1066A000FA480078012822D0F6F71CFAF849884207
:1066B0001DD3FAF7DDFC00280DD0F648807DF021CF
:1066C00088437030F34988750846C07C0009000192
:1066D000C01DC87418E0EF48807DF0218843ED4963
:1066E00088750846C07C00090001C8740CE0E948C0
:1066F000807DF02188437030E64988750846C07C6B
:1067000000090001C01DC874E248C07CF021884324
:106710007030E049C8740846007EF021884370302C
:10672000DC4908760846807D00090001401C887518
:106730000846407DF02188431030D6494875084608
:10674000407D00090001401C48750846007DF0218D
:1067500088431030CF4908750846007D00090001C4
:10676000401C087533000AF0A7FA062E261E140CEA
:10677000042FC848007D00090001C01DC5490875E7
:1067800000BFC448007DF02188437030C1490875BE
:1067900000BFC048407D00E0ADE100090001C01D20
:1067A000BC49487500BFBB48407DF021884370302C
:1067B000B849487500BFB748807D00090001C01D79
:1067C000B449887500BF00E000BF00BF04980028EE
:1067D0005ED1AE48007801285AD0F6F783F9AC496B
:1067E000884255D3AB48C07FF0218843A949C87778
:1067F0000846807F0009000188770846407FF02125
:106800008843A44948770846007FF0218843A1497E
:1068100008770846C07DF02188439E49C875084620
:10682000C07F00090001C8770846807FF0218843B7
:10683000984988770846407F00090001C01D4877C5
:106840000846807EF0218843924988760846807EFB
:106850000009000188760846407E0009000148765C
:106860000846007E0009000108760846007F0009FE
:10687000000108770846C07EF02188438549C87624
:106880000846407EF0218843703082494876B8E15E
:1068900064213846F1F75AFC0546012D07D17D48A1
:1068A000C07FF021884370307A49C87705E0794885
:1068B000C07FF02188437749C8770A213846F1F72D
:1068C00045FC0A210090F1F741FC0D46642F02D3EC
:1068D0007148445D01E07148445DE007C00F002845
:1068E00007D06C48807F00090001C01D6949887786
:1068F00005E06848807F000900016649887702202A
:106900002040002807D06348407FF0218843703042
:106910006049487705E05F48407FF02188435D4942
:10692000487704202040002807D05A48007FF021F3
:10693000884370305749087705E05648007FF021BA
:1069400088435449087708202040002807D0514840
:10695000C07DF021884370304E49C87505E04D4830
:10696000C07DF02188434B49C87510202040002885
:1069700007D04848C07F00090001C01D4549C877BD
:1069800005E04448C07F000900014249C877202043
:106990002040002807D03F48807FF0218843703096
:1069A0003C49887705E03B48807FF021884339499E
:1069B000887740202040002807D03648407F0009D3
:1069C0000001C01D3349487705E03248407F000987
:1069D0000001304948770A213846F1F7B7FB0D46E8
:1069E0002D48445DE007C00F002807D02948807E6D
:1069F000F021884370302749887605E02548807E5D
:106A0000F02188432349887602202040002807D0BF
:106A10002048807E00090001C01D1E49887605E0DF
:106A20001C48807E000900011A4988760420204015
:106A3000002807D01748407E00090001C01D1549F5
:106A4000487605E01348407E000900011149487668
:106A500008202040002807D00E48007E00090001D1
:106A6000C01D0C49087605E00A48007E00090001B7
:106A70000849087610202040002811D00548007FE2
:106A800000090001C01D034908770FE0F90000204C
:106A9000B80B000038270020EC1B0200FF1B02008F
:106AA0005948007F000900015749087720202040FD
:106AB000002807D05448C07EF021884370305249E6
:106AC000C87605E05048C07EF02188434E49C8761C
:106AD00040202040002807D04B48407EF0218843CA
:106AE0007030494948768CE04748407EF021884321
:106AF0004549487685E04448807D000900014249C7
:106B000088750846407DF02188433F49487508460E
:106B1000407D0009000148750846007DF02188434A
:106B2000394908750846007D0009000108750846C6
:106B3000C07C00090001C8740846807DF0218843AC
:106B4000314988750846C07CF02188432E49C874B5
:106B50000846007EF02188432B4908760846C07F0E
:106B6000F02188432849C8770846807F0009000142
:106B700088770846407FF0218843234948770846B4
:106B8000007FF0218843204908770846C07DF02126
:106B900088431D49C8750846C07F00090001C877B1
:106BA0000846807FF0218843174988770846407F50
:106BB0000009000148770846807EF0218843124989
:106BC00088760846807E0009000188760846407E67
:106BD0000009000148760846007E00090001087699
:106BE0000846007F0009000108770846C07EF021B2
:106BF00088430549C8760846407EF021884302490B
:106C0000487605B0F0BD00003827002010B50146D9
:106C1000002200200A0EFE4B985CC307DB0F002BFE
:106C200007D0FC4BDB7FF024A3437033F94CE377B0
:106C300005E0F84BDB7FF024A343F64CE377022317
:106C40000340002B07D0F34BDB7F1B091B01DB1D2F
:106C5000F04CE37705E0EF4BDB7F1B091B01ED4CAC
:106C6000E37704230340002B07D0EA4B9B7F1B09EB
:106C70001B01DB1DE74CA37705E0E64B9B7F1B095F
:106C80001B01E44CA37708230340002B09D0E14B00
:106C900020335B781B091B01DB1DDE4C2034637045
:106CA00007E0DC4B20335B781B091B01D94C2034F7
:106CB000637010230340002B09D0D64B20331B7880
:106CC000F024A3437033D34C2034237007E0D14B1E
:106CD00020331B78F024A343CE4C20342370202390
:106CE0000340002B09D0CB4B20331B781B091B0121
:106CF000DB1DC84C2034237007E0C64B20331B78C3
:106D00001B091B01C34C2034237040230340002B7C
:106D100007D0C04B9B7FF024A3437033BD4CA377B7
:106D200005E0BC4B9B7FF024A343BA4CA377FF2321
:106D30001B040B401A0CB64B985CC307DB0F002BEF
:106D400007D0B44B1B7F1B091B01DB1DB14C237704
:106D500005E0B04B1B7F1B091B01AE4C23770223C0
:106D60000340002B07D0AB4BDB7EF024A3437033F2
:106D7000A84CE37605E0A74BDB7EF024A343A54CAB
:106D8000E37604230340002B07D0A24B9B7EF02424
:106D9000A34370339F4CA37605E09E4B9B7EF0246B
:106DA000A3439C4CA37608230340002B07D0994BA8
:106DB0005B7FF024A3437033964C637705E0954BDB
:106DC0005B7FF024A343934C637710230340002B95
:106DD00007D0904B5B7F1B091B01DB1D8D4C63773C
:106DE00005E08C4B5B7F1B091B018A4C63772023DA
:106DF0000340002B07D0874B1B7FF024A343703345
:106E0000844C237705E0834B1B7FF024A343814C04
:106E1000237740230340002B07D07E4BDB7E1B09EA
:106E20001B01DB1D7B4CE37605E07A4BDB7E1B0907
:106E30001B01784CE376FF231B020B401A0A744BAC
:106E4000985CC307DB0F002B07D0724B1B7EF0242E
:106E5000A34370336F4C237605E06E4B1B7EF0240A
:106E6000A3436C4C237602230340002B07D0694BCD
:106E70001B7E1B091B01DB1D664C237605E0654B61
:106E80001B7E1B091B01634C237604230340002B4C
:106E900007D0604BDB7D1B091B01DB1D5D4CE375DF
:106EA00005E05C4BDB7D1B091B015A4CE375082395
:106EB0000340002B07D0574B9B7E1B091B01DB1D9A
:106EC000544CA37605E0534B9B7E1B091B01514C90
:106ED000A37610230340002B07D04E4B5B7EF0249B
:106EE000A34370334B4C637605E04A4B5B7EF02442
:106EF000A343484C637620230340002B07D0454B27
:106F00005B7E1B091B01DB1D424C637605E0414B98
:106F10005B7E1B091B013F4C637640230340002B23
:106F200007D03C4BDB7DF024A3437033394CE37531
:106F300005E0384BDB7DF024A343364CE375CAB241
:106F4000334B985CC307DB0F002B07D0314B1B7D05
:106F5000F024A34370332F4C237505E02D4B1B7D8C
:106F6000F024A3432B4C237502230340002B07D0AE
:106F7000284B1B7D1B091B01DB1D264C237505E0DF
:106F8000244B1B7D1B091B01224C2375042303404A
:106F9000002B07D01F4BDB7C1B091B01DB1D1D4C8D
:106FA000E37405E01B4BDB7C1B091B01194CE374EC
:106FB00008230340002B07D0164B9B7CF024A343EF
:106FC0007033144CA37405E0124B9B7CF024A34354
:106FD000104CA37410230340002B07D00D4B5B7D96
:106FE000F024A34370330B4C637505E0094B5B7DC4
:106FF000F024A343074C637520230340002B0BD0E0
:10700000044B5B7D1B091B01DB1D024C637509E012
:10701000EC1B0200182700200C4B5B7D1B091B0199
:107020000A4C637540230340002B07D0074BDB7CE1
:10703000F024A3437033054CE37405E0034BDB7C81
:10704000F024A343014CE37410BD00001827002076
:1070500000B501287ED1FE4AD278F0239A437032DF
:10706000FB4BDA701A46127912091201D21D1A71FD
:107070001A461279F0239A437032F54B1A711A4668
:10708000527912091201D21D5A711A465279F0230F
:107090009A437032EE4B5A711A46D2791209120194
:1070A000D21DDA711A46D279F0239A437032E84B36
:1070B000DA711A46527A12091201D21D5A721A4610
:1070C000527AF0239A437032E14B5A721A46927AFE
:1070D000F0239A437032DE4B9A721A469278F0236C
:1070E0009A437032DA4B9A701A46D27A1209120118
:1070F000D21DDA721A46527812091201D21D5A7044
:107100001A46D27AF0239A437032D14BDA721A4679
:10711000203AD27FF0239A437032CD4B203BDA776E
:10712000CB4A127B12091201D21D20331A731A4660
:10713000203A927F12091201D21D203B9A77C44A4D
:10714000127BF0239A437032C14B1A731A46203ACD
:10715000127F00E0F2E1F0239A437032BC4B203BF7
:107160001A77BB4A527B12091201D21D20335A737F
:107170001A46203AD27E12091201D21D203BDA763D
:10718000B44AD278F0239A437032B24BDA701A467E
:10719000127B12091201D21D1A731A4612791209B2
:1071A0001201D21D1A711A46927AF0239A43703254
:1071B000A84B9A721A461279F0239A437032A54B63
:1071C0001A711A46527912091201D21D5A711A46C1
:1071D000927912091201D21D9A711A46127A120975
:1071E0001201D21D1A721A46127AF0239A43703293
:1071F000984B1A721A46527A12091201D21D5A720B
:10720000934A927912091201521C914B9A711A46B3
:107210009279F0239A4310328D4B9A711A46127A62
:1072200012091201521C1A721A46127AF0239A435A
:107230001032874B1A721A46927A12091201521CA6
:107240009A721A46D27812091201521CDA701A4642
:10725000927812091201521C9A701A465278F02341
:107260009A4310327A4B5A701A461278F0239A4396
:107270001032774B1A701A46127812091201521CFA
:107280001A701A46203AD27F12091201521C203B72
:10729000DA771A46927FF0239A4310326C4B203BE8
:1072A0009A771A46527FF0239A431032684B203B5C
:1072B0005A771A46527F12091201521C5A771A46FF
:1072C000127F12091201521C1A771A46D27EF0233D
:1072D0009A4310325E4B203BDA761A46927EF023B8
:1072E0009A4310325A4B203B9A765A4A127BF0232B
:1072F0009A431032574B1A731A46D27AF0239A43A4
:107300001032544BDA721A46D27A12091201521C08
:10731000DA721A46927A12091201521C9A721A46AD
:10732000527AF0239A4310324A4B5A721A465279D3
:10733000F0239A431032474B5A711A46D279F02300
:107340009A431032434BDA710B0009F0B5FC19F384
:10735000E9DFD5CBC1B7ADA3998F87786E645A505A
:10736000463E362E261E160EF5003A4AD279F023F6
:107370009A437032374BDA7100BF364A5279F023A4
:107380009A437032334B5A7100BF324A527AF0231B
:107390009A4370322F4B5A7200BF2E4A927A1209CA
:1073A0001201D21D2B4B9A7200BF2A4AD27A1209BF
:1073B0001201D21D274BDA7200BF264AD27AF0237F
:1073C0009A437032234BDA7200BF224A127BF023B9
:1073D0009A4370321F4B1A7300BF1D4A203A927EA7
:1073E000F0239A4370321A4B203B9A7600BF184A1A
:1073F000203AD27EF0239A437032154B203BDA7646
:1074000000BF134A203A127F12091201D21D104BFD
:10741000203B1A7700BF0E4A203A527F1209120110
:10742000D21D0B4B203B5A7700BF094A203A527FAE
:10743000F0239A437032064B203B5A7700BF044A30
:10744000203A927FF0239A437032014B203B03E0B5
:1074500084260020582700209A7700BFDC4AD27F7C
:1074600012091201D21DDA4BDA7700BFD84A203256
:10747000127812091201D21DD54B20331A7000BFA9
:10748000D34A20321278F0239A437032D04B203303
:107490001A7000BFCE4A20325278F0239A437032DD
:1074A000CB4B20335A7000BFC94A20329278120960
:1074B0001201D21DC64B20339A7000BFC44A20323D
:1074C000D27812091201D21DC14B2033DA7000BFED
:1074D000BF4A2032927A12091201D21DBC4B2033CE
:1074E0009A7200BFBA4A2032127AF0239A4370325D
:1074F000B74B20331A7200BFB54A2032127A1209F4
:107500001201D21DB24B20331A7200BFB04A203292
:107510009279F0239A437032AD4B20339A7100BFB9
:10752000AB4A2032927912091201D21DA84B2033A6
:107530009A7100BF01E0FFE700BF47E1A44A203293
:10754000D278F0239A43A24B2033DA701A4612798C
:10755000120912011A711A461279F0239A439C4BB0
:1075600020331A711A465279120912015A711A46B9
:107570005279F0239A43964B20335A711A46D279A6
:1075800012091201DA711A46D279F0239A43904B0C
:107590002033DA711A46527A120912015A721A46C7
:1075A000527AF0239A438A4B20335A721A46927ABF
:1075B000F0239A43864B20339A721A469278F0232E
:1075C0009A43834B20339A701A46D27A12091201D9
:1075D000DA721A465278120912015A701A46D27A91
:1075E000F0239A437A4B2033DA72794AD27FF02320
:1075F0009A43774BDA771A462032127B120912012E
:1076000020331A73724A927F12091201203B9A7733
:107610001A462032127BF0239A436D4B20331A73A3
:107620006B4A127FF0239A43694B1A771A4620322D
:10763000527B1209120120335A73654AD27E120915
:107640001201203BDA76634AD278F0239A43614BE9
:10765000DA701A46127B120912011A731A4612794D
:10766000120912011A711A46927AF0239A43594B61
:107670009A721A461279F0239A43564B1A711A4697
:107680005279120912015A711A469279120912019D
:107690009A711A46127A120912011A721A46127A4D
:1076A000F0239A434B4B1A721A46527A120912016E
:1076B0005A72474A2032927912091201444B203300
:1076C0009A711A469279F0239A43414B20339A716A
:1076D0001A46127A120912011A721A46127AF02305
:1076E0009A433B4B20331A721A46927A12091201BE
:1076F0009A721A46D27812091201DA701A469278F2
:10770000120912019A701A465278F0239A43304BAC
:1077100020335A701A461278F0239A432C4B2033A8
:107720001A701A461278120912011A70284AD27F6A
:1077300012091201203BDA771A46927FF0239A430E
:10774000234B9A771A46527FF0239A43204B5A775D
:107750001A46527F120912015A771A46127F1209ED
:1077600012011A771A46D27EF0239A43184BDA7622
:107770001A46927EF0239A43154B9A76154A127B4D
:10778000F0239A43134B1A731A46D27AF0239A4382
:10779000104BDA721A46D27A12091201DA721A46BC
:1077A000927A120912019A721A46527AF0239A4377
:1077B000084B5A721A465279F0239A43054B5A7174
:1077C0001A46D279F0239A43024BDA7100BD0000C9
:1077D0006426002058270020F7B582B006461746D9
:1077E000002500200190002E7ED1F9F743FB0528EB
:1077F0005FD1F9F73DFC00280DD0FA484079F0211F
:1078000088437030F74948710846807800090001C4
:10781000C01D88700AE0F3484079F0218843F1499F
:10782000487108468078000900018870ED48C079E9
:1078300000090001EB49C871084680790009000180
:107840008871084640790009000148710846007AAD
:10785000F0218843E34908720846007A00090001D4
:1078600008720846C079F0218843DE49C87108468D
:10787000C07800090001C87008468078F02188436C
:10788000D849887008464078F0218843D549487027
:107890000846407800090001487008460079000950
:1078A000000108710846C078F0218843CD49C870AE
:1078B00029E2CC484079F02188437030C9494871A9
:1078C0000846807800090001C01D88700846C0790C
:1078D00000090001C871084680790009000188711B
:1078E00008464079000900E034E00001487108468C
:1078F000007AF0218843BB4908720846007A0009E3
:10790000000108720846C079F0218843B549C87162
:107910000846C07800090001C87008468078F02148
:107920008843B049887008464078F0218843AD49C3
:107930004870084640780009000148700846007900
:107940000009000108710846C078F0218843A54964
:10795000C870ADE7012E5FD1F9F78AFB00280DD082
:10796000A0484079F021884370309E49487108460C
:10797000807800090001C01D88700AE099484079AC
:10798000F021884397494871084680780009000132
:1079900088709448C079000900019249C87108466E
:1079A00080790009000188710846407900090001CA
:1079B00048710846007AF02188438A4908720846CF
:1079C000007A0009000108720846C079F021884356
:1079D0008449C8710846C07800090001C87008468B
:1079E0008078F02188437F49887008464078F021EC
:1079F00088437C4948700846407800090001487077
:107A0000084600790009000108710846C078F02195
:107A100088437449C870EAE3022E7DD1F9F72AFA47
:107A200005287AD1F9F724FB002877D0012F76D1E9
:107A30000A210398F0F78AFB0546F9F739FA00287E
:107A400002D16948445D01E06848445DE007C00F29
:107A5000002807D06348C07900090001C01D6149B2
:107A6000C87105E05F48C079000900015D49C8712F
:107A700002202040002807D05A48807900090001E0
:107A8000C01D5849887105E05648807900090001F9
:107A90005449887104202040002807D0514840797B
:107AA00000090001C01D4F49487105E04D4840796B
:107AB000000900014B49487108202040002807D0E8
:107AC0004848007AF021884370304649087205E042
:107AD0004448007AF021884342490872102020402F
:107AE000002807D03F48007A00090001C01D3D4929
:107AF000087205E03B48007A000900013949087224
:107B00002020204000280BD03648C079F02188433F
:107B100070303449C87109E0AEE242E1F4E0A4E01B
:107B20003048C079F02188432E49C8714020204058
:107B3000002807D02B484079F0218843703029492C
:107B4000487105E027484079F0218843254948716C
:107B50000A210398F0F7FAFA0D462348445DE0073E
:107B6000C00F002807D01F48C07800090001C01DC1
:107B70001C49C87005E01B48C0780009000119497C
:107B8000C87002202040002807D016488078F021D5
:107B9000884370301349887005E012488078F021DE
:107BA00088431049887004202040002807D00D48E1
:107BB0004078F021884370300A49487005E0094850
:107BC0004078F02188430749487008202040002869
:107BD0000ED00448407800090001C01D01494870DA
:107BE0000CE00000A4260020EC1B0200FF1B02009A
:107BF000FE48407800090001FC49487010202040F0
:107C0000002807D0F948007900090001C01DF74994
:107C1000087105E0F548007900090001F349087191
:107C200020202040002807D0F048C078F021884369
:107C30007030EE49C87005E0EC48C078F021884308
:107C4000EA49C87040202040002807D0E7488078E3
:107C500000090001C01DE5498870C8E2E34880784A
:107C600000090001E1498870C1E2E0484079F02153
:107C700088437030DD49487108468078000900016A
:107C8000C01D88700846C07900090001C871084607
:107C900080790009000188710846407900090001D7
:107CA00048710846007AF0218843D0490872084696
:107CB000007A0009000108720846C079F021884363
:107CC000CA49C8710846C07800090001C870084652
:107CD0008078F0218843C549887008464078F021B3
:107CE0008843C2494870084640780009000148703E
:107CF000084600790009000108710846C078F021A3
:107D00008843BA49C87072E2B8484079F021884384
:107D1000B649487108468078000900018870084615
:107D2000C07900090001C871084680790009000186
:107D30008871084640790009000148710846007AB8
:107D4000F0218843A94908720846007A0009000119
:107D500008720846C079F0218843A449C8710846D2
:107D6000C07800090001C87008468078F021884377
:107D70009E49887008464078F02188439B494870A6
:107D8000084640780009000148700846007900095B
:107D9000000108710846C078F02188439349C870F3
:107DA00025E2012F73D10A210398F0F7CFF9054698
:107DB000F9F77EF8002802D18D48445D01E08D4836
:107DC000445DE007C00F002807D08848C07900094B
:107DD0000001C01D8549C87105E08448C0790009CB
:107DE00000018249C87102202040002807D07F4846
:107DF000807900090001C01D7C49887105E07B483D
:107E00008079000900017949887104202040002808
:107E100007D07648407900090001C01D73494871B8
:107E200005E0724840790009000170494871082056
:107E30002040002807D06D48007AF0218843703038
:107E40006A49087205E06948007AF0218843674969
:107E5000087210202040002807D06448007A0009EA
:107E60000001C01D6149087205E06048007A000900
:107E700000015E49087220202040002808D05B489D
:107E8000C079F021884370305849C87106E09DE000
:107E90005648C079F02188435449C8714020204099
:107EA000002807D051484079F021884370304F496D
:107EB000487105E04D484079F02188434B494871AD
:107EC0000A210398F0F742F90D464948445DE0075E
:107ED000C00F002807D04548C07800090001C01D28
:107EE0004249C87005E04148C078000900013F4997
:107EF000C87002202040002807D03C488078F0213C
:107F0000884370303949887005E038488078F0211E
:107F100088433649887004202040002807D0334821
:107F20004078F021884370303049487005E02F4890
:107F30004078F02188432D494870082020400028CF
:107F400007D02A48407800090001C01D2749487021
:107F500005E02648407800090001244948701020B7
:107F60002040002807D02148007900090001C01DE9
:107F70001E49087105E01D480079000900011B49F0
:107F8000087120202040002807D01848C078F02130
:107F9000884370301549C87005E01448C078F02156
:107FA00088431249C87040202040002807D00F485D
:107FB000807800090001C01D0C49887017E10B484A
:107FC0008078000900010949887010E1074840796C
:107FD000F0218843703005494871084680780009CF
:107FE0000001C01D88700846C07905E0A426002065
:107FF000EC1B0200FF1B020000090001C8710846CB
:108000008079000900018871084640790009000163
:1080100048710846007AF02188437649087208467C
:10802000007A0009000108720846C079F0218843EF
:108030007049C8710846C07800090001C870084638
:108040008078F02188436B49887008464078F02199
:108050008843684948700846407800090001487024
:10806000084600790009000108710846C078F0212F
:1080700088436049C870BAE0032E9FD1F8F7FAFE32
:1080800005285FD1F8F7F4FF00280DD05948407952
:10809000F0218843703057494871084680780009BC
:1080A0000001C01D88700AE052484079F0218843E1
:1080B00050494871084680780009000188704D4891
:1080C000C079000900014B49C87108468079000950
:1080D000000188710846407900090001487108468E
:1080E000007AF0218843434908720846007A000963
:1080F000000108720846C079F02188433D49C871E3
:108100000846C07800090001C87008468078F02150
:1081100088433849887008464078F02188433549BB
:108120004870084640780009000148700846007908
:108130000009000108710846C078F02188432D49E4
:10814000C87054E02B480079F021884370302949E9
:10815000087108464079F0218843703025494871FC
:108160000846807800090001C01D88700846C07963
:1081700000090001C8710846807900090001887172
:10818000084640790009000148710846007AF0214C
:108190008843184908720846007A000900010872ED
:1081A0000846C079F02188431249C8710846C07852
:1081B00000090001C87008468078F02188430D4905
:1081C000887008464078F02188430A49487008467C
:1081D0004078000900014870084600790009000154
:1081E00008710846C078F02188430249C87005B07C
:1081F000F0BD0000A426002070B505460C46012DF8
:108200007ED1B148407D00090001C01DAE494875CE
:108210000846007DF02188431030AB4908750846B8
:10822000007D00090001401C08750846C07CF02153
:1082300088431030A449C8740846807CF0218843E4
:108240001030A14988740846807C00090001401C58
:108250008874F8F769FF022803D0F8F765FF012852
:108260006CD19A480078012868D0F4F73BFC984913
:10827000884263D3F8F7FCFE00282FD09248007D97
:10828000F02188437030904908750846007D000948
:108290000001C01D08750846C07CF021884370307D
:1082A0008949C8740846807CF0218843703086492B
:1082B00088740846807C00090001C01D8874084647
:1082C000407DF021884370307F4948750846407CE6
:1082D000F021884370307C494874F4E07A48007D8E
:1082E000F02188431030784908750846007D000960
:1082F0000001401C08750846C07CF021884300E05E
:10830000B4E010307049C8740846807CF02188437E
:1083100010306D4988740846807C00090001401CBB
:1083200088740846407DF0218843674948750846AF
:10833000407CF021884364494874C4E0F8F788FD24
:10834000002824D1F4F7CEFB614988421FD3F8F707
:108350008FFE00280ED05C48407DF02188437030AD
:10836000594948750846407CF02188437030564989
:1083700048741AE05448407DF021884352494875BA
:108380000846407CF02188434F4948740DE04E4830
:10839000407DF021884370304B4948750846407C49
:1083A000F0218843703048494874F8F751FD01289E
:1083B0002AD146480078012826D0F4F793FB444997
:1083C000884221D34048407DF021884370303E49A7
:1083D00048750846407CF021884370303A4948741B
:1083E000F8F746FE002807D03748007DF021884383
:1083F00070303549087566E03348007DF0218843C8
:108400001030314908755EE0230008F055FC062C59
:10841000241C140C042D2C48807C00090001C01D74
:108420002949887400BF2848807CF0218843703037
:108430002549887400BF2448C07CF02188437030EF
:108440002149C87400BF2048007D00090001C01DFB
:108450001D49087500BF1C48007DF021884370301D
:108460001949087500BF00E000BF2CE01648407DA8
:10847000F0218843144948750846007DF02188435F
:10848000114908750846007D000900010875084675
:10849000C07CF02188430C49C8740846807CF021D8
:1084A0008843094988740846807C00090001887463
:1084B0000846407D0009000148750846407CF021CF
:1084C00088430149487470BD84260020F9000020CB
:1084D000B80B000030B50246002901D1002000E0B1
:1084E0000720130008F0E8FB0F09141F2B37435037
:1084F0005D67727C88929FA9B500574B5B7EF02424
:10850000A3430401F0252C402343534C6376A1E0A0
:10851000524B9B79F024A3430401F0252C402343C4
:108520004E4CA37196E04D4B2033DB791B091B01A8
:108530000407240F2343494C2034E3718AE0464B5F
:108540002033DB7C1B091B010407240F2343424C0F
:108550002034E3747EE0404B40331B781B091B0141
:108560000407240F23433C4C4034237072E03A4B01
:108570002033DB7FF024A3430401F0252C40234368
:10858000354C2034E37765E0334B20335B7BF024BC
:10859000A3430401F0252C4023432F4C2034637364
:1085A00058E02E4B9B791B091B010407240F234322
:1085B0002A4CA3714EE0294B9B7CF024A343040179
:1085C000F0252C402343254CA37443E0234BDB7E52
:1085D0001B091B010407240F2343204CE37639E0D9
:1085E0001D4B2033DB7F1B091B010407240F234392
:1085F000194C2034E3772DE0174B9B7E1B091B01A0
:108600000407240F2343144CA37623E0134B203399
:108610009B79F024A3430401F0252C4023430F4C05
:108620002034A37116E00D4BDB7D1B091B010407F1
:10863000240F2343094CE3750CE0074B20335B7C8C
:108640001B091B010407240F2343034C20346374CC
:1086500000E000BF00BF30BD6426002038270020A6
:10866000F7B582B00746154600260024FE4800787C
:10867000012804D0F4F736FAFC49884279D2FC4844
:10868000407CF02188437030F94948740846807C6A
:1086900000090001C01D88740846007D0009000122
:1086A000C01D08750846007DF02188437030F049F0
:1086B00008750846807CF02188437030EC49887446
:1086C0000846C07C00090001C01DC8740846C07C73
:1086D000F02188437030E649C8740846407C0009A0
:1086E0000001C01D48740846407D00090001C01DFE
:1086F00048750846407DF02188437030DC49487554
:108700000846007CF02188437030D9490874084637
:10871000007C00090001C01D08740846C07BF021E0
:1087200088437030D249C873FF220A210020FBF72A
:10873000BDF8FF2213210020FBF7B8F8FF2211211A
:108740000020FBF7B3F8FF2212210020FBF7AEF860
:10875000FF220E210020FBF7A9F8FF220F210020A5
:10876000FBF7A4F8FF2210210020FBF79FF8F4E3A9
:10877000FFE7039836283DD019DC08287ED007DCB7
:10878000801E030008F098FA0635A8FCFBFAF97E73
:10879000102874D006DC092872D00D2871D00E285C
:1087A00070D1FDE333286ED03428F9D170E13F2831
:1087B0006AD00FDC3738082864D243007B449B889A
:1087C0005B009F448A009702FF025F005F00650321
:1087D000CB0318004E287BD006DC402879D04128F6
:1087E00078D04D28DCD1BBE14F2874D05028D7D1A8
:1087F0004FE100BF00BF9E48407CF02188439C4968
:1088000048740846807C0009000188740846007D91
:1088100000090001C01D08750846007DF02188434D
:108820007030934908750846807CF0218843904950
:1088300088740846C07C00090001C01DC874084641
:10884000C07CF02188438A49C8740846407C0009EE
:10885000000148740846407D00090001487508463B
:10886000407DF0218843824948750846007CF0210C
:1088700088437F4908740846007C06E0A1E2FDE3D6
:1088800037E2D2E3FBE394E028E00009000108743A
:108890000846C07BF02188437549C873FF220A212E
:1088A0000020FBF703F8FF2213210020FAF7FEFF58
:1088B00000220E211046FAF7F9FF00220F21104680
:1088C000FAF7F4FF002210211046FAF7EFFF77E2E3
:1088D000ABE110E2DDE26DE000BF00BF6448407C28
:1088E000F0218843624948740846807C00090001F1
:1088F00088740846007D00090001C01D08750846FF
:10890000007DF02188437030594908750846807C05
:10891000F0218843564988740846C07C000900014C
:10892000C8740846C07CF02188435149C874084681
:10893000407C0009000148740846407D00090001A0
:10894000C01D48750846407DF02188434849487558
:108950000846007CF0218843454908740846007C9D
:108960000009000108740846C07BF0218843404993
:10897000C873FF220A21002003E055E1EFE086E002
:1089800016E0FAF793FFFF2213210020FAF78EFF7B
:1089900000220E211046FAF789FF00220F2110460F
:1089A000FAF784FF002210211046FAF77FFF8EE7C6
:1089B00000BF00BF2E48407CF02188432C494874FA
:1089C0000846807C00090001C01D88740846007DAF
:1089D00000090001C01D08750846007DF02188438C
:1089E0007030234908750846807CF0218843703038
:1089F0001F4988740846C07C00090001C8740846F5
:108A0000C07CF02188431A49C8740846407C00099C
:108A1000000148740846407D000900014875084679
:108A2000407DF0218843124948750846007CF021BA
:108A300088430F4908740846007C00090001087447
:108A40000846C07BF02188430949C873FF220A21E8
:108A50000020FAF72BFFFF2213210020FAF726FF50
:108A600000220E21104605E0F9000020B80B00009E
:108A7000A4260020FAF71AFF00220F211046FAF769
:108A800015FF002210211046FAF710FF1FE700BF64
:108A900000BFFE48407CF0218843FC4948740846EA
:108AA000807C00090001C01D88740846007D000913
:108AB0000001C01D08750846007DF0218843703014
:108AC000F24908750846807CF0218843EF49887494
:108AD0000846C07C00090001C8740846C07CF0212B
:108AE0008843EA49C8740846407C00090001C01D5B
:108AF00048740846407D0009000148750846407DDD
:108B0000F0218843E14948750846007CF0218843FC
:108B1000DE4908740846007C000900010874084614
:108B2000C07BF0218843D949C873FF220A21002065
:108B3000FAF7BCFEFF2213210020FAF7B7FE00224D
:108B40000E211046FAF7B2FE00220F211046FAF766
:108B5000ADFE002210211046FAF7A8FEF6E300BF92
:108B6000CA48407CF0218843C84948740846807C44
:108B70000009000188740846007D0009000108759D
:108B80000846007DF02188437030C04908750846CA
:108B9000807CF0218843BD4988740846C07C000968
:108BA0000001C8740846C07CF02188437030B74982
:108BB000C8740846407C0009000148740846407D9E
:108BC0000009000148750846407DF0218843AF49FF
:108BD00048750846007CF0218843AC490874084673
:108BE000007C0009000108740846C07BF02188431E
:108BF000A649C873FF220A210020FAF757FEFF2278
:108C000013210020FAF752FE00220E211046FAF737
:108C10004DFE00220F211046FAF748FE00221021D7
:108C20001046FAF743FE91E300BF9848407CF021DC
:108C30008843964948740846807C0009000188747E
:108C40000846007D0009000108750846007DF021F6
:108C5000884370308D4908750846807CF021884330
:108C60008A4988740846C07C00090001C874084617
:108C7000C07CF02188438549C8740846407C0009BF
:108C8000000148740846407D000900014875084607
:108C9000407DF021884370307C4948750846007C4F
:108CA000F0218843794908740846007C00090001D6
:108CB00008740846C07BF02188437449C873FF22BA
:108CC0000A210020FAF7F2FDFF2213210020FAF713
:108CD000EDFD00220E211046FAF7E8FD00220F21DB
:108CE0001046FAF7E3FD002210211046FAF7DEFDE8
:108CF0002CE300BF00BF6548407CF0218843703002
:108D0000624948740846807C00090001C01D8874CF
:108D10000846007D00090001C01D08750846007D59
:108D2000F02188437030594908750846807CF0214D
:108D30008843564988740846C07C00090001C874FD
:108D40000846C07CF02188435049C8740846407CDE
:108D50000009000148740846407D0009000148757B
:108D60000846407DF0218843484948750846007C04
:108D7000F0218843454908740846007C0009000139
:108D800008740846C07BF02188434049C873FF221D
:108D90000A210020FAF78AFDFF2213210020FAF7AA
:108DA00085FD00220E211046FAF780FD00220F21DA
:108DB0001046FAF77BFD002210211046FAF776FDE7
:108DC000C4E200BF3148407CF02188432F494874F9
:108DD0000846807C0009000188740846007D00096F
:108DE000000108750846007DF0218843703027494E
:108DF00008750846807CF021884324498874084619
:108E0000C07C00090001C8740846C07CF02188437A
:108E100070301E49C8740846407C0009000148743F
:108E20000846407D0009000148750846407DF02154
:108E30008843164948750846007CF0218843134949
:108E400008740846007C0009000108740846C07BCD
:108E5000F02188430D49C873FF220A210020FAF748
:108E600025FDFF2213210020FAF720FD00220E210C
:108E70001046FAF71BFD00220F211046FAF716FDE7
:108E8000002210211046FAF711FD5FE2A42600200F
:108E900000BFFC48407CF0218843FA4948740846EA
:108EA000807C0009000188740846007D00090001EB
:108EB00008750846007DF02188437030F149087537
:108EC0000846807CF0218843EE4988740846C07CBF
:108ED00000090001C8740846C07CF0218843E949B4
:108EE000C8740846407C0009000148740846407D6B
:108EF0000009000148750846407DF0218843703024
:108F0000E04948750846007CF0218843DD49087433
:108F10000846007C0009000108740846C07BF02167
:108F20008843D849C873FF220A210020FAF7BEFC03
:108F3000FF2213210020FAF7B9FC00220E2110466F
:108F4000FAF7B4FC00220F211046FAF7AFFC00221A
:108F500010211046FAF7AAFCF8E1F8E1C948407C74
:108F6000F02188437030C74948740846807C000966
:108F70000001C01D88740846007D00090001C01D65
:108F800008750846007DF0218843BE4908750846EB
:108F9000807CF0218843BB4988740846C07C00E08F
:108FA000A9E000090001C8740846C07CF02188438C
:108FB000B449C8740846407C00090001487408465A
:108FC000407D0009000148750846407DF021884336
:108FD000AC4948750846007CF0218843A9490874CB
:108FE0000846007C0009000108740846C07BF02197
:108FF0008843A449C873FF220A210020FAF756FCCF
:10900000FF2213210020FAF751FC00220E21104606
:10901000FAF74CFC00220F211046FAF747FC002219
:1090200010211046FAF742FC90E19648407CF0216E
:109030008843944948740846807C0009000188747C
:109040000846007D0009000108750846007DF021F2
:1090500088438C4908750846807CF02188438949FB
:1090600088740846C07C00090001C8740846C07CAA
:10907000F02188438349C874084601E09EE003E17B
:10908000407C0009000148740846407D0009000149
:1090900048750846407DF02188437A49487508465E
:1090A000007CF0218843774908740846007C000959
:1090B000000108740846C07BF02188437030714974
:1090C000C87300220A211046FAF7F0FB0022132190
:1090D0001046FAF7EBFBFF220E210020FAF7E6FB21
:1090E00000220F211046FAF7E1FB00221021104662
:1090F000FAF7DCFB2AE16348407CF02188436149B0
:1091000048740846807C0009000188740846007D88
:109110000009000108750846007DF021884359497F
:1091200008750846807CF0218843564988740846B3
:10913000C07C00090001C8740846C07CF021884347
:109140005049C8740846407C00090001487408462C
:10915000407D0009000148750846407DF0218843A4
:10916000484948750846007CF02188434549087401
:109170000846007C00090001C01D08740846C07B39
:10918000F02188433F49C87300220A211046FAF7AC
:109190008DFB002213211046FAF788FB00220E21D6
:1091A0001046FAF783FBFF220F210020FAF77EFB1F
:1091B000002210211046FAF779FBC7E03148407CC5
:1091C000F02188432F4948740846807C000900013B
:1091D00088740846007D0009000108750846007D76
:1091E000F0218843274908750846807CF021884390
:1091F000244988740846C07C00090001C8740846E8
:10920000C07CF02188431F49C8740846407C00098F
:10921000000148740846407D000900014875084671
:10922000407DF0218843174948750846007CF021AD
:1092300088437030134908740846007C0009000117
:1092400008740846C07BF02188430E49C873002289
:109250000A211046FAF72AFB002213211046FAF7DA
:1092600025FB00220E211046FAF720FB00220F21D9
:109270001046FAF71BFBFF2210210020FAF716FB1D
:1092800064E00000A4260020FD48407CF0218843D3
:10929000FB4948740846807C000900018874084630
:1092A000007D0009000108750846007DF021884313
:1092B000F34908750846807CF0218843F04988749A
:1092C0000846C07C00090001C8740846C07CF02133
:1092D0008843EB49C8740846407C00090001487483
:1092E0000846407D0009000148750846407DF02190
:1092F0008843E34948750846007CF0218843E049EB
:1093000008740846007C0009000108740846C07B08
:10931000F0218843DA49C87300220A211046FAF77F
:10932000C5FA002213211046FAF7C0FA00220E21D6
:109330001046FAF7BBFA00220F211046FAF7B6FAE8
:10934000002210211046FAF7B1FA00BF00BF002F2B
:1093500003D0CC48007A002808D1F3F7C3FBCA49F0
:10936000884203D3C9480078012872D1FF22112115
:109370000020FAF79BFAFF2212210020FAF796FA52
:10938000C2480078012804D0F3F7ACFBBE498842FC
:1093900016D2BF48807BF02188437030BC49887367
:1093A000084640300078F02188437030B849403199
:1093B00008700846007800090001C01D08702DE003
:1093C0007D20C000854214D2B148807BF0218843C3
:1093D000AF498873084640300078F02188437030E8
:1093E000AB49403108700846007800090001087058
:1093F00014E0A748807BF02188437030A44988732B
:10940000084640300078F0218843A1494031087077
:109410000846007800090001C01D08707D20C000CA
:10942000854205D201462846EEF790FE064604E046
:1094300098492846EEF78AFE0646944800780128A7
:1094400004D0F3F74FFB9049884203D29248845DE1
:1094500002E0A0E29148845DE007C00F002809D037
:109460008B484030C07800090001C01D8849403158
:10947000C87007E086484030C07800090001844980
:109480004031C87002202040002807D08048C079B1
:1094900000090001C01D7E49C87105E07C48C07903
:1094A000000900017A49C87104202040002807D033
:1094B0007748807900090001C01D7549887105E071
:1094C00073488079000900017149887108202040A3
:1094D000002807D06E484079F021884370306C49ED
:1094E000487105E06A484079F0218843684948712D
:1094F00010202040002807D065484079000900016D
:10950000C01D6349487105E06148407900090001C8
:109510005F49487120202040002807D05C4800792E
:10952000F021884370305A49087105E058480079A5
:10953000F02188435649087140202040002807D078
:1095400053488079F021884370305149887105E093
:109550004F488079F02188434D4988717D20C000B3
:10956000854213D264212846EEF7F0FD06464748AF
:109570000078012804D0F3F7B5FA4349884202D2B3
:109580004548845D23E04548845D20E06421284609
:109590003230EEF7DBFD7D21C9000090EEF7D6FDFD
:1095A000019164210198EEF7D1FD06463C488542C1
:1095B00008D236480078012804D0F3F793FA3249EC
:1095C000884202D23448845D01E03448845DE0077B
:1095D000C00F002809D02E4840308078F021884301
:1095E00070302B494031887007E02948403080783E
:1095F000F02188432649403188700220204000280D
:1096000007D02348807A00090001C01D20498872D4
:1096100005E01F48807A000900011D498872042076
:109620002040002807D01A48407A00090001C01DD8
:109630001749487205E01648407A000900011449AC
:10964000487208202040002807D01148007AF021F5
:10965000884370300E49087205E00D48007AF02109
:1096600088430B4908721020204000281AD008486F
:10967000007A00090001C01D0549087218E00000C9
:10968000A4260020680A0020B80B0000F900002082
:1096900018270020A0860100EC1B0200FF1B02001F
:1096A00010270000FE48007A00090001FC490872FA
:1096B00020202040002807D0F948C079F0218843B5
:1096C0007030F749C87105E0F548C079F02188434A
:1096D000F349C87140202040002807D0F048407A64
:1096E000F02188437030EE49487205E0EC48407A3A
:1096F000F0218843EA4948727D20C000854219D292
:109700000A212846EEF722FD0A210190EEF71EFD00
:109710000E460A2D08D2E3480078012804D0F3F75A
:10972000E1F9E149884202D2E048845D12E0E04874
:10973000845D0FE0642128463230EEF707FD0A21F0
:109740000090EEF703FD0A210190EEF7FFFC0E46B4
:10975000D6498C5DE007C00F002809D0D0484030C2
:10976000807800090001C01DCD494031887007E0B4
:10977000CB484030807800090001C94940318870E9
:1097800002202040002807D0C548807B0009000146
:10979000C01DC349887305E0C148807B00090001F2
:1097A000BF49887304202040002807D0BC48407B74
:1097B00000090001C01DBA49487305E0B848407B64
:1097C00000090001B649487308202040002807D04E
:1097D000B348007BF02188437030B149087305E03D
:1097E000AF48007BF0218843AD490873102020402A
:1097F000002807D0AA48C07A00090001C01DA84966
:10980000C87205E0A648C07A00090001A449C872E0
:1098100020202040002807D0A148807AF0218843EA
:1098200070309F49887205E09D48807AF021884316
:109830009B49887240202040002807D09848407BF0
:10984000F021884370309649487305E09448407B86
:10985000F0218843924948737D20C000854207D299
:109860000A212846EEF772FC0E469048845D0BE014
:10987000642128463230EEF769FC0A210190EEF7A8
:1098800065FC0E4689498C5DE007C00F002809D0B1
:10989000834840304078F02188437030804940311F
:1098A000487007E07E4840304078F02188437C498A
:1098B0004031487002202040002809D078484030CC
:1098C000407800090001C01D75494031487007E02B
:1098D00073484030407800090001714940314870B8
:1098E00004202040002807D06D48007CF0218843E8
:1098F00070306B49087405E06948007CF0218843AA
:109900006749087408202040002807D06448007C7C
:1099100000090001C01D6249087405E06048007C30
:10992000000900015E49087410202040002807D07B
:109930005B48C07BF021884370305949C87305E00B
:109940005748C07BF02188435549C87320202040E8
:10995000002807D05248C07B00090001C01D5049B3
:10996000C87305E04E48C07B000900014C49C8732C
:1099700040202040002807D04948407C00090001D1
:10998000C01D47494874ECE04548407C000900018F
:1099900043494874E5E000220A211046F9F786FFA2
:1099A000002213211046F9F781FF002211211046F1
:1099B000F9F77CFF002212211046F9F777FF002209
:1099C0000E211046F9F772FF00220F211046F9F719
:1099D0006DFF002210211046F9F768FF3048403033
:1099E000C078000900012E494031C8702C48C07968
:1099F000000900014039C87108468079000900015A
:109A0000887108464079F021884325494871084605
:109A1000407900090001487108460079F021884327
:109A20001F49087108468079F02188431C498871D4
:109A3000084640308078F0218843194940318870C9
:109A40001748807A00090001403988720846407A38
:109A50000009000148720846007AF0218843104945
:109A600008720846007A0009000108720846C079A9
:109A7000F02188430A49C8710846407AF02188439A
:109A8000074948720846403080780009000140319B
:109A900088700348807B000900014039887309E021
:109AA00018270020F9000020B80B0000EC1B020072
:109AB000FF1B02000846407B00090001487308466E
:109AC000007BF0218843284908730846C07A0009C2
:109AD0000001C8720846807AF021884322498872C2
:109AE0000846407BF02188431F49487308464030B0
:109AF0004078F02188431C4940314870084640783E
:109B00000009000148701848007CF021884316497C
:109B100008740846007C0009000108740846C07BF0
:109B2000F02188431049C8730846C07B0009000132
:109B3000C8730846407C0009000148740846807BD1
:109B4000F021884308498873084640300078F021A6
:109B50008843054940310870084600780009000133
:109B6000087005B0F0BD000018270020F7B582B0DE
:109B700007460E460121FF200830FBF799FF01211F
:109B8000FC48FBF795FFFC48007801287ED0F2F7EF
